:100000000C94CA120C94FB120C94FB120C94FB126D
:100010000C94FB120C94FB120C94FB120C94FB122C
:100020000C94FB120C94FB120C94FB120C94FB121C
:100030000C94FB120C94FB120C94FB120C94FB120C
:100040000C94FB120C94C7930C94FB120C94FB12AF
:100050000C94FB120C94FB120C943C550C94CCA504
:100060000C94FB120C94EF300C94E5300C94FB12C2
:100070000C94FB120C94FB120C94FB120C94FB12CC
:100080000C94FB120C94FB120C94FB120C94FB12BC
:100090000C94FB120C94FB120C94FB120C94FB12AC
:1000A0000C94FB120C94FB120C94FB120C94FB129C
:1000B0000C94FB120C94FB120C94FB120C94FB128C
:1000C0000C94FB120C94FB120C94FB120C94FB127C
:1000D0000C94FB120C94FB120C94FB120C94FB126C
:1000E0000C94FB12783F7B3F6A3F6E3F743FB23FF8
:1000F0007F3F833F893F8D3F913F973F9B3F9F3F8E
:10010000B23FA53FA93FAD3F4E80BD7EF67E8A80BF
:10011000F67EF67EF67EF67EF67EF67EF67EF67E3F
:10012000F67EF67EF67EF67EF67EF67EF67EF67E2F
:10013000F67EF67EF67EF67EF67EF67EF67EF67E1F
:10014000F67EF67E8480F67EF67EF67EF67EF67E7F
:10015000F67EF67EF67E5D80F67EF67EF67EF67E96
:10016000F67EF67EF67EF67EF67EF67EA180F37E45
:10017000E6A4EBA4F0A4FAA404A57DA50EA516A5FB
:100180001EA528A532A53CA54BA555A57DA55FA517
:1001900069A573A5084AD73B3BCE016E84BCBFFD61
:1001A000C12F3D6C74319ABD56833DDA3D00C77F47
:1001B00011BED9E4BB4C3E916BAAAABE00000080E0
:1001C0003F05A84CCDB2D44EB93836A9020C50B96F
:1001D000918688083CA6AAAA2ABE000000803F009B
:1001E0000C94F7880C941F780C94768A0C94BE8635
:1001F0000C948B780C944F910C94E6A40C94893F4A
:100200000C94F67E0C94F6840C949F3F0C947378B7
:100210000C94967D0C945D800C9454910C943791C1
:100220000C94C7770C94E97B0C94567D0C94477E14
:100230000C94AC670C947E8A0C947F3F0C947DA543
:100240000C9428A50C940F8A0C9483670C94AC77BB
:100250000C946A3F0C94B23F0C9416A50C945E91DA
:100260000C944E800C94C18F0C946E3F0C94A27D24
:100270000C9423670C94E0770C94CA8F0C94EA38A2
:100280000C94E8880C9438780C94743F0C948A8011
:100290000C944A7E0C9455A50C948D780C9464783B
:1002A0000C94BF7B0C9484800C9469A50C94CB7B3C
:1002B0000C94BB860C9473A50C94BD3E0C94479093
:1002C0000C946F920C9443910C94477D0C94D17BC9
:1002D0000C94833F0C94D38F0C94F37E0C948F7802
:1002E0000C943D910C94AD3F0C94CF880C94B1AD1F
:1002F0000C94913F0C9400AE0C9436310C944BA5A9
:100300000C94E37B0C94EBA40C9437310C94037E97
:100310000C944D7E0C94D77B0C949C870C94827823
:100320000C94973F0C94C57B0C94F9770C94C18680
:100330000C94EF7B0C94FB880C945FA50C943A31E1
:100340000C947B3F0C9432A50C9468910C941EA5E0
:100350000C94A1800C94F87B0C94A53F0C9491789C
:100360000C940C780C94A93F0C949B3F0C94F0A433
:100370000C9421930C94FAA40C94FD880C94288A74
:100380000C9449910C943CA50C94F9880C944B78EE
:100390000C944D670C94BD7E0C94783F0C94639143
:1003A0000C94DD7B0C948D3F0C9404A50C940EA54D
:1003B0000C9459910C940E8C4E414E494E4954590F
:1003C000494E46CDCCCC3D0AD7233C17B7D1387720
:1003D000CC2B329595E6241FB14F0A000020410036
:1003E00000C84200401C4620BCBE4CCA1B0E5AAE80
:1003F000C59D7400407A10F35A00A0724E1809008F
:1004000010A5D4E80000E87648170000E40B540279
:100410000000CA9A3B000000E1F5050000809698B4
:1004200000000040420F000000A086010000001004
:100430002700000000E80300000000640000000046
:10044000000A00000000000100000000002C76D827
:1004500088DC674F0823DFC1DFAE59E1B1B796E50D
:10046000E3E453C63AE651997696E8E6C28426EB71
:10047000898C9B62ED407C6FFCEFBC9C9F40F2BA84
:10048000A56FA5F490055A2AF75C936B6CF9676D1C
:10049000C11BFCE0E40D47FEF520E6B500D0ED9071
:1004A0002E0300943577050080841E080000204E3E
:1004B0000A000000C80C333333330F986E128311D7
:1004C00041EF8D2114893BE65516CFFEE6DB18D1AE
:1004D000844B381BF77C1D901DA4BBE42420328480
:1004E000725E228100C9F124ECA1E53D27434F4D06
:1004F0004D554E49434154494F4E0044525952556F
:100500004E004552524F525300494E464F0045430C
:10051000484F0047322F4733206261642070617278
:10052000616D65746572730A00536C6565702E2E7B
:100530002E00436C69636B20746F20526573756D78
:10054000652E2E2E004E6F204D6F76652E00456E67
:10055000642066696C65206C6973740A0042656783
:10056000696E2066696C65206C6973740A00286E78
:100570006F2066696C65290043757272656E742020
:1005800066696C653A20005344207072696E746924
:100590006E67206279746520004E6F74205344208A
:1005A0007072696E74696E670A0044656C6574697F
:1005B0006F6E206661696C65642C2046696C653AD3
:1005C000200046696C652064656C657465643A005A
:1005D00025697920256964202569682025696D20B1
:1005E000256973005072696E742074696D653A20D4
:1005F00000496E76616C69642050696E204D6F64AD
:10060000650A0020543A300A006F6666004445428D
:1006100055473A004D3131322053687574646F7715
:100620006E004D313133205300434E43204F464638
:100630002E004348414D4245525F54454D5045526E
:100640004154555245004D4F54494F4E5F4D4F4414
:10065000455300544845524D414C5F50524F54450C
:100660004354494F4E004155544F5245504F5254F8
:100670005F53445F5354415455530050524F4D50B3
:10068000545F535550504F525400454D45524745C5
:100690004E43595F50415253455200434153455FC9
:1006A0004C494748545F4252494748544E4553537A
:1006B00000544F47474C455F4C49474854530053FB
:1006C0004F4654574152455F504F5745520042558F
:1006D000494C445F50455243454E54004C455645A5
:1006E0004C494E475F44415441005A5F50524F427B
:1006F00045004155544F4C4556454C005052494ECB
:10070000545F4A4F420050524F47524553530041A5
:1007100055544F5245504F52545F54454D5000561A
:100720004F4C554D45545249430042494E41525950
:100730005F46494C455F5452414E53464552005323
:10074000455249414C5F584F4E5F584F4646004610
:1007500049524D574152455F4E414D453A4D6172A8
:100760006C696E20322E302E352E33202847697466
:100770004875622920534F555243455F434F4445C6
:100780005F55524C3A68747470733A2F2F676974CE
:100790006875622E636F6D2F4D61726C696E46696C
:1007A000726D776172652F4D61726C696E20505267
:1007B0004F544F434F4C5F56455253494F4E3A3179
:1007C0002E30204D414348494E455F545950453ADB
:1007D000434E432045585452554445525F434F556C
:1007E0004E543A3020555549443A63656465326148
:1007F00032662D343161322D343734382D3962313F
:10080000322D6335356336326633363766660A0015
:100810002F2F2000416363656C65726174696F6E90
:100820003A2050003F4A206F7574206F6620726135
:100830006E67652028302E303120746F20302E33C3
:10084000290A0020204D61783A200020204D696E51
:100850003A2000536F667420656E6473746F707312
:100860003A200046523A0050726F746563746564B2
:100870002050696E0A00486F6D6520257325732529
:1008800073204669727374004F66667365747320D3
:100890004170706C696564004572723A20546F6FE4
:1008A000206661722100546F6F206661722066724B
:1008B0006F6D207265666572656E636520706F6925
:1008C0006E740A00454550524F4D204F4B0A00446C
:1008D0006F6E65207072696E74696E672066696CF0
:1008E000650A004D3737004D3331000E050905020A
:1008F00005FB04ED044572726F72207772697469AA
:100900006E6720746F20454550524F4D210A004DAF
:10091000656469612052656D6F766564004D65643C
:10092000696120496E7365727465640062757379DC
:100930003A2070617573656420666F7220696E700D
:1009400075740A00627573793A2070617573656415
:1009500020666F7220757365720A00627573793A4A
:100960002070726F63657373696E670A0053544F2A
:10097000505045442E20005072696E746572207389
:10098000746F707065642064756520746F20657283
:10099000726F72732E2046697820746865206572C4
:1009A000726F7220616E6420757365204D3939391C
:1009B00020746F20726573746172742E20285465E0
:1009C0006D706572617475726520697320726573EC
:1009D00065742E2053657420697420616674657295
:1009E0002072657374617274696E67290A004E6FB4
:1009F00020436865636B73756D2077697468206C3C
:100A0000696E65206E756D6265722C204C61737421
:100A1000204C696E653A2000636865636B73756D81
:100A2000206D69736D617463682C204C6173742050
:100A30004C696E653A20004C696E65204E756D629A
:100A40006572206973206E6F74204C617374204C42
:100A5000696E65204E756D6265722B312C204C617C
:100A60007374204C696E653A20004D31313000536B
:100A7000442072656164206572726F720A002121E0
:100A8000204B494C4C20636175736564206279206A
:100A90004B494C4C20627574746F6E2F70696E0AEE
:100AA000002121204B494C4C206361757365642003
:100AB000627920746F6F206D75636820696E616361
:100AC000746976652074696D65202D206375727276
:100AD000656E7420636F6D6D616E643A20006563AE
:100AE000686F3A004572726F723A00204D393220B9
:100AF000580020496E76616C69642065787472755F
:100B00006465722000363726033C3D380E2E303E99
:100B1000121A1C1824221E0800014361703A006555
:100B20006E7175657565696E672022006F6B005286
:100B30006573656E643A20004572723A207574667A
:100B40003820666F6E74206E6F7420696E697469E8
:100B5000616C697A65642E00000C0D00FE070226A8
:100B600003BC017FFE08FE08FE05080806000040E1
:100B7000F0C88888987810050808060000C0F88832
:100B800088888888F80505050600012030F830209F
:100B90000508080600002070F820202020E0050944
:100BA000090600FF2070A8A8B888887020050606EE
:100BB000060001E08CEA8C8A0A0509090600FFF8A4
:100BC000A88888888888A8F8050A0A0600FE2050A8
:100BD00050505088A8A8887003030306000340A063
:100BE00040FFFFFFFFFFFFFFFFFFFFFFFFFFFFFFD4
:100BF000FFFFFFFFFFFFFF0000000605FF010707E3
:100C000006020080808080800080030303060105C7
:100C1000A0A0A005060606000050F85050F85005A8
:100C200009090600FF2070A8A07028A870200507F9
:100C300007060000C8C8102040989805070706005E
:100C40000040A0A040A89068010303060205808030
:100C5000800309090601FF20404080808040402039
:100C60000309090601FF8040402020204040800504
:100C7000070706000020A8702070A82005050506BB
:100C800000012020F820200203030601FFC040805D
:100C9000050101060003F8020202060100C0C005BA
:100CA00007070600000810102040408005070706CF
:100CB0000000708898A8C8887003070706010040E4
:100CC000C040404040E0050707060000708808105B
:100CD0002040F8050707060000F808103008887063
:100CE00005070706000010305090F81010050707A0
:100CF000060000F880F00808887005070706000065
:100D0000304080F0888870050707060000F808105A
:100D1000102020200507070600007088887088884A
:100D200070050707060000708888780810600205C3
:100D300005060100C0C000C0C00206060601FFC0D3
:100D4000C000C0408003050506010120408040200E
:100D5000050303060002F800F803050506010180FB
:100D60004020408005070706000070881020200002
:100D7000200507070600007088B8A8B8807005072E
:100D800007060000708888F888888805070706002D
:100D900000F04848704848F00507070600007088D2
:100DA0008080808870050707060000F048484848A2
:100DB00048F0050707060000F88080F08080F805FD
:100DC0000707060000F88080F0808080050707068E
:100DD00000007088808098887005070706000088EA
:100DE0008888F8888888030707060100E0404040AB
:100DF0004040E00507070600003810101010906012
:100E00000507070600008890A0C0A0908805070786
:100E1000060000808080808080F8050707060000BB
:100E200088D8A8888888880507070600008888C8A9
:100E3000A898888805070706000070888888888831
:100E400070050707060000F08888F080808005079D
:100E50000706000070888888A890680507070600C4
:100E600000F08888F0A090880507070600007088C9
:100E70008070088870050707060000F820202020F1
:100E80002020050707060000888888888888700564
:100E90000707060000888888885050200507070645
:100EA000000088888888A8A85005070706000088E1
:100EB0008850205088880507070600008888502041
:100EC000202020050707060000F80810204080F8C1
:100ED0000309090601FFE080808080808080E005B2
:100EE000070706000080404020101008030909068B
:100EF00001FFE020202020202020E0050303060041
:100F0000052050880501010600FEF80303030601D1
:100F100005804020050505060000700878887805E2
:100F200007070600008080F0888888F00505050620
:100F300000007080808870050707060000080878A8
:100F4000888888780505050600007088F08070059F
:100F50000707060000304840E0404040050707060C
:100F600000FE7088888878087005070706000080F2
:100F700080F0888888880307070601004000C04089
:100F80004040E00409090601FE1000301010101066
:100F9000906005070706000080808890E090880335
:100FA0000707060100C04040404040E00505050637
:100FB0000000D0A8A8A8A8050505060000B0C888AC
:100FC0008888050505060000708888887005070771
:100FD0000600FEF0888888F080800507070600FE7E
:100FE00078888888780808050505060000B0C8805C
:100FF000808005050506000078807008F005070769
:101000000600002020F82020201805050506000015
:10101000888888986805050506000088888850201B
:101020000505050600008888A8A8500505050600E6
:101030000088502050880507070600FE88888850E1
:10104000204080050505060000F8102040F803093F
:10105000090601FF2040404080404040200109092E
:101060000602FF80808080808080808003090906DE
:1010700001FF8040404020404040800503030600BF
:101080000248A890FF5061757365205072696E74B4
:10109000002568753A25303268750025687564202A
:1010A00025303268753A25303268750020202020BE
:1010B000202020005072696E742041626F72746546
:1010C00064004D3235003FFFF038007030FC3020B6
:1010D000FC102078102030102C00D02E31D02F7B27
:1010E000D02F7BD02E31D02C00D020301020781083
:1010F00020FC1030FC303800703FFFF03FFFF0382C
:1011000000703186302387102787902F87D02F03D8
:10111000D02030102078102078102030102F03D0ED
:101120002F87D02787902387103186303800703F73
:10113000FFF05072696E742066726F6D204D6564A9
:101140006961004D6F76652025736D6D004D6F767A
:101150006520302E316D6D004D6F766520316D6DDF
:10116000004D6F76652031306D6D004D6F766520D6
:1011700041786973004578747275646572004D6FCB
:101180007665205A004D6F76652059004D6F766563
:1011900020580000002100240027002A002D0030E4
:1011A00000330001010000040107010A01000022D0
:1011B00000250028002B002E003100340002010021
:1011C00000050108010B0100002000230026002972
:1011D000002C002F0032000001000003010601096D
:1011E0000105050505070508080808020202020AAC
:1011F0000A080804040404010101010101010103BA
:1012000003030303030303040707070C0C0C0C0C74
:101210000C0C0C0202020206060606060606060B67
:101220000B0B0B0B0B0B0B010210202008081020DE
:101230004010204080020102010804020101020462
:101240000810204080804020100804020180040221
:101250000180402010080402010804020101020478
:101260000810204080010204081020408000000A7D
:101270000B02090C0D0E080703040100000000001A
:10128000000000000000000000000000000000005E
:10129000000000000000000000121110000000001B
:1012A000000000000000000000000000000000003E
:1012B0000000005072696E7420506175736564009F
:1012C000220A00556E6B6E6F776E20636F6D6D61D5
:1012D0006E643A202200434E432052656164792EA9
:1012E000005072696E74696E672E2E2E003B2000CE
:1012F00024F4D43050C38E20C2A24017828B7011C8
:10130000127A910D816CD90AA861E108C758660765
:10131000615143061E4B5D05C145A7041A411104E6
:10132000093D9803713931034036DB026533910280
:10133000D4305402802E1D02632CEE01752AC501A3
:10134000B028A001102781018F2564012B244B01B7
:10135000E0223401AC211F018D200D01801FFC0013
:10136000841EED00971DDF00B81CD200E61BC600EE
:10137000201BBC00641AB200B219A8000A19A00010
:101380006A189900D117910040178B00B516840098
:1013900031167E00B31579003A157300C7146F003B
:1013A00058146A00EE1366008813630025135E006C
:1013B000C7125B006C12570015125400C111510086
:1013C00070114F0021114B00D61049008D104700BD
:1013D0004610440002104200C00F4000800F3E0043
:1013E000420F3C00060F3B00CB0E3800930E370037
:1013F0005C0E3500270E3400F30D3200C10D3100B4
:10140000900D3000600D2E00320D2D00050D2C00CA
:10141000D90C2B00AE0C2900850C29005C0C270090
:10142000350C27000E0C2600E80B2400C40B24000A
:10143000A00B23007D0B23005A0B2100390B210048
:10144000180B2000F80A1F00D90A1E00BB0A1E0054
:101450009D0A1D00800A1D00630A1C00470A1B002C
:101460002C0A1B00110A1A00F7091A00DD091900DD
:10147000C4091900AB091900920917007B0918006B
:10148000630917004C0916003609160020091600DA
:101490000A091500F5081500E0081400CC0814002E
:1014A000B8081400A4081400900813007D08120066
:1014B0006B08130058081200460812003408110087
:1014C000230811001208110001081100F007100094
:1014D000E0071000D0071000C0071000B0070F0091
:1014E000A107100091070E0083070F0074070F007B
:1014F00065070E0057070E0049070E003B070D0059
:101500002E070E0020070D0013070D0006070D0023
:10151000F9060C00ED060D00E0060C00D4060C00E8
:10152000C8060C00BC060C00B0060C00A4060B009C
:1015300099060C008D060B0082060B0077060B0047
:101540006C060B0061060A0057060B004C060A00E9
:1015500042060A0038060A002E060A0024060A007F
:101560001A060A001006090007060A00FD05090010
:10157000F4050900EB050900E2050900D905090099
:10158000D0050900C7050900BE050900B50508001A
:10159000AD050800A50509009C0508009405080094
:1015A0008C050800840508007C0508007405080007
:1015B0006C050700650508005D0507005605080075
:1015C0004E050700470507004005080038050700DD
:1015D000310507002A050700230507001C05060042
:1015E000160507000F05070008050600020507009D
:1015F000FB040600F5040700EE040600E8040600FC
:10160000E2040700DB040600D5040600CF04060050
:10161000C9040600C3040600BD040600B7040600A2
:10162000B1040500AC040600A6040600A0040500F1
:101630009B04060095040500900406008A0405003A
:1016400085040500800406007A0405007504050081
:10165000700405006B0405006604050061040500C4
:101660005C04050057040500520405004D04050004
:1016700048040500430405003E0404003A04050044
:1016800035040500300404002C0405002704040080
:10169000230405001E0404001A04040016040500B7
:1016A000110404000D0404000904050004040400EE
:1016B00000040400FC030400F8030400F403040025
:1016C000F0030400EC030400E8030400E403040056
:1016D000E0030400DC030400D8030400D403040086
:1016E000D0030400CC030400C8030300C5030300B7
:1016F00024F404D9201BC40C5C0E9804C4095F02B6
:1017000065077101F405F900FB04B3004804870084
:10171000C10369005803550003034500BE023A00A7
:101720008402310053022A0029022500040220000D
:10173000E4011C00C8011900AF0117009801140052
:1017400084011300710110006101100051010E00AD
:1017500043010D0036010B002B010B0020010B0093
:10176000150109000C01090003010800FB00080035
:10177000F3000800EB000700E4000600DE000600AE
:10178000D8000600D2000600CC000500C700050006
:10179000C2000500BD000400B9000400B50004004B
:1017A000B1000400AD000400A9000400A50003007E
:1017B000A20003009F0004009B00030098000300A8
:1017C0009500020093000300900003008D000200CA
:1017D0008B000300880002008600020084000300E2
:1017E000810002007F0002007D0002007B000200F9
:1017F0007900020077000100760002007400020008
:1018000072000100710002006F0002006D00010013
:101810006C0002006A00010069000200670001001C
:101820006600010065000100640002006200010022
:1018300061000100600001005F0002005D00010026
:101840005C0001005B0001005A000100590001002A
:10185000580001005700010056000100550001002A
:101860005400010053000000530001005200010029
:1018700051000100500001004F0001004E00000027
:101880004E0001004D0001004C0001004B00000023
:101890004B0001004A00010049000100480000001F
:1018A000480001004700010046000000460001001A
:1018B0004500000045000100440001004300000015
:1018C000430001004200000042000100410000000E
:1018D00041000100400001003F0000003F00010006
:1018E0003E0000003E0001003D0000003D00010000
:1018F0003C0000003C0000003C0001003B000000F8
:101900003B0001003A0000003A00010039000000ED
:1019100039000100380000003800000038000100E4
:1019200037000000370001003600000036000000DC
:1019300036000100350000003500000035000100D0
:1019400034000000340000003400010033000000C7
:1019500033000000330001003200000032000000BC
:1019600032000100310000003100000031000100B0
:101970003000000030000000300001002F000000A7
:101980002F0000002F0000002F0001002E0000009B
:101990002E0000002E0001002D0000002D00000090
:1019A0002D0000002D0001002C0000002C00000084
:1019B0002C0000002C0001002B0000002B00000078
:1019C0002B0000002B0001002A0000002A0000006C
:1019D0002A0000002A000100290000002900000060
:1019E0002900000029000000290001002800000053
:1019F0002800000028000000280000002800010046
:101A0000270000002700000027000000270000003A
:101A1000270001002600000026000000260000002C
:101A2000260000002600010025000000250000001F
:101A30002500000025000000250000002500010011
:101A40002400000024000000240000002400000006
:101A500024000100230000002300000023000000F8
:101A600023000000230000002300000023000100E9
:101A700022000000220000002200000022000000DE
:101A800022000000220001002100000021000000CF
:101A900021000000210000002100000021000000C2
:101AA00021000100200000002000000020000000B4
:101AB00020000000200000002000000020000000A6
:101AC000200001001F0000001F0000001F00000098
:101AD0001F0000001F0000001F0000001F00010089
:101AE0001E0000001E0000001E0000001E0000007E
:101AF000043700001E290000511B00005810000090
:101B000010090000CC040000780200004101000030
:101B100020436F756E7420583A004D383420582099
:101B200059205A2045002062797465733B20637206
:101B300063200053657474696E67732053746F7209
:101B40006564202800454550524F4D206461746102
:101B500073697A65206572726F722E0A0020737441
:101B60006F7265642073657474696E677320726543
:101B7000747269657665642028004572723A204562
:101B80004550524F4D2043524300202863616C63FF
:101B9000756C6174656429210A0020213D2000458F
:101BA0004550524F4D20435243206D69736D61740F
:101BB0006368202D202873746F72656429200045A6
:101BC00072723A20454550524F4D20496E646578F7
:101BD00000496E6465783A20004572723A204545A6
:101BE00050524F4D2056657273696F6E00204D61E3
:101BF000726C696E3D563736290A00454550524F82
:101C00004D2076657273696F6E206D69736D6174B6
:101C100063682028454550524F4D3D0068747470EC
:101C20003A2F2F6D61726C696E66772E6F72670046
:101C3000322E302E352E33002020506C616E6E65B2
:101C40007242756666657242797465733A20002047
:101C500046726565204D656D6F72793A2000436F5D
:101C60006D70696C65643A204F637420323720329E
:101C70003032300A00204C617374205570646174F6
:101C800065643A20323032302D30332D3331207CB0
:101C900020417574686F723A20286E6F6E652C2033
:101CA00064656661756C7420636F6E666967290A86
:101CB00000322E302E352E330A004D61726C696E63
:101CC0000020536F66747761726520526573657486
:101CD0000A00205761746368646F672052657365FA
:101CE000740A002042726F776E206F7574205265FF
:101CF0007365740A002045787465726E616C2052B9
:101D0000657365740A00506F77657255700A0073C9
:101D1000746172740A006175746F25632E670047E1
:101D200032385859004D31303031006572726F725F
:101D30002077726974696E6720746F2066696C65BC
:101D40000A00446F6E6520736176696E672066696C
:101D50006C652E0A004D323900456E6473746F70E5
:101D600073002553202563202563202563202563E8
:101D700000656E6473746F7073206869743A200034
:101D800001FFFFFFFFFFFFFFFFFFFFFFFFFF0FFF51
:101D9000FFFFFFFFFFFFFFFFFFFFFFFF1E00000031
:101DA0000000000000000007FFFF380000000000F6
:101DB000000000000003FFFF7000000000000000B2
:101DC00000000001FFFF60000000000000000000B4
:101DD0000000FFFF600000000000000000000000A5
:101DE0007FFFC000000000000000007800003FFFFF
:101DF000C00FC0FC00000000007818001FFFC03FAB
:101E0000E1FF0000000000783C000FFFC07FF3FFFF
:101E10008000000000783C0007FFC0FFFFFFC0000B
:101E2000000000783C0003FFC1F87F87E00000005D
:101E30000078000001FFC1F03F03E00000000078DF
:101E4000000000FFC1E01E01E01F0003E0783C033A
:101E5000F07FC1E01E01E07FC00FF8783C07FC3F37
:101E6000C1E01E01E1FFE01FFC783C0FFE1FC1E056
:101E70001E01E3FFF03FFE783C1FFE0FC1E01E0194
:101E8000E3F3F83F3E783C3F3F07C1E01E01E7E047
:101E9000FC7C1F783C3E1F07C1E01E01E7C07C7C34
:101EA0000F783C3C0F03C1E01E01E7807C780F787F
:101EB0003C3C0F03C1E01E01E7803C7800783C3CCD
:101EC0000F03C1E01E01E7803C7800783C3C0F0323
:101ED000C1E01E01E7803C7800783C3C0F03C1E084
:101EE0001E01E7C03C7800783C3C0F03C1E01E01B6
:101EF000E3E03C78007C3C3C0F03C1E01E01E3FFC3
:101F00003FF8007FBC3C0F03C1E01E01E1FF3FF83A
:101F1000003FBFFC0F03C1E01E01E0FF3FF8001FC0
:101F2000BFFC0F03C1E01E01E07F3FF8000FBFFCC4
:101F30000F03600000000000000000000000000728
:101F400060000000000000000000000000067000BB
:101F500000000000000000000000000E380000003B
:101F60000000000000000000001C1E000000000037
:101F700000000000000000780FFFFFFFFFFFFFFFE1
:101F8000FFFFFFFFFFF001FFFFFFFFFFFFFFFFFF6E
:101F9000FFFFFF802053697A653A200043616E6E2F
:101FA0006F74206F70656E207375626469722000B3
:101FB00053442063617264206F6B0A006F70656E1A
:101FC000526F6F74206661696C65640A00766F6C8D
:101FD000756D652E696E6974206661696C65640A49
:101FE00000534420696E6974206661696C0A004D73
:101FF0003234004D32332025730046696C652073FE
:10200000656C65637465640A0046696C65206F7071
:10201000656E65643A2000454E4420535542524F48
:102020005554494E450A002220706F7300222070DB
:102030006172656E743A2200535542524F555449AD
:102040004E452043414C4C207461726765743A22BE
:1020500000747279696E6720746F2063616C6C2004
:102060007375622D67636F64652066696C657320A4
:102070007769746820746F6F206D616E79206C656C
:1020800076656C732E204D4158206C6576656C200A
:1020900069733A310A0057726974696E6720746F08
:1020A0002066696C653A2000667265736800646F2B
:1020B000696E67004E6F7720007C3C3E5E2B3D3F93
:1020C0002F5B5D3B2C2A225C005654726176204DBA
:1020D000696E00566D696E00566D6178205A005623
:1020E0006D6178205900566D6178205800416D610E
:1020F00078205A00416D6178205900416D61782047
:102100005800412D54726176656C00412D52657402
:102110007261637400416363656C004A756E637439
:10212000696F6E20446576005A73746570732F6D05
:102130006D005973746570732F6D6D0058737465FD
:1021400070732F6D6D00416476616E63656420531A
:10215000657474696E677300496E6974004D34323A
:102160003800496E697469616C697A65204545502B
:10217000524F4D0053746570732F6D6D004A657238
:102180006B00416363656C65726174696F6E0056C4
:10219000656C6F636974790053657420486F6D6571
:1021A000204F66667365747300526573746F726551
:1021B0002044656661756C7473004C6F61642053D4
:1021C000657474696E67730053746F72652053652C
:1021D0007474696E6773005072656865617420413C
:1021E000425320436F6E66005072656865617420CB
:1021F000504C4120436F6E6600436F6E6669677591
:10220000726174696F6E003F0043616E63656C00BC
:102210004261636B0053746F70004D32310043684C
:10222000616E6765204D656469610054656D706518
:1022300072617475726500526573756D65205072B8
:10224000696E74004E6F204D656469610054756E4F
:10225000650053746F70205072696E7400496E6629
:102260006F2053637265656E005374617274205001
:1022700072696E740043616E6E6F7420656E746572
:1022800072207375626469723A2000022E2E004D2E
:102290006F74696F6E0046616E20537065656400EF
:1022A0004D61696E004D38340044697361626C653C
:1022B0002053746570706572730047323800417541
:1022C000746F20486F6D6500000000000000000082
:1022D000000000000000FA430000FA4300009842AA
:1022E0000000484200004842000080400202040012
:1022F00000A0400000A04000000040FFFFFF576129
:10230000726E696E673A20486F6D696E672042751C
:102310006D702044697669736F72203C20310A0029
:1023200020520048617264636F646564204465668E
:1023300061756C742053657474696E6773204C6F9B
:10234000616465640A0020204D3230362058004810
:102350006F6D65206F66667365743A00204A0020D1
:10236000204D323035204200416476616E636564F1
:102370003A20423C6D696E5F7365676D656E745F90
:1023800074696D655F75733E20533C6D696E5F6661
:10239000656564726174653E20543C6D696E5F745E
:1023A000726176656C5F66656564726174653E2016
:1023B0004A3C6A756E635F6465763E002054002077
:1023C000204D323034205000416363656C6572618A
:1023D00074696F6E2028756E6974732F7332293A91
:1023E00020503C7072696E745F616363656C3E205F
:1023F000523C726574726163745F616363656C3EC5
:1024000020543C74726176656C5F616363656C3EF9
:102410000020204D3230312058004D6178696D75B3
:102420006D20416363656C65726174696F6E20280D
:10243000756E6974732F7332293A0020204D323043
:10244000332058004D6178696D756D20666565644F
:1024500072617465732028756E6974732F73293ADD
:102460000053746570732070657220756E69743ADC
:102470000020204D3134392043203B20556E6974B3
:102480007320696E2043656C736975730A00202898
:102490006D6D29002020473231202020203B20551F
:1024A0006E69747320696E206D6D006F70656E00CB
:1024B000545249474745524544007A5F6D696E0062
:1024C000795F6D696E00785F6D696E005265706F3F
:1024D0007274696E6720656E6473746F70207374B4
:1024E000617475730A00486F6D696E672046616993
:1024F0006C65640000007A440000C8420000A040FF
:102500000000C8410000C8420000C8420080C94322
:102510000000FA43C8000000C8000000640000008A
:102520001027000020453A00205A3A0020593A006E
:102530006F70656E206661696C65642C2046696CFD
:10254000653A2000506C656173652052657365744F
:10255000005052494E5445522048414C5445440085
:1025600025533A202553004B494C4C45442E20001E
:102570005072696E7465722068616C7465642E2097
:102580006B696C6C28292063616C6C6564210A009E
:1025900000AEB1AD11241FBECFEFD1E2DEBFCDBF83
:1025A00000E00CBF12E0A0E0B2E0E8E4FCE701E0EC
:1025B0000BBF02C007900D92AE3FB107D9F722E1E1
:1025C000AEEFB2E001C01D92A03CB207E1F712E10C
:1025D000C9ECD2E100E006C021970109802FFE017D
:1025E0000E9469BAC83CD10780E00807A9F70E9499
:1025F00003A80C9412BE0C9400002F923F924F92AD
:102600005F926F927F928F929F92AF92BF92CF9282
:10261000DF92EF92FF920F931F93CF93DF93CDB78B
:10262000DEB7C155D1090FB6F894DEBF0FBECDBFDE
:1026300062968FAF62972091090321962FAF219761
:1026400081E0809309038091BD038D3409F41FC29A
:10265000843511F40C944C1E873411F00C944A1EEE
:102660002090BB033090BC0334E02316310409F4FE
:102670000FC154F437FC07C28091290C52E0251693
:1026800031040CF079C02FC08AE52816310409F412
:102690004DC164F4A5E12A16310411F40C944C1ECA
:1026A000BCE12B16310409F431C1EDC1EBE52E1666
:1026B000310409F43FC1FCE52F16310409F0E3C1F0
:1026C000FEE32F2EF2E03F2EAEEDEA2EACE0FA2E26
:1026D000A1E0BDE0B9A3A8A3B1E1CB2EBDE0DB2E04
:1026E00000E010E068C1813011F00C944C1E0E9493
:1026F0009F268BEE9CE00E94C99A2AE037ED43E2C8
:102700005CE360910002709101028091020290915D
:1027100003020E94EAB36B017C0160910C0270918C
:102720000D02072E000C880B990B0E948BB39B01A6
:10273000AC01C701B6010E94EAB369837A838B8337
:102740009C83C12CD12C76018E010F5F1F4F27EF88
:102750003CE043EF5CE06FEE7CE08BEE9CE00E949F
:10276000585280E1EBEEFCE0A1E0BDE001900D925B
:102770008A95E1F70C944C1E813011F00C944C1E9C
:102780000E949F2682E50E949226882309F44EC06B
:102790000E9412266B017C0120E030E0A9010E941A
:1027A00084B3882311F40C94181F2091010D3091EB
:1027B000020D4091030D5091040D28A339A34AA3A3
:1027C0005BA38091050D9091060DA091070DB0912E
:1027D000080D8CA39DA3AEA3BFA38090EB0C90909B
:1027E000EC0CA090ED0CB090EE0C4090EF0C5090E3
:1027F000F00C6090F10C7090F20CA501940168A1AE
:1028000079A18AA19BA10E9484B381110C94591EC5
:10281000A30192016CA17DA18EA19FA10E9484B30E
:10282000882311F40C94181F0C94591E89E40E94FB
:102830009226882329F00E9412266B017C0103C096
:10284000C12CD12C76018AE40E949226882311F4AF
:102850000C941F1F0E94122668A779A78AA79BA71E
:1028600020E030E0A901C701B6010E9484B38111C4
:102870000C942C1F20E030E0A90168A579A58AA559
:102880009BA50E9484B381110C942C1F0C94181FDB
:1028900080E50E949226882329F00E94DE256B01A4
:1028A0007C0103C0C12CD12C760183E50E949226C5
:1028B000882361F00E94122620E030E04AE754E4C9
:1028C0000E94EAB30E94EDBB6B017C010E948C94D4
:1028D00080914012811105C060E089E295E00E947C
:1028E000723E0E94C0A5C60ED71EE81EF91E0E94A9
:1028F000C0A5DC01CB018C199D09AE09BF09B7FD4C
:1029000002C00C944C1E0E94D92AF1CF8091EA0C8F
:102910008770873011F00C94B72260E08FE40E943A
:10292000642781110C944C1E0C94B722109208035A
:102930000C944C1E8FE0809308030C944C1E0E9454
:1029400012262B013C01133049F0D6012D913D9107
:102950004D915C910E9479BA2B013C01E8A1F9A14B
:102960002081318142815381C301B2010E9479BA31
:102970004B015C012DEB37E346E855EB0E94DABCD6
:1029800087FD21C02DEB37E346E855E3C501B401CF
:102990000E9484B31816BCF01F5FF4E0EF0EF11C28
:1029A00028A139A12C5F3F4F39A328A334E0C30EDF
:1029B000D11C143031F1F10181911F010E94922646
:1029C000882351F3BCCF133051F440920D0D509237
:1029D0000E0D60920F0D7092100D01E0DDCFA5017C
:1029E0009401D7016D917D918D919C910E947ABA4D
:1029F000F7016083718382839383812F0E94FA9809
:102A0000CBCF0023E1F12091D4093091D509409139
:102A1000D6095091D70960910D0D70910E0D8091DE
:102A20000F0D9091100D0E94EAB30E94E7BC6093D5
:102A3000B60D7093B70D8093B80D9093B90D90912A
:102A4000940D8091950D981719F00E94FB9617C070
:102A50000E948C940E9482964091B60D5091B70DC1
:102A60006091B80D7091B90D40932A0A50932B0ACA
:102A700060932C0A70932D0A81110E948F960E94F8
:102A8000C79B0C944C1E0E9451530C944C1E809179
:102A9000BB039091BC038E36910509F466C40CF01B
:102AA000A8C08F31910509F448C30CF05CC0873190
:102AB000910509F41EC2ECF58231910509F4F8C4C0
:102AC0006CF497FF02C00C94471E823091050CF401
:102AD00094C1419709F4EEC10C94471E85319105CC
:102AE00009F4FCC10CF0FDC1449711F00C94471E91
:102AF0008DE595E00E94AC2886E79DE00E94BF74BA
:102B00008BE1E6E7FDE0DE01119601900D928A95DA
:102B1000E1F760E070E0CE0101960E94AC6DCE015D
:102B200001960E94B3768EE495E00E94AC280C9446
:102B30004C1E8B31910509F41FC23CF4893191057B
:102B400009F4F6C10CF4E9C10CC28D31910509F408
:102B500063C20CF067C28091B9039091BA030E94DE
:102B6000416C0C944C1E8335910509F49AC40CF504
:102B70008C34910509F4A5C36CF48A32910509F4EB
:102B800086C38B34910509F499C3809711F00C9496
:102B9000471EA2C28135910509F46AC40CF07AC4BB
:102BA0008D34910511F00C94471E0E940E670C9411
:102BB0004C1E8936910509F497C364F48535910557
:102BC00009F4A2C40CF474C48C35910509F4BFC493
:102BD0000C94471E8B36910509F4BAC30CF497C3C5
:102BE0008C36910511F00C94471E109250040C94F1
:102BF0004C1E833D910509F439C60CF0A6C08737F9
:102C0000910509F47FC50CF080C08237910509F465
:102C100028C53CF48037910509F402C40CF4B6C30E
:102C200005C48537910509F423C50CF031C58337F8
:102C3000910511F00C94471E8FE497E00E94AC2898
:102C400060E08FE397E00E94F33660E08AE297E06D
:102C50000E94F33661E08DE691E20E94F33660E077
:102C60008FE197E00E94F33660E08FE097E00E94EA
:102C7000F33660E086E097E00E94F33661E08CEF87
:102C800096E00E94F33660E082EF96E00E94F33611
:102C900060E08AEE96E00E94F33660E08CED96E00C
:102CA0000E94F33660E08EEC96E00E94F33660E01E
:102CB0008FEB96E00E94F33660E081EB96E00E9495
:102CC000F33660E08BE996E00E94F33660E08AE834
:102CD00096E00E94F33660E08BE796E00E94F336C0
:102CE00060E086E696E00E94F33661E083E596E0D8
:102CF0000E94F33660E086E496E00E94F33660E0DE
:102D000082E396E00E94F336C7C78B3C910509F435
:102D10002EC55CF48937910509F4FFC40CF4F5C4A1
:102D2000893C910509F400C5B2C78D3C910509F4B1
:102D300071C50CF43BC58E3C910509F0A8C726E986
:102D4000E22E2AE0F22E10E07FC5853F41E0940795
:102D500009F452C72CF58039A1E09A0709F4DEC6C0
:102D600074F4823E910509F479C68C32E1E09E0745
:102D700009F4BFC68C3D910509F089C748C68C3A55
:102D8000F1E09F0709F4CDC6843F21E0920709F4E2
:102D900030C78A39914009F07AC70E94C3277CC79F
:102DA0008C3042E0940709F446C764F4873FA1E001
:102DB0009A0709F427C70CF422C7883F914009F409
:102DC0002AC765C7873EF3E09F0709F43CC7893EE1
:102DD00023E0920709F445C7803A934009F057C7AA
:102DE0002091B9033091BA039091330F9260909380
:102DF000330FC9010E94416C4FC780E50E949226A3
:102E0000882329F00E94DE256B017C0103C0C12CC0
:102E1000D12C760183E50E949226882361F00E94DE
:102E2000122620E030E04AE754E40E94EAB30E9410
:102E3000EDBB6B017C010E948C948091B903909151
:102E4000BA03009721F061E00E94E63E05C060E011
:102E500082E395E00E94723E1091090383E0809323
:102E6000090381E080935004C114D104E104F1040A
:102E700031F00E94C0A5C60ED71EE81EF91E809133
:102E80005004882311F40C94D923C114D104E10413
:102E9000F10411F40C94D5230E94C0A5DC01CB01F0
:102EA0008C199D09AE09BF09B7FF02C00C94D52348
:102EB0000C94D9238091B50384FF02C00C94E023C5
:102EC0008091B70387FF02C00C94E0238091B80380
:102ED000837011F00C94E0230C94FC230E94BD6AD3
:102EE000DBC60E94016A8091330F877F8093330F86
:102EF000D3C6E091B903F091BA038081882329F009
:102F0000803209F410823196F8CF60E08091B903E5
:102F10009091BA030E948F6CBFC60E9448288823F4
:102F200021F00E94106A0E94EA660E941753B4C6FC
:102F30008091330F82FF03C08B7F8093330F80918A
:102F4000D304813091F782E08093D3040E94C0A51E
:102F50006093780A7093790A80937A0A90937B0A37
:102F6000E4CF8091330F83FF97C683E50E949226BA
:102F700081110C940B2490C683E40E944926882377
:102F800011F188E795E00E94AC288091200D8823FC
:102F900091F0BE016F5F7F4F8DE19DE00E948673CF
:102FA0008E010F5F1F4FD8018D918D01882339F05D
:102FB0000E94A528F8CF8EE695E00E94AC288AE012
:102FC0000E94A52869C68091330F82FF20C087E840
:102FD00095E00E94AC2860912F0F7091300F809186
:102FE000310F9091320F4AE00E942A298FE20E940D
:102FF000A52860912B0F70912C0F80912D0F90912F
:103000002E0F4AE00E942A290E94B22A45C689E969
:1030100095E00E94AC2840C68091330F8E7F80934C
:10302000330F3AC68091330F83FF36C60E943A535E
:103030008091330F83FF30C64091B9035091BA039A
:10304000BE01645E7F4F80E00E942EA28C0100973B
:1030500009F422C66C8D7D8D19821C8222E0AC01A0
:10306000CE0101960E94B976811102C0F12C14C0E4
:10307000CE0101960E949CA18823C1F361E0CE019C
:1030800001960E942E73009789F325EEFC012083A0
:103090001C820E94B66EF82ECE0101960E94B37675
:1030A000B801FF2081F082EC95E00E94BB288AE005
:1030B0000E94A52810922F0F1092300F1092310FFE
:1030C0001092320FE9C58AEA95E00E94BB2882E59A
:1030D0009DE10E94AC28E0C58091330F82FD0E94E3
:1030E0008C948091330F83FFD7C560E080E50E9408
:1030F0006427182F682F8091B9039091BA030E941A
:103100008F6C83E50E949226882381F00E94EE2531
:10311000AB01BC0140932F0F5093300F6093310FE0
:103120007093320F8DE19DE00E94A9700E94106A99
:103130001111B2C50E94EA66AFC50E949B667B0171
:103140008C0120E831E541E050E00E94DAB9C90184
:103150006DE671E00E9422BA4B015C01C801B70123
:1031600020E13EE040E050E00E94DAB9CA01B90136
:1031700028E130E040E050E00E94DAB9762E672E78
:10318000C62ED72EECE32E2E312C412C512CC8010B
:10319000B701A20191010E94DAB9F62EE72ECA0109
:1031A000B901A20191010E94DAB9CB018E010F5F32
:1031B0001F4F8114910499F0EF92FF927F936F93C8
:1031C0006F927F92BF92AF929F928F9280ED95E027
:1031D0009F938F931F930F930E941CB313C0A1144E
:1031E000B104B1F0EF92FF927F936F936F927F9251
:1031F000BF92AF9284ED95E09F938F931F930F93AF
:103200000E941CB30FB6F894DEBF0FBECDBF30C016
:10321000CD2879F0EF92FF927F936F936F927F9218
:1032200088ED95E09F938F931F930F930E941CB39B
:10323000E9CF892B69F0EF92FF927F936F938CED2A
:1032400095E09F938F931F930F930E941CB3DACF47
:10325000EF92FF9280EE95E09F938F931F930F93D1
:103260000E941CB30F900F900F900F900F900F9033
:1032700060E0C8010E94E63E0E94D228B80184EEB8
:1032800095E00E94BB288AE00E94A52805C56DE054
:1032900070E080E50E9451278C0197FDFDC4E82E67
:1032A00060E089E40E94642781110C941C24802F23
:1032B0000E9416A68111EFC30C941C240E94EA669A
:1032C000EBC48091D304813009F0E6C482E080939E
:1032D000D3040E94C0A56093780A7093790A809302
:1032E0007A0A90937B0AD8C40E94DE2987FD08C021
:1032F0008CE29BE00E94AC2883E096E00E94AC2820
:103300002196EFAD2197E09309030C94AB2580E55E
:103310000E949226811108C081E40E9449268111F1
:1033200008C06FEF70E008C00E94FE258111B4C490
:10333000F3CF6091F00470E083E50E94E0368F3FA8
:10334000910519F010F08FEF90E08093F004A4C481
:1033500080E50E949226811103C01092F0049CC463
:103360000E94FE25811198C4F8CF8EE40E94922617
:10337000882309F491C40E94EE256093420470935F
:103380004304809344049093450486C483E50E94DB
:103390004926882359F083E50E949226882319F054
:1033A0000E94FE2501C080E08093B3090E94D228CC
:1033B0008DE096E00E94AC288091B309882369F1E2
:1033C0007BEEE72E78E0F72E00E010E020E0809121
:1033D000B30990E0A0E0B0E0002E04C0B695A79538
:1033E000979587950A94D2F780FF0EC0DD24D39479
:1033F000D20E222319F08CE20E94A528F7018591B4
:1034000094910E94AC282D2D0F5F1F4FF2E0EF0E1C
:10341000F11C05301105D9F6D2CD89E096E0CDCD6D
:1034200061E084E196E00E94FAA036C483E50E9440
:103430009226882371F00E94FE25282F30E02D333C
:1034400031051CF48093040227C48CE380930402AA
:1034500023C40E94D2284091040250E060E070E052
:1034600082E296E00E9497298AE00E94A52814C46F
:103470000E940E670E949C940E94452868EE73E0AB
:1034800080E090E00E94852760E089E296E00E945B
:10349000723E02C4809108038F7D8061809308038F
:1034A000FBC3809108038F7E806280930803F4C37E
:1034B00083E50E949226882399F00E94122620E03C
:1034C00030E04AE754E40E94EAB30E94EDBB609307
:1034D0000502709306028093070290930802DCC3F2
:1034E0008091B50384FF02C00C9459248091B703E6
:1034F00087FF02C00C9459248091B803837011F0A7
:103500000C9459240C94852483E50E944926882331
:1035100009F4C2C30E94C0A5609302037093030321
:1035200080930403909305030E94122620E030E06C
:103530004AE754E40E94EAB30E94EDBB6093FE02A6
:103540007093FF028093000390930103A5C30E9430
:10355000DE2987FDA1C39091B50394FD04C090912D
:10356000B70397FF0AC05EE3C52E52E0D52E64EB89
:10357000E62E69E0F62E10E009C09091B803937032
:1035800091F7682F81E00E94772A86C3D6018D913A
:103590006D010E949226882309F459C0133009F066
:1035A0004FC00E9412264B015C0120E030E040EA4F
:1035B00051E40E9484B387FF3AC0A5019401609151
:1035C000D4097091D5098091D6099091D7090E94AC
:1035D00074BB2B013C019B01AC016091E40970912B
:1035E000E5098091E6099091E7090E94EAB36093AA
:1035F000E4097093E5098093E6099093E7096091E7
:10360000E4047091E5048091E6049091E7040E943F
:1036100089B3A30192010E94EAB30E94EDBB6093BB
:10362000E4047093E5048093E6049093E7048092A9
:10363000D4099092D509A092D609B092D70907C0B3
:103640000E941226F701648B758B868B978B1F5F08
:10365000F4E0EF0EF11C143009F098CF0E9430987E
:103660001BC30E94F89E8AEA9DE00E947E5514C307
:103670008091B9039091BA03009709F456CCDC010C
:103680002C91222309F451CC60E00E94E63E04C351
:103690000091B9031091BA0394E0F12C40E09150ED
:1036A00021F1F8018081282F2B7F213421F4218101
:1036B0002133D9F407C08035C1F4818180538A3029
:1036C00048F013C0813421F0853421F441E002C078
:1036D000FF24F39498012E5F3F4F89012F5F3F4FE6
:1036E000F80180818032C9F3DACF41110E94D228DB
:1036F000FF2021F080E198E00E94AC28C8010E94E0
:10370000B82ACAC20E944E9CC7C281E08093930A25
:103710008093920A0E946A9CBFC21092930A1092F0
:10372000920A0E946A9CB8C20E94DE2987FDB4C238
:103730004EE3E42E42E0F42E04EB19E0D7018D9124
:103740007D010E944926882359F00E9412260E947A
:10375000EDBBF80160837183828393830E9445945B
:103760000C5F1F4FF9E0043C1F0741F795C20E9410
:10377000DE2987FD91C23EE3E32E32E0F32E04EB17
:1037800019E0D7018D917D010E944926882339F0E7
:103790000E941226F80164A375A386A397A30C5F69
:1037A0001F4FF9E0043C1F0761F776C28091B60312
:1037B00087FF02C00C9488248091B7038E7011F0AB
:1037C0000C9488244091E8095091E9096091EA0934
:1037D0007091EB0984E198E00E94072A4091EC097E
:1037E0005091ED096091EE097091EF0980E293E24A
:1037F0000E94072A4091F0095091F1096091F20965
:103800007091F3098CEB93E20E94072A8AE00E94F0
:10381000A52842C28091B50381FF02C00C94CE243A
:103820008091B60381FF02C00C94CE248091B7032F
:103830008C7011F00C94CE242FC21F5FB4E0EB0EFD
:10384000F11C133009F41BC988E5810F0E94492639
:10385000882399F30E941226D7016D937D938D934F
:103860009C931397812F0E94FA98E7CF4090110DF7
:103870005090120D6090130D7090140D209117024E
:10388000309118024091190250911A02C301B201FD
:103890000E947ABA68A379A38AA39BA38090150D8E
:1038A0009090160DA090170DB090180D20911B024E
:1038B00030911C0240911D0250911E02C501B401BD
:1038C0000E947ABA6CA37DA38EA39FA3C090190D0A
:1038D000D0901A0DE0901B0DF0901C0D20911F024E
:1038E000309120024091210250912202C701B6017D
:1038F0000E947ABA68A779A78AA79BA7209123027A
:10390000309124024091250250912602C301B20158
:103910000E947ABA2B013C012091270230912802A3
:103920004091290250912A02C501B4010E947ABA3D
:103930004B015C0120912B0230912C0240912D0211
:1039400050912E02C701B6010E947ABA6B017C0128
:103950000E94D22883E598E00E94AC2883E50E946B
:103960004926982F882371F0209106033091070390
:10397000232B31F00E94FE2591E0811101C090E0DF
:1039800090932F0280912F02882319F088EF94E002
:1039900002C08BE497E00E94AC288BE498E00E9480
:1039A000AC2848A159A16AA17BA187E194E20E94B9
:1039B000072A4CA15DA16EA17FA189E891E10E9437
:1039C000072A48A559A56AA57BA582E891E10E942E
:1039D000072A82EB90E10E94AC2883E498E00E94E1
:1039E000AC28B301A20187E194E20E94072AB50145
:1039F000A40189E891E10E94072AB701A60182E8A3
:103A000091E10E94072A8AE00E94A52845C183E52A
:103A10000E949226882331F00E94EE2570930D02B9
:103A200060930C028091B5039091B603A091B70307
:103A3000B091B803892B8A2B8B2B09F02DC1609193
:103A40000C0270910D0283E698E00E94D12985E274
:103A50000E94A5288AE00E94A5281EC180E50E9438
:103A60004926882309F418C160E070E080E50E94CF
:103A70005127F82E6FEF7FEF83E50E9451278C01CD
:103A80000196039708F008C1F7FC06C18F2D0E942C
:103A900016A6882339F00E94CE2887E698E00E9477
:103AA000AC28FAC00E948C9460E08F2D0E94504395
:103AB0000F3FEFEF1E0731F00130110571F000E00C
:103AC00010E00DC08F2D0E94F84231E020E0892BDC
:103AD00009F030E0032F122F02C001E010E08F2D1B
:103AE0000E94F8428017910709F4D6C00E94D92A93
:103AF000F6CF64E071E083E50E94E0368C0168EE69
:103B000073E080E50E94E0368938F3E19F0710F00A
:103B100088E893E1B8010E94453EBEC00E948C94A3
:103B2000BBC09091EA0C90FD02C087E001C086E026
:103B300091FD8D7F9E012F5F3F4F190192FF87C737
:103B40008B7F09F0B1C708EC12E241E05DE059A3B8
:103B500048A39BEFC92E92E2D92E7901F801659115
:103B6000759185919491A8A1B9A18D909D90AD90EA
:103B7000BD90B9A3A8A3A50194010E9479BA2B0115
:103B80003C01F701608371838283938320E030E0FE
:103B900040EA51EC0E94DABC87FD0AC020E030E028
:103BA00040EA51E4C301B2010E9484B318162CF418
:103BB000F601849118160CF47AC7D7018D909D9068
:103BC000AD90BD907D0120E030E040EA51ECC501B0
:103BD000B4010E94DABC87FD75C720E030E040EAFE
:103BE00051E4C501B4010E9484B318160CF07EC7DD
:103BF00069C70E94B15C50C00E946B9E4DC00E947C
:103C0000C49D4AC061E083E50E94642791E0892752
:103C10000E94759C41C081E08093FB0C0E94426130
:103C20001092FB0C8823C1F10E94D22884EC98E00A
:103C30000E94AC2831C08091330F82FF2DC0806478
:103C40008093330F29C081E08093290C10924F0498
:103C500060E083E50E94642781111EC00E94BC348D
:103C60001BC00E949B666D3371058105910520F094
:103C700087EE98E00E940D3783EE98E00E940D37A2
:103C80008FEC98E00E94AC280E949C9405C00E9492
:103C9000515302C00E9451536296FFAD6297F111D9
:103CA00002C00E94AC3421962FAD219720930903C6
:103CB00052C711E032E02316310409F010E020E091
:103CC00030E0A901C701B6010E9484B3881F88278C
:103CD000881F1813A4C020E030E040E85FE328A765
:103CE00039A74AA75BA728A139A14AA15BA1C501B1
:103CF000B4010E9479BA20E030E040E05FE30E9426
:103D0000EAB368A379A38AA39BA32CA13DA14EA1EA
:103D10005FA1C301B2010E9479BA20E030E040E027
:103D20005FE30E94EAB36CA37DA38EA39FA328A1A7
:103D300039A14AA15BA1CA01B9010E94EAB34B01B2
:103D40005C012CA13DA14EA15FA1CA01B9010E9455
:103D5000EAB39B01AC01C501B4010E947ABA0E948A
:103D600028BD4B015C019B01AC01C701B6010E945B
:103D700079BA2B013C01A5019401C701B6010E944B
:103D80007ABA9B01AC01C301B2010E94EAB36B0194
:103D90007C0120E030E0A9010E94DABC87FD07C069
:103DA000C701B6010E9428BD2B013C0103C0412C74
:103DB000512C32016CA17DA18EA19FA19058A5012B
:103DC00094010E9474BB28A539A54AA55BA50E9451
:103DD000EAB3A30192010E94EAB328A139A14AA142
:103DE0005BA10E947ABA6B017C01A501940168A1D4
:103DF00079A18AA19BA10E9474BB28A539A54AA5D7
:103E00005BA50E94EAB3A30192010E94EAB32CA130
:103E10003DA14EA15FA10E947ABA0C942C1480E0BF
:103E200090E0A0E8BFEB88A799A7AAA7BBA75BCFA4
:103E30000E94CE2883E195E00E94AC282DCF20E09F
:103E400030E0A901C701B6010E9484B3882381F341
:103E500018A619A61AA61BA6A7019601505828A3B2
:103E600039A34AA35BA388A599A5AAA5BBA5B05869
:103E70008CA39DA3AEA3BFA3CA01B9010E94EAB35C
:103E80004B015C012CA13DA14EA15FA1CA01B9016A
:103E90000E94EAB39B01AC01C501B4010E947ABA49
:103EA0000E9428BD6CAF7DAF8EAF9FAF2091010DFA
:103EB0003091020D4091030D5091040D2CA73DA7A8
:103EC0004EA75FA7A70196016CA57DA58EA59FA50E
:103ED0000E947ABA25966CAF7DAF8EAF9FAF2597C3
:103EE0008091050D9091060DA091070DB091080DE0
:103EF00088AB99ABAAABBBAB9C01AD0168A579A51A
:103F00008AA59BA50E947ABA29966CAF7DAF8EAF29
:103F10009FAF29972091EB0C3091EC0C4091ED0C68
:103F20005091EE0C2CAB3DAB4EAB5FAB25962CAD60
:103F30003DAD4EAD5FAD25976CA97DA98EA99FA91A
:103F40000E9479BA6B017C018091EF0C9091F00C8A
:103F5000A091F10CB091F20C88AF99AFAAAFBBAFB2
:103F600029962CAD3DAD4EAD5FAD2997BC01CD017D
:103F70000E9479BA4B015C01A701960168A179A161
:103F80008AA19BA10E94EAB32B013C01A5019401E7
:103F90006CA17DA18EA19FA10E94EAB39B01AC01FF
:103FA000C301B2010E947ABA2B013C01A501940120
:103FB00068A179A18AA19BA10E94EAB34B015C018F
:103FC000A70196016CA17DA18EA19FA10E94EAB3D9
:103FD0009B01AC01C501B4010E9479BAA301920111
:103FE0000E94F9BA6B017C0120E030E0A9010E9437
:103FF00084B387FF0AC02BED3FE049EC50E4C701D2
:10400000B6010E947ABA6B017C012BED3FE049ECCE
:1040100050E4C701B6010E9474BB20E030E040ECE0
:1040200051E40E94EAB30E9458BB0E94EDBB8B0191
:10403000672B11F401E010E032E02316310451F453
:104040002BED3FE049EC50E4C701B6010E9479BA7C
:104050006B017C0120E030E0A901C701B6010E949C
:1040600084B3811122C02CA93DA94EA95FA96CA5DA
:104070007DA58EA59FA50E9484B3811116C028AD91
:1040800039AD4AAD5BAD68A979A98AA99BA90E94FF
:1040900084B381110AC008E110E02BEDC22E2FE09D
:1040A000D22E29ECE22E20E4F22E8091090D90917F
:1040B0000A0DA0910B0DB0910C0D88AB99ABAAAB7A
:1040C000BBAB9C01AD016091F30C7091F40C80913D
:1040D000F50C9091F60C0E9479BA2B013C01A701D6
:1040E00096016CAD7DAD8EAD9FAD0E94EAB34B01E4
:1040F0005C0120E030E0A901C301B2010E9484B359
:104100008823C9F0A5019401C501B4010E94EAB356
:104110004B015C01A3019201C301B2010E94EAB309
:104120009B01AC01C501B4010E947ABA0E9428BD6E
:104130004B015C010DC020E030E0A901C501B401D4
:104140000E94DABC87FF04C0B7FAB094B7F8B09405
:104150002FE632E143E85AE3C501B4010E9484B37B
:1041600087FDFAC12091F70C3091F80C4091F90CC1
:104170005091FA0C28AF39AF4AAF5BAF80910D0D6B
:1041800090910E0DA0910F0DB091100D8CAB9DABC9
:10419000AEABBFAB2AE037ED43E25CE360910002D7
:1041A0007091010280910202909103020E94EAB391
:1041B0006CA77DA78EA79FA760910C0270910D023E
:1041C000072E000C880B990B0E948BB39B01AC014E
:1041D0006CA57DA58EA59FA50E94EAB36C8F7D8FEF
:1041E0008E8F9F8FC501B4010E941CBC0E94EDBB45
:1041F0001B016017710708F41801B10180E090E01D
:104200000E9489B34B015C019B01AC01C701B6015F
:104210000E9474BB6CA77DA78EA79FA7A5019401E0
:10422000C301B2010E9474BB2D966CAF7DAF8EAFFF
:104230009FAF2D972CA93DA94EA95FA968AD79AD77
:104240008AAD9BAD0E9479BAA50194010E9474BB0E
:1042500061966CAF7DAF8EAF9FAF61972CA53DA5EA
:104260004EA55FA5CA01B9010E94EAB320E030E083
:1042700040E05FE30E94EAB39B01AC0160E070E0C4
:1042800080E89FE30E9479BA68AF79AF8AAF9BAFAD
:1042900028A939A94AA95BA929873A874B875C874E
:1042A0008CA99DA9AEA9BFA98D879E87AF87B88B22
:1042B0000E94C0A59B01AC0128533F4F4F4F5F4F59
:1042C0002CAF3DAF4EAF5FAF48A059A06AA07BA016
:1042D00041E050E059AB48AB59E15CAB88A999A9E2
:1042E0008215930508F00FC10E9474550E94C0A565
:1042F000DC01CB012CAD3DAD4EAD5FAD821B930B10
:10430000A40BB50BB7FD0EC00E94C0A59B01AC016C
:1043100028533F4F4F4F5F4F2CAF3DAF4EAF5FAF76
:104320000E94D92A3CA931503CAB3323E9F12CA19E
:104330003DA14EA15FA168AD79AD8AAD9BAD0E9454
:10434000EAB36B017C019201A3016CA57DA58EA54A
:104350009FA50E94EAB3A70196010E947ABA7B0149
:104360008C019201A30168AD79AD8AAD9BAD0E942D
:10437000EAB34B015C012CA13DA14EA15FA16CA54C
:104380007DA58EA59FA50E94EAB39B01AC01C50146
:10439000B4010E9479BA2B013C01C701D8018CA35A
:1043A0009DA3AEA3BFA34FC048A959A9BA0180E0FD
:1043B00090E00E9489B32CA53DA54EA55FA50E9463
:1043C000EAB34B015C010E946FBB6B017C01C5012C
:1043D000B4010E941ABD4B015C01A701960168A1BE
:1043E00079A18AA19BA10E94EAB32B013C01A501FE
:1043F000940168A579A58AA59BA50E94EAB3A301AB
:1044000092010E947ABA2B013C01A501940168A196
:1044100079A18AA19BA10E94EAB34B015C01A7018B
:10442000960168A579A58AA59BA50E94EAB39B0180
:10443000AC01C501B4010E9479BA6CA37DA38EA31F
:104440009FA359E15CAB9201A30125966CAD7DADB4
:104450008EAD9FAD25970E947ABA69837A838B834C
:104460009C832CA13DA14EA15FA129966CAD7DAD91
:104470008EAD9FAD29970E947ABA6D837E838F831C
:1044800098872D962CAD3DAD4EAD5FAD2D976985CE
:104490007A858B859C850E947ABA69877A878B8713
:1044A0009C8761962CAD3DAD4EAD5FAD61976D853E
:1044B0007E858F8598890E947ABA6D877E878F87DF
:1044C000988BCE0101960E94C99AC12CD12C90E8FC
:1044D000E92E9FE3F92E8E01045E1F4F9E01235F9C
:1044E0003F4FAE01475F5F4FBE016B5F7F4FCE0115
:1044F00001960E945852882331F088A999A9019603
:1045000099AB88ABEBCE80E1EBEEFCE0DE011196DF
:1045100001900D928A95E1F7CE0101960E94C99A09
:10452000C12CD12C76018E01045E1F4F9E01235FAA
:104530003F4FAE01475F5F4FBE016B5F7F4FCE01C4
:1045400001960E94585280E1FE013196A1E0BDE043
:1045500001900D928A95E1F70E94C0A56093020335
:1045600070930303809304039093050395CB0E94FB
:104570008C948091000290910102A0910202B0916E
:10458000030280930C0390930D03A0930E03B0934A
:104590000F0380910C0290910D0290930B03809376
:1045A0000A0384E690E090930D0280930C0281E070
:1045B0008093930A0E946A9C88E50E944926182FDE
:1045C00089E50E944926082F8AE50E944926101392
:1045D000EAC0181711F0012FE6C001E011E0332402
:1045E000339480E1E1E0FDE0ABEEBCE001900D92A0
:1045F0008A95E1F782E50E949226882369F00E945D
:1046000012266B017C0120E030E0A9010E9484B3F6
:10461000882309F495C006C0C12CD12C80EAE82E6D
:1046200080E4F82E111103C0002309F493C0809197
:10463000950A82FD09C06091090D70910A0D809163
:104640000B0D90910C0D03C060E070E0CB01A70151
:1046500096010E947ABA2B013C016093F30C70938F
:10466000F40C8093F50C9093F60C2091090D309189
:104670000A0D40910B0D50910C0D0E94DABC1816DA
:104680000CF05EC08090010D9090020DA090030D83
:10469000B090040DC090050DD090060DE090070D70
:1046A000F090080DE8EEF2E285919591A591B49114
:1046B0008C8F9D8FAE8FBF8F85E595E5A5E0B3E428
:1046C00089839A83AB83BC834092090D50920A0D73
:1046D00060920B0D70920C0DCE014C960E946A9B5D
:1046E0008092010D9092020DA092030DB092040DE4
:1046F000C092050DD092060DE092070DF092080DC4
:10470000CE0101960E946A9B2091090D30910A0DFD
:1047100040910B0D50910C0DC301B2010E9484B366
:1047200087FF0CC04092090D50920A0D60920B0D4C
:1047300070920C0DCE014C960E946A9B0E948C9444
:10474000112319F080E00E941A99002319F081E0EA
:104750000E941A99332019F082E00E941A990E944F
:10476000859B8091920A8093930A80910C0390918B
:104770000D03A0910E03B0910F038093000290935C
:104780000102A0930202B093030280910A03909168
:104790000B0390930D0280930C0283E080930E0232
:1047A0000E94C79B79CA382E1CCF0E94D92A0C942C
:1047B0003F1710925004109309030E9417536CCABC
:1047C00088E50E944926882311F05F98129889E5B0
:1047D0000E944926882311F08A9847988AE50E940A
:1047E0004926882329F08091080181708093060171
:1047F00085E40E94492650CA60E085E495E00E9465
:10480000723E5F9812988A9847988091080181704B
:104810008093060141CA0E94EE25AB01BC01409382
:104820002F0F5093300F6093310F7093320F8DE143
:104830009DE00E94A97030CA8DE40E9492268823D0
:10484000D9F00E94FE25813069F038F0823079F489
:1048500062E0802F0E9450431FCA60E0802F0E94B8
:1048600050431ACA61E0802F0E94504315CA81EF5D
:1048700095E00E94AC2810CA83E50E949226882306
:1048800009F40ACA0E94FE25F82EB8E0EB1203C014
:104890008093F00401CA61E0802F0E9450436F2D85
:1048A000802F0E9421436F2D70E0802F0E94BDA4B5
:1048B000F3C90E948C9488E50E944926882339F028
:1048C0005F9A129A8091950A8E7F8093950A89E566
:1048D0000E944926882339F08A9A479A8091950A3E
:1048E0008D7F8093950A8AE50E944926882309F4E2
:1048F0007FCF80910801809581708093060180911F
:10490000950A8B7F8093950A73CF0E949C94C4C9AB
:1049100083E50E949226882391F00E9412266093DC
:10492000E8097093E9098093EA099093EB09609391
:10493000F0097093F1098093F2099093F30980E5EF
:104940000E949226882351F00E9412266093E80963
:104950007093E9098093EA099093EB0982E50E943C
:104960009226882351F00E9412266093EC097093DE
:10497000ED098093EE099093EF0984E50E94922659
:10498000882309F489C90E9412266093F009709364
:10499000F1098093F2099093F3097EC982E40E94A1
:1049A0004926882351F00E94DE256093C409709344
:1049B000C5098093C6099093C70983E50E944926DB
:1049C000882351F00E9412266093F4097093F50930
:1049D0008093F6099093F70984E50E94492688237D
:1049E00051F00E9412266093F8097093F9098093A0
:1049F000FA099093FB098AE40E944926882309F466
:104A00004BC90E9412266B017C012AE037ED43E27C
:104A10005CE30E94DABC87FD13C02AE939E949E961
:104A20005EE3C701B6010E9484B318164CF0C09231
:104A3000D404D092D504E092D604F092D7042CC9C5
:104A40000E94CE2884E298E00E94AC2825C92FED70
:104A500032E081FF03C041EE52E002C04DEF52E070
:104A600080FF03C083EE92E002C08DEF92E03F939F
:104A70002F935F934F939F938F9386E798E09F9335
:104A80008F933F922F920E941CB30E94D228C101A3
:104A90000E94B82A60E0C1010E94E63E0FB6F89479
:104AA000DEBF0FBECDBFF8C82DEF32E0D2CFB7FAD0
:104AB000B094B7F8B094D7018D929D92AD92BC920C
:104AC00013977BC80E94CE2886EA98E00E94AC2803
:104AD00061E088E998E00E94723E0E94F18068E2FD
:104AE00070E088EC90E00E94453ED6C80C5F1F4FF6
:104AF000BFEFCB1ADB0AE2E2043D1E0709F02EC825
:104B000086E9E82E8AE0F82E10E0F101819191917A
:104B1000A191B1911F01F70181939193A193B19359
:104B20007F01812F0E94FA981F5F133071F70E9456
:104B3000C79B60E088E898E00E94723E63E972E0FB
:104B400084E690E00E94453E6AEB72E084E690E0E5
:104B50000E94453EA1C8CF5ADF4F0FB6F894DEBF82
:104B60000FBECDBFDF91CF911F910F91FF90EF90BE
:104B7000DF90CF90BF90AF909F908F907F906F907D
:104B80005F904F903F902F900895282F80910803B9
:104B9000233021F485FD0EC084FD0EC090E0A0E01E
:104BA000B0E004C0B695A795979587952A95D2F75A
:104BB0008170089581E0089580E008958091060352
:104BC00090910703009731F04AE050E060E070E018
:104BD0000C94A8B160E070E0CB01089580910603C9
:104BE00090910703009731F04AE050E060E070E0F8
:104BF0000C947AB060E070E0CB0108950E94EE253D
:104C000097FD0CC00E94EE256F3F7105810591054F
:104C100009F034F40E94EE25862F089580E008956F
:104C20008FEF08950F931F93CF9380910603909178
:104C30000703009711F1FC018F01C1912C2F2F7DEB
:104C4000A9F0C53411F0C536B9F7F801108260E05B
:104C500070E080910603909107030E941EAFF80157
:104C6000C083562F472F382F292F0BC060E070E0EC
:104C7000CF911F910F910C941EAF50E040E030E0B7
:104C800020E0652F742F832F922FCF911F910F91CA
:104C9000089581548A3108F042C0E82FF0E0409135
:104CA000B5035091B6036091B7037091B80304C087
:104CB00076956795579547958A95D2F7842F817099
:104CC00040FF2FC0E556FC4F9081992309F1E091F8
:104CD000A904F091AA04E90FF11D908120ED290F9C
:104CE0002A3098F09E3211F491810CC09D3211F05F
:104CF0009B3271F4918120ED290F2A3030F09E32E1
:104D000039F4928190539A3018F42E2F9F2F02C0BD
:104D100020E090E02093060390930703089580E03D
:104D2000089508950E944926882341F081E020914A
:104D3000060330910703232B09F480E008958F9236
:104D40009F92AF92BF92CF92DF92EF92FF920F931A
:104D50001F93CF938BEEE82E8CE0F82E01E01DE040
:104D600091E1C92E9DE0D92EC0E088E58C0F0E940C
:104D70009226882311F10E9412264B015C018C2F90
:104D80000E94C525882351F0F8012081318142819C
:104D90005381C501B4010E947ABA09C0F60120818D
:104DA000318142815381C501B4010E9479BAF70172
:104DB00060837183828393830AC0F801808191812B
:104DC000A281B381F70180839183A283B383CF5FF4
:104DD000F4E0EF0EF11C0C5F1F4F84E0C80ED11CF5
:104DE000C33019F685E40E949226882301F10E94BF
:104DF00012266B017C0183E00E94C525882371F097
:104E000020910D0D30910E0D40910F0D5091100D10
:104E1000C701B6010E947ABA6B017C01C092F70CFF
:104E2000D092F80CE092F90CF092FA0C10C080913C
:104E30000D0D90910E0DA0910F0DB091100D80935E
:104E4000F70C9093F80CA093F90CB093FA0C86E44D
:104E50000E9492268823C9F00E94122620E030E0AA
:104E6000A9010E94DABC181684F40E94122620E0E0
:104E700030E040E752E40E9474BB609300027093FC
:104E800001028093020290930302CF911F910F9130
:104E9000FF90EF90DF90CF90BF90AF909F908F905A
:104EA0000895CF93DF93D62FC72F0E949226882391
:104EB00029F00E94EE25262F972F02C02D2F9C2F20
:104EC000822FDF91CF910895CF93DF93D82FC62FF4
:104ED0000E949226882379F080910603909107031F
:104EE000892B11F461E00DC00E94FE2561E0811163
:104EF00008C060E006C08D2F0E9449268111F2CFC4
:104F00006C2F862FDF91CF910895CF92DF92EF9291
:104F1000FF926B017C0183E3C816D104E104F10424
:104F200070F082E3C81AD108E108F10862E370E08A
:104F300080E090E00E9486A50E947455ECCFC701E6
:104F4000B6010E9486A5FF90EF90DF90CF900C9461
:104F500074555F9A129A8091950A8E7F8093950A74
:104F60008A9A479A8091950A8D7F8093950A8091BD
:104F7000080180958170809306018091950A8B7F4E
:104F80008093950A08954F925F926F927F928F92CD
:104F90009F92AF92BF92CF92DF92EF92FF920E94C8
:104FA0008296F82E8091950D8093940D8093930DA9
:104FB0008093920D84E68093910D0E94959688EEE1
:104FC00093E09093B2098093B109F1100E948F96FB
:104FD00081E08093110A0E948C9481E00E94A6983F
:104FE0004B015C0180E00E94A6982B013C0160937C
:104FF0001303709314038093150390931603809208
:10500000170390921803A0921903B0921A0382E03A
:105010000E94A6986B017C0160931B0370931C0394
:1050200080931D0390931E0383E00E94A6984092F4
:10503000010D5092020D6092030D7092040D80924A
:10504000050D9092060DA092070DB092080DC0922A
:10505000090DD0920A0DE0920B0DF0920C0D6093A9
:105060000D0D70930E0D80930F0D9093100DFF900A
:10507000EF90DF90CF90BF90AF909F908F907F90F8
:105080006F905F904F900C94859B1092F004089560
:105090009091330F93FB882780F993FF06C081E03E
:1050A0009091200D911101C080E008958091D3046A
:1050B000823061F00E944828882349F08091330FA4
:1050C00082FB882780F991E08927089581E008957F
:1050D0008F929F92AF92BF92CF92DF92EF92FF9208
:1050E0000F93CF93DF931F92CDB7DEB75C016B01B7
:1050F0007A014901F501808191810E94B4B98983C7
:10510000002311F0F6018083BE016F5F7F4FC40161
:105110000E94E09EF50180819181019691838083B8
:10512000FFEFCF1ADF0A81E0E81AF10819F780E0F3
:105130000F90DF91CF910F91FF90EF90DF90CF9084
:10514000BF90AF909F908F9008959091C00095FF71
:10515000FCCF8093C6000895CF93DF93FC01849128
:10516000EF012196882321F00E94A528FE01F7CFA8
:10517000DF91CF9108950F931F93CF93DF938B010E
:105180000E94AC28E8018991882319F00E94A52883
:10519000FACFDF91CF911F910F91089584EE9AE09D
:1051A0000C94AC288EED9AE00C94AC287F928F92F0
:1051B0009F92AF92BF92CF92DF92EF92FF920F93A6
:1051C0001F93CF93DF931F92CDB7DEB77C015901B8
:1051D0008B016B01C40ED51E0C151D0559F1F7018D
:1051E00080809180F80171908F017982C4010E94C2
:1051F000B4B9781691F0672DC4010E94BCB9C401FE
:105200000E94B4B99981891741F00E94D22885EF94
:1052100098E00E94AC2881E00EC0BE016F5F7F4F16
:10522000C5010E94E09EF7018081918101969183E2
:105230008083D2CF80E00F90DF91CF911F910F91AB
:10524000FF90EF90DF90CF90BF90AF909F908F90A6
:105250007F9008958F929F92AF92BF92EF92FF92AC
:105260000F931F93CF93DF93CDB7DEB7A0970FB601
:10527000F894DEBF0FBECDBF6115710581059105A4
:1052800091F100E0842E912CA12CB12C102FEE2452
:10529000E394F12CEC0EFD1EE00EF11C07FDFA94D8
:1052A000A50194010E94DAB9F7016083B901CA012E
:1052B0000F5F611571058105910541F71F3F31F1C0
:1052C000E1E0F0E0EC0FFD1FE10FF11D17FDFA9595
:1052D00080818A3010F097E301C090E3890F0E942B
:1052E000A5281150EBCF80E3A0960FB6F894DEBF4F
:1052F0000FBECDBFDF91CF911F910F91FF90EF9027
:10530000BF90AF909F908F900C94A528A0960FB659
:10531000F894DEBF0FBECDBFDF91CF911F910F91EB
:10532000FF90EF90BF90AF909F908F900895CF9295
:10533000DF92EF92FF926A017B010E94AC284AE063
:10534000C701B601FF90EF90DF90CF900C942A290F
:10535000CF93DF93EB010E94AC28BE0180E090E088
:105360004AE0DF91CF910C942A29CF92DF92EF92FD
:10537000FF926B017C0197FF0BC08DE20E94A52874
:10538000F094E094D094C094C11CD11CE11CF11C99
:105390004AE0C701B601FF90EF90DF90CF900C94E8
:1053A0002A29CF93DF93EB010E94AC28BE01DD0FC9
:1053B000880B990BDF91CF910C94B529CF9384E59D
:1053C0000E949226882301F10E94FE25C82F87FDA6
:1053D0001CC00E94D2288DE40E94A5286091BB03C6
:1053E0007091BC03072E000C880B990B0E94B52905
:1053F0006C2FCC0F770B82EF9AE00E94D1298AE0C4
:105400000E94A5288FEF01C080E0CF9108958F9270
:105410009F92AF92BF92CF92DF92EF92FF926A017A
:105420007B010E94AC2820E030E0A901C701B60151
:105430000E9484B387FF07C08DE20E94A528F7FA77
:10544000F094F7F8F0942BE037ED43EA5BE3C70103
:10545000B6010E947ABA4B015C010E94EDBB6B0160
:105460007C010E9489B39B01AC01C501B4010E947B
:1054700079BA4B015C014AE0C701B6010E942A29B2
:105480008EE20E94A52820E030E040E251E4C50110
:10549000B4010E94EAB34B015C010E94E6BB6B01C0
:1054A000770FEE08FF08C701B6010E94B529C701B2
:1054B000B6010E948BB39B01AC01C501B4010E94EF
:1054C00079BA20E030E040E251E40E94EAB30E9461
:1054D000E6BB072E000C880B990BFF90EF90DF9036
:1054E000CF90BF90AF909F908F900C94B529882358
:1054F00019F00E94D22803C080E20E94A5284091A2
:10550000C8095091C9096091CA097091CB098BEE05
:105510009AE00E94072A4091CC095091CD096091F0
:10552000CE097091CF0989E891E10E94072A409144
:10553000D0095091D1096091D2097091D30982E8C4
:1055400091E10E94072A4091D4095091D5096091B8
:10555000D6097091D70983E29BE10E94072A8AE06D
:105560000C94A5288DE00E94A5288AE00C94A5281B
:10557000CF93DF93EC018991882319F00E94A5282D
:10558000FACFDF91CF910C94B22A8091BE03909113
:10559000BF03981759F0E92FF0E0E254FC4F8281E5
:1055A0009F5F9F779093BF0390E008958FEF9FEFE9
:1055B00008954F925F926F927F928F929F92AF92D7
:1055C000BF92CF92DF92EF92FF920F931F93CF93F0
:1055D000DF9300D01F921F92CDB7DEB70E94C0A507
:1055E0004B015C01809116028F3FD1F00E94C0A553
:1055F0000091CE0C1091CF0C2091D00C3091D10C99
:10560000DC01CB01801B910BA20BB30BB7FD08C0D3
:105610008091940D9091950D8F5F8F70891337C590
:105620000E94093F80914A0482FF39C0809129037A
:10563000811137C091E090932903209150042111EA
:1056400003C080919A0C89278093830410925004A0
:1056500083E080930E0210924A040E94C0A5DC01F0
:10566000CB018C509E4FAF4FBF4F80934B04909314
:105670004C04A0934D04B0934E0468E873E182E0BB
:1056800090E00E94453E16E0115059F00E94E43D22
:1056900062E070E080E090E00E9486A5F5CF109275
:1056A000290380910901817091E098271091D90C0C
:1056B0001917A9F19093D90C811113C564EF71E00A
:1056C00080E090E00E9485270E94BD6A123009F0B8
:1056D00002C510921A0E0E94F26981E0809348047C
:1056E00086EC90E19093FE0C8093FD0C1092000DDF
:1056F0001092FF0C83E080930E020E94C0A54B0124
:105700005C01DC01CB018C599F4FAF4FBF4F8093A1
:10571000250390932603A0932703B0932803809139
:10572000250390912603A0912703B09128039501AA
:105730008401081B190B2A0B3B0B37FF05C0809116
:10574000CD0C882309F471C1D501C4018C599F4F38
:10575000AF4FBF4F8093250390932603A093270359
:10576000B093280360914904062E000C770B77FF55
:1057700003C0719561957109062E000C770B880B9B
:10578000990B0E948BB32B013C0120E030E040E8F4
:1057900050E40E94DABC87FF06C08091830488230E
:1057A00009F494C082C080918904882309F456C00A
:1057B000C0907F04D0908004E0908104F090820437
:1057C000C114D104E104F104E1F120E030E040E84B
:1057D0005EE3C301B2010E94EAB32B013C01C501A3
:1057E000B4016C197D098E099F090E9489B39B0140
:1057F000AC01C301B2010E9474BB20E030E04AE773
:1058000054E40E94EAB36B017C0120E030E040EAFE
:1058100052E40E94DABC87FF0FC020E030E040EF86
:1058200051E4C701B6010E94DABC87FD0AC02AE034
:1058300030E040E050E009C024E630E040E050E0D5
:1058400004C021E030E040E050E080927F0490927C
:105850008004A0928104B092820404C021E030E070
:1058600040E050E0A09149040A2E000CBB0B0E94BE
:1058700071BA24E030E040E050E00E944ABA8091E2
:105880008D0490918E04A0918F04B0919004820FAA
:10589000931FA41FB51F80938D0490938E04A09333
:1058A0008F04B093900410924904D501C401885626
:1058B000954CAF4FBF4F8093210390932203A09349
:1058C0002303B093240381E080930E028091D60DD0
:1058D0009091D70D8A5E984341F480910902882304
:1058E00009F411C48150809309020E948296C090ED
:1058F000EC04D090ED04E090EE04F090EF04811100
:105900000E948F96D701C6013AE0B695A795979564
:1059100087953A95D1F7009721E0A207B10520F0CD
:105920008FEF9FEFA0E0B0E09695879520910E0253
:10593000211105C03091CD0C311143C43FC00097F7
:1059400039F040911F035091200348175907B0F5D3
:105950008091CD0C882309F4E6C383E00E94903245
:1059600081E08093FC0DE091D60DF091D70D199553
:10597000109288048091CD0C81112DC01092830467
:105980008091D60D9091D70D8A5E9843F9F40E94CC
:10599000C0A5DC01CB0188199909AA09BB090091AE
:1059A0001F031091200320E030E0081719072A0791
:1059B0003B0720F49093200380931F038091D60D22
:1059C0009091D70D8A5E984309F4C3C38091D80C97
:1059D0008111BFC3D8C38CED9DE00E945D9F91E013
:1059E000811101C090E09093CD0C882339F2809111
:1059F000D60D9091D70D8A5E9843B9F40E94C0A548
:105A0000DC01CB0188199909AA09BB0900911F0380
:105A10001091200320E030E0081719072A073B0700
:105A200020F49093200380931F030E94C0A56B0174
:105A30007C0180910402882359F180910903882315
:105A400039F140912A0350912B0360912C037091FE
:105A50002D0397018601041B150B260B370B37FD11
:105A60002AC0833079F03CF4813094F00E94D2282F
:105A70008BE599E00BC0843059F40E94D2288CE267
:105A800099E004C00E94D22884E499E00E94AC28E6
:105A90002091040230E0A8EEB3E00E9407BAC60EDF
:105AA000D71EE81EF91EC0922A03D0922B03E09263
:105AB0002C03F0922D038091270C843008F0E6C16E
:105AC0008091270C843008F00DC18091BE03909125
:105AD000BF03891B8F7709F405C10E94C52A97FD72
:105AE000EFCF8A3019F08D3009F0F3C010923203F5
:105AF0008091400490914104FC01ED5CFC4F1082C8
:105B0000892B39F0109241041092400403E313E012
:105B100003C00E947455D4CFF8018191803211F4F2
:105B20008F01FACF8E3409F07AC00115110509F4FE
:105B300076C06AE67AE0C8010E9402B37C01892B34
:105B400041F06EE470E0C80104960E94CFBD00975A
:105B500009F4C8014AE050E060E070E001960E945C
:105B60007AB060932E0370932F0380933003909349
:105B700031038090420490904304A0904404B0907C
:105B800045042FEF821A920AA20AB20A6815790513
:105B90008A059B0531F0EF2821F460E087E39AE065
:105BA00051C06AE270E0C8010E9407BE9C010097E4
:105BB00009F1982F901BF12C992339F09150F8019D
:105BC000E90FF11D8081F826F7CF4AE050E060E050
:105BD00070E0C90101960E947AB0CF2CD12CE12C43
:105BE000F12C6C157D058E059F0541F060E088E184
:105BF0009AE028C060E08EEE99E024C080912E03E8
:105C000090912F03A0913003B0913103809342040F
:105C100090934304A0934404B093450416C080912C
:105C2000330F80FF12C065E57DE1C8010E9402B319
:105C3000009729F0FC01838180538A3030F460E0C2
:105C40008EEE99E00E94D8344DC08091290C8130AD
:105C5000E1F067E470E0C8010E94CFBD0097A9F0B1
:105C60004AE050E060E070E001960E947AB0643053
:105C700071058105910548F487E799E00E94AC28F9
:105C800060E08DE699E00E94723E65EE72E0C80128
:105C90000E94DABD892B11F4109250046AEE72E072
:105CA000C8010E94DABD892B29F461E084E196E005
:105CB0000E94FAA06FEE72E0C8010E94DABD892B43
:105CC00011F40E94C32761E083E393E00E9416353C
:105CD000F7CE20E434E043E353E062E373E00E9454
:105CE0008234EECE8091330F82FFD0C01A821982A7
:105CF00011E040912F0F5091300F6091310F709152
:105D0000320F80912B0F90912C0FA0912D0FB091FD
:105D10002E0F481759076A077B0708F410E000E6C2
:105D200080E1F82E99E6E92E8091270C843008F066
:105D3000ADC01111ABC08091250D9091260DA091A1
:105D4000270DB091280D80932F0F9093300FA093C3
:105D5000310FB093320F41E050E0BE016B5F7F4FD7
:105D60008DE19DE00E944071019719F48D8190E0D2
:105D700002C08FEF9FEF40902F0F5090300F609038
:105D8000310F7090320F80902B0F90902C0FA090BD
:105D90002D0FB0902E0F11E0481459046A047B04B3
:105DA00008F410E08F3FFFEF9F0761F44814590497
:105DB0006A047B0438F40E94CE288FE69AE00E94A1
:105DC000AC28B2CF4091A20A8A3079F08D3069F0C8
:105DD000481459046A047B0408F4E6C189819A8155
:105DE000009719F001969A83898310929303898111
:105DF0009A81FC01049FE00DF11D1124EA55F54F35
:105E00001082892B31F01A82198280E00E940135BC
:105E100002C00E947455481459046A047B0408F4B3
:105E200083CF0E948C948DE19DE00E947D738091D0
:105E30002A0F882331F1815080932A0FE89EC001F8
:105E4000112462E0805D934F0E948F6CE0912A0FD5
:105E500024E0E29FF0011124E45DF34F4081518181
:105E60006281738140932F0F5093300F6093310FF5
:105E70007093320F8DE19DE00E94A9700E94106A1C
:105E800053CF0E94016AF092290C4ECF0E94C0A508
:105E90006B017C014091FE025091FF026091000372
:105EA00070910103411551056105710531F1809132
:105EB000020390910303A0910403B0910503840FA2
:105EC000951FA61FB71F97018601081B190B2A0BE8
:105ED0003B0B37FD12C00E94CE286091A90470913F
:105EE000AA0481EA9AE00E94BB288AE00E94A528C1
:105EF00060E080E090E00E94FAA04091050250919D
:105F00000602609107027091080241155105610572
:105F1000710509F448C09091940D8091950D9817E2
:105F200059F00E94C0A5609302037093030380930D
:105F300004039093050337C08091020390910303FB
:105F4000A0910403B0910503840F951FA61FB71FEE
:105F5000A7019601281B390B4A0B5B0B57FD21C08B
:105F600080919A0381111FC081E080939A035F9A08
:105F7000129A8091950A8E7F8093950A8A9A479A01
:105F80008091950A8D7F8093950A80910801809574
:105F90008170809306018091950A8B7F8093950A8A
:105FA00002C010929A03809198039091990390995E
:105FB00002C0019604C0181619062CF4019790939C
:105FC00099038093980380919803909199038E3E52
:105FD00092405CF00E94CE288EE79AE00E94AC28A6
:105FE00060E080E090E00E94FAA08091940390919C
:105FF0009503A0919603B091970397018601081B22
:10600000190B2A0B3B0B37FD28C09091940D809102
:10601000950D981751F0E091950D1BE4E19FF0016B
:106020001124E95BFA4F608102C06091F00466239D
:1060300011F070E002C060E070E088E00E94BDA452
:1060400024E6C20ED11CE11CF11CC0929403D09234
:106050009503E0929603F09297030E9474550E9474
:10606000E43D0F900F900F900F900F90DF91CF9124
:106070001F910F91FF90EF90DF90CF90BF90AF9066
:106080009F908F907F906F905F904F900895E091D8
:10609000160234E0E302F0011124EE5BFD4F808133
:1060A0009181A281B38189839A83AB83BC83C12C04
:1060B000D12C76018E010F5F1F4F2DE03DE049E0AE
:1060C0005DE065E07DE081E09DE00E9458528FEF49
:1060D00080931602A5CA60E08DE199E00E94723EAD
:1060E000FCCA0E94016A8091330F877F8093330F2F
:1060F000123009F4F2CA60E08FE099E00E94723E2B
:106100000E94F180EACA8CE08093090280911F030B
:106110009091200301979093200380931F0381E0C7
:1061200080930E02E2CB223050F0243028F024304D
:1061300031F410920E0203C081E080930E0288EDCC
:106140009DE00E94C8A081E0809388048093CD0CDC
:1061500004CC88E9880E8AE3981EA11CB11C8092A9
:10616000210390922203A0922303B09224038091F2
:10617000CD0C81115ACC80910E02813009F055CCA2
:1061800010920E0252CC8091210390912203A09193
:106190002303B0912403881A990AAA0ABB0AB7FC00
:1061A000E6CF0E94F180E3CF049FA00111244A555D
:1061B000554F9E012F5F3F4F63E973E00E94823489
:1061C000B3CD009709F4C9CBBCCB1F920F920FB689
:1061D0000F9211240F900FBE0F901F9018951F92D1
:1061E0000F920FB60F9211240BB60F922F938F932D
:1061F0009F93EF93FF932091BF03E091BE0381E053
:106200008E0F8F779091C600281729F0F0E0E254A6
:10621000FC4F9283E82FE093BE03FF91EF919F9193
:106220008F912F910F900BBE0F900FBE0F901F906C
:1062300018958EBD0DB407FEFDCF08958FEF8EBD6E
:106240000DB407FEFDCF8EB50895909164009B7F3D
:1062500090936400982F906A96959CBD80FD03C032
:1062600091E0863009F490E09DBD0895089580E0A6
:1062700090E00895DF92EF92FF920F931F93CF93D8
:10628000DF93EC01D62E1CAD0BAD7C0184E0E80E53
:10629000F11CE98DFA8DC7011995412F480F2D2D5D
:1062A000602FC7010E9483699BAD890F8BAF81E08E
:1062B00090E0DF91CF911F910F91FF90EF90DF90D1
:1062C00008958F929F92AF92BF92CF92DF92EF92FA
:1062D000FF920F931F93CF93DF93EC018B015A0131
:1062E0008A859B858617970731F0888199810E945E
:1062F00033681B870A87888599850196D1F1CE80FE
:10630000DF80D5010C91002349F1E880F980602FEE
:10631000C7010E948B68F701118911954501FFEFB4
:106320008F1A9F0AD4018D914D01882349F0F701FE
:106330009089190F082F682FC7010E948B68F2CF30
:10634000003241F0D70153969C91539751968C910E
:10635000890F02C0F7018089180F01C010E0C10E3B
:10636000D11C888599858C159D0518F481E090E0F5
:1063700024C0FC801A819E81190FC880D980D60163
:106380005596ED91FC915697C6011995F80E00E0CF
:10639000D5012D915D01222341F04F2D612FC601C2
:1063A0000E948369180F080FF3CF8E819F81800FA1
:1063B000911D9F838E8380E090E0DF91CF911F91AC
:1063C0000F91FF90EF90DF90CF90BF90AF909F9094
:1063D0008F90089511989091020187FD64C091708B
:1063E00090930001119A0000119890910201382FAA
:1063F000330F86FD56C0917090930001119A0000F2
:10640000119880910201232F220F36FD48C0817020
:1064100080930001119A0000119880910201922F3F
:10642000990F26FD3AC0817080930001119A0000F7
:10643000119880910201292F220F96FD2CC08170A6
:1064400080930001119A0000119880910201922F0F
:10645000990F26FD1EC0817080930001119A0000E3
:10646000119880910201292F220F96FD10C0817092
:1064700080930001119A000011988091020126FD7D
:106480008095817080930001119A00000895809595
:10649000EECF8095E0CF8095D2CF8095C4CF809508
:1064A000B6CF9095A8CF90959ACF9CE0899F802DEC
:1064B000112491E0980F909347042CE0280F20932B
:1064C000A60430E02E5F3F4F4091100E50E024179D
:1064D000350714F480E00895292F30E04091120E22
:1064E00050E024173507B4F7662341F08E5F0E9411
:1064F000C1408091A6048E5F0E94C1408091A60495
:106500009091100E891730F32091120E909147044C
:10651000291700F31092130E8093140E81E0089552
:10652000482F50E020914604022E000C330B4217F6
:10653000530741F08093460468E57BE08CED9DE0D5
:106540000C9433680895EF92FF920F931F93CF93AB
:10655000DF93CDB7DEB72C970FB6F894DEBF0FBE32
:10656000CDBF6F3F71058105910509F060F488ED9D
:106570009DE00E943A31E091E00DF091E10D3196FD
:10658000849190E03EC01091130E0091140E209162
:106590004804211109C048E35BE0602F812F0E946D
:1065A000A1A080E090E027C0E090E00DF090E10D28
:1065B0002CED3DE03A832983212F30E03C832B836F
:1065C000202F30E03E832D8318861F822FEF3FEF70
:1065D0003A8729871C861B869E012F5F3F4FAB01A0
:1065E000BC01C7010E948F9FB7018CED9DE00E9406
:1065F00033688F819885180F1093130E0093140E33
:1066000099272C960FB6F894DEBF0FBECDBFDF9151
:10661000CF911F910F91FF90EF9008950F93CF931B
:10662000DF93982F862FEA01692F0E945532882325
:1066300061F143E16091A704CE010E944C84C82F10
:10664000CC0F8C0FC82FCC0FC73040F060E270E049
:1066500080E090E00E94A332C81BF6CF8091A60490
:106660009AE79093130E8093140E602F000F770B10
:10667000880B990B0E94A33260E270E080E090E00A
:10668000DF91CF910F910C94A332DF91CF910F91B5
:106690000895EF92FF920F931F93CF93DF93CDB79F
:1066A000DEB72C970FB6F894DEBF0FBECDBF1091AA
:1066B000130E0091140E20914804211109C048E3E3
:1066C0005BE0602F812F0E94A1A080E090E026C0B7
:1066D000E090E00DF090E10D2CED3DE03A83298350
:1066E000212F30E03C832B83202F30E03E832D830D
:1066F00018861F827A8769871C861B869E012F5FFA
:106700003F4F47E45EE7BC01C7010E9466A0B701A6
:106710008CED9DE00E9433688F819885180F10934F
:10672000130E0093140E99272C960FB6F894DEBF23
:106730000FBECDBFDF91CF911F910F91FF90EF90D2
:1067400008956FEF7FEF0C944933EF92FF920F9310
:106750001F93CF93DF93CDB7DEB72C970FB6F89486
:10676000DEBF0FBECDBF1091130E0091140E20910D
:106770004804211109C048E35BE0602F812F0E948B
:10678000A1A080E090E026C0E090E00DF090E10D47
:106790002CED3DE03A832983212F30E03C832B838D
:1067A000202F30E03E832D8318861F827A876987E9
:1067B0001C861B869E012F5F3F4F4AE45EE7BC01AB
:1067C000C7010E9466A0B7018CED9DE00E9433686E
:1067D0008F819885180F1093130E0093140E99272C
:1067E0002C960FB6F894DEBF0FBECDBFDF91CF91D0
:1067F0001F910F91FF90EF9008956FEF7FEF0C9432
:10680000A533AF92BF92CF92DF92EF92FF920F9398
:106810001F93CF93DF935C016B010E94B284E82E3B
:10682000C6010E94D484F12C03E110E0081B110979
:106830000E151F0514F0C5E201C0CFE18C2F90E0CA
:10684000AC014E5F5F4F2091100E30E042175307AE
:106850003CF009972091120E30E028173907DCF53B
:10686000D0E0C114D10409F442C06AE370E080E0D2
:1068700090E00E94A3320E151F0584F4C45F80913E
:10688000100EC817A0F12C2F30E02950310980914B
:10689000120E90E0821793071CF429C0DD2339F112
:1068A000802F880F080F000F0093130EC093140E53
:1068B00060E270E080E090E00E94A332C601DF91C8
:1068C000CF911F910F91FF90EF90DF90CF90BF90ED
:1068D000AF900C94FD336091A7041092130EC093F7
:1068E000140E45E1C5010E944C84D1E0BACFDF917E
:1068F000CF911F910F91FF90EF90DF90CF90BF90BD
:10690000AF900895CF93DF93DB01E9019C91913023
:1069100001F1943018F094509C930CC08C3529F4FC
:106920009C5F9C93943031F414C08B3319F481E054
:106930008C930FC0E881F9819F012F5F3F4F39830E
:106940002883E40FF51F8083888199818F35910515
:1069500074F7DF91CF910895E091260CF0E0EA5EA4
:10696000F14F8081882339F08CE29BE00E94AC28B3
:106970008AE00C94A5280895EEEBF3E080818183F2
:106980008FE29BE00E94AC288091420490914304E6
:10699000A0914404B0914504BC01CD016F5F7F4FCD
:1069A0008F4F9F4F0E94B5290E94B22A0C94AC349D
:1069B0000F931F93CF938C01C62F0E94CE28C8013E
:1069C0000E94AC2860914204709143048091440479
:1069D000909145040E94B5290E94B22AC11104C0B9
:1069E0000E94C52A0196E1F70E94BC34EC2FEE0FFD
:1069F000FF0BE05CFB4F11821082CF911F910F9132
:106A000008959091A20AE92FF0E0EA5EF14F8083A9
:106A10009F5F943018F49093A20A02C01092A20AC9
:106A20008091270C8F5F8093270C0895CF93FC01F2
:106A300020812B33A9F02091270C243088F4C62F15
:106A4000BC018091A20AF0E68F9FC00111248A55F3
:106A5000954F0E94E3BD8C2F0E94013581E001C05B
:106A600080E0CF9108950F931F93CF93FC01208175
:106A70002223B9F02A30A9F02D3099F08C0160E082
:106A80000E941635C82F882369F00E94D228B801C9
:106A90008FE19BE00E94BB2880EC92E10E94AC2831
:106AA00001C0C1E08C2FCF911F910F9108957F926B
:106AB0008F929F92AF92BF92CF92DF92EF92FF920E
:106AC0000F931F93CF93DF931092BA031092B903E1
:106AD0002FE32093BD031092BC031092BB031092CE
:106AE000B5031092B6031092B7031092B8039C013D
:106AF000F90190812F5F3F4F9032D1F38FE9890FD9
:106B00008A3108F490529E3489F4818190ED980F77
:106B10009A3008F42BC18D3209F428C18B3231F43C
:106B200025C1FD01119680818032D9F3F093AA042A
:106B3000E093A9048F010F5F1F4F70808FE9870DCD
:106B40008A3118F440EE842E780C6AE270E0C801B5
:106B50000E94CFBD009731F0FC01319780818032D7
:106B6000E1F311823DE4932E791441F024E5A22E45
:106B70007A1421F097E4B92E7B1014C1F8018081BA
:106B80000F5F1F4F8032D1F380538A3008F00AC163
:106B90007092BD031092BC031092BB036AE0209177
:106BA000BB033091BC03629FC001639F900D112411
:106BB0009093BC038093BB033196DF0111974C91F6
:106BC000042E000C550B40535109480F591F509388
:106BD000BC034093BB03808180538A3000F3DF0104
:106BE00031968C918032D9F38DE478121AC04E31EF
:106BF000510591F03CF44731510571F04C3151058C
:106C000081F40AC04537510564F04737510524F037
:106C1000403A93E0590729F4B093BA03A093B9031B
:106C2000C1C01092BA031092B9036091A904C12C9B
:106C3000D12C7601C394FD0131968C919FE9980F78
:106C40009A3110F480521AC0882309F4ABC0813203
:106C5000A9F4CDE47C1212C04032510579F4F093CE
:106C6000BA03E093B90363E270E0CF010E94CFBDA5
:106C7000009709F497C0FC01108294C02FEB280FF5
:106C80002A3108F04BC0DF01FD018081119680326E
:106C9000D9F390ED980F9A30B0F08E3211F48181D3
:106CA0000EC08D3219F08B3209F06CC0818190EDED
:106CB000980F9A3040F08E3209F064C08281805380
:106CC0008A3008F05FC0CF01A22FB0E04601570123
:106CD00004C0880C991CAA1CBB1C2A95D2F79501EC
:106CE00084018090B5039090B603A090B703B09054
:106CF000B803082919292A293B290093B5031093C1
:106D0000B6032093B7033093B803009711F0861BA6
:106D100001C080E0A556BC4F8C930AC08091B90396
:106D20009091BA03892B21F4B093BA03A093B903CD
:106D3000808181548A3138F4DF017DCF90ED980F46
:106D40009A3040F4F901DF01EF0189919E01811130
:106D5000F5CF71CF93ED980F9230A0F38B3291F372
:106D6000DF0131968C918032D9F365CFDF01129625
:106D70009D012F5F3F4F8C9180538A3008F0D1CE18
:106D8000D901F6CF8091B9039091BA03009739F4F5
:106D9000DF011197B093BA03A093B90395CF80E0B8
:106DA00090E092CFDF91CF911F910F91FF90EF90E4
:106DB000DF90CF90BF90AF909F908F907F9008957D
:106DC000CF93DF93D62FC72F0E949226882329F0D6
:106DD0000E94EE25262F972F02C02D2F9C2F822F49
:106DE000DF91CF9108950F931F93CF938C01C62FFE
:106DF0008AE19BE00E94AC28C8010E94AC288AE38B
:106E00000E94A5286C2F70E080E090E00E94B529D8
:106E1000CF911F910F910C94B22A4F925F926F9273
:106E20007F928F929F92AF92BF92CF92DF92EF921A
:106E3000FF920F931F93CF93DF93CDB7DEB77C0103
:106E40004DB65EB66090A9047090AA048DB69EB649
:106E50006AE070E0C7010E94C7B26C01009721F0A0
:106E60008C010E191F0904C0C7010E94D2B28C0107
:106E7000C80101962DB73EB7281B390B0FB6F89401
:106E80003EBF0FBE2DBF8DB79EB701965C01A80116
:106E9000B7010E94F3B2F501E00FF11F1082C501A6
:106EA0000E94573581E00E94FD12C114D10451F0B7
:106EB00076019FEFE91AF90A0FB6F8949EBE0FBE4D
:106EC0008DBEC4CF0FB6F8949EBE0FBE8DBEC3015B
:106ED0000E9457350FB6F8945EBE0FBE4DBEDF91CF
:106EE000CF911F910F91FF90EF90DF90CF90BF90C7
:106EF000AF909F908F907F906F905F904F9008958C
:106F0000CF93DF93C091260C80E6C89FE001112447
:106F1000CA55D54F8091B30980FF05C00E94D22881
:106F2000CE010E94B82ACE010E94573580E0DF9141
:106F3000CF910C94FD129C0197FF0AC0EE27FF270A
:106F4000E81BF90BE436F1050CF44CC08DE230C0BF
:106F5000283E83E038073CF1C90168EE73E00E94E7
:106F600036BACB01EAE0F0E0BF010E9436BA805D9C
:106F70008093A104C90164E670E00E9436BACB0197
:106F8000BF010E9436BA805D8093A204C901BF018F
:106F90000E9436BACB01BF010E9436BA805D809351
:106FA000A304F9013EC0F90124363105DCF080E28A
:106FB0008093A104CF0164E670E00E9436BACB0151
:106FC0002AE030E0B9010E9436BA805D8093A204C5
:106FD000CF01B9010E9436BACB01B9010E9436BA7D
:106FE000805D1DC080E28093A1048093A204EA30FA
:106FF000F10584F037FF02C08DE201C080E280938A
:10700000A204CF016AE070E00E9436BA605D60932E
:10701000A30407C037FF02C08DE201C080E2809365
:10702000A304CF016AE070E00E9436BA805D8093CD
:10703000A40481EA94E008950E9417530E9448280E
:10704000882319F08091330F82FD0C94EA668FEE4D
:107050009FE19093A50A8093A40AF7CFCF92DF9285
:10706000EF92FF92FC01C080D180E280F38020E0AB
:1070700030E0A901C701B6010E9484B387FF08C0B0
:10708000C701B601905820E030E040E251E406C06C
:1070900020E030E040E251E4C701B6010E94EAB3CB
:1070A00020E030E040EA50E40E947ABA20E030E08C
:1070B00040E251E40E9474BB0E94E6BBFB01E03158
:1070C00087E2F80740F0CF0160E177E20E9422BA40
:1070D00080E3860F01C080E28093A004E83E83E055
:1070E000F80760F0CF0168EE73E00E9422BACB018E
:1070F0006AE070E00E9422BA805D01C080E2809365
:10710000A104E436F10560F0CF0164E670E00E946E
:1071100022BACB016AE070E00E9422BA805D01C011
:1071200080E28093A204EA30F10560F02AE030E0CA
:10713000CF01B9010E9422BACB01B9010E9422BA43
:10714000805D01C080E28093A304CF016AE070E01B
:107150000E9422BA805D8093A40480EA94E0FF90AC
:10716000EF90DF90CF9008959C0197FD0EC084367C
:10717000910584F064E670E00E9436BACB016AE0C3
:1071800070E00E9436BA805D06C0319521953109C4
:107190008DE201C080E28093A2042A30310564F0C0
:1071A000EAE0F0E0C901BF010E9436BACB01BF019D
:1071B0000E9436BA805D01C080E28093A304C901B9
:1071C0006AE070E00E9436BA805D8093A40482EA8F
:1071D00094E008954F925F926F927F928F929F9268
:1071E000AF92BF92CF92DF92EF92FF920F93CF9325
:1071F000DF9300D01F921F92CDB7DEB710928904A3
:1072000080918304109283048823B1F020E040E051
:1072100060E070E08EE09CE80E94D27D81E0809387
:10722000480486EC90E19093FE0C8093FD0C109244
:10723000000D1092FF0C86C420910C0230910D02BB
:1072400040918D0450918E04C901840F951F2436FE
:10725000310559F44730510514F0069722C04A3FD2
:107260005F4F0CF02CC306961CC0243631052CF45D
:10727000853691050CF023C304C08436910524F4AF
:107280001EC38A3091053CF0883EE3E09E072CF057
:1072900087EE93E002C08AE090E02817390731F4C6
:1072A00011C08A30910584F78AE090E090930D0236
:1072B00080930C0210928D0410928E0410928F0411
:1072C0001092900480918804882309F416C22091BA
:1072D000110D3091120D4091130D5091140D6091CC
:1072E000010D7091020D8091030D9091040D0E948B
:1072F0007ABA4B015C012091150D3091160D409129
:10730000170D5091180D6091050D7091060D80912B
:10731000070D9091080D0E947ABA69837A838B8356
:107320009C832091190D30911A0D40911B0D5091A5
:107330001C0D6091090D70910A0D80910B0D9091BB
:107340000C0D0E947ABA2B013C0120E030E04AE7A4
:1073500054E40E94EAB36B017C0120E030E0A90113
:10736000C301B2010E9484B387FD05C020E030E074
:1073700040EA50E404C020E030E040EA50ECC701AD
:10738000B6010E947ABA20E030E040E251E40E9467
:1073900074BB0E94E6BB2B013C0197FF0AC07094AE
:1073A000609450944094411C511C611C711C8DE2EE
:1073B00001C080E280939E04F0E14F16F7E25F0681
:1073C0006104710494F0C301B20120E137E240E0AE
:1073D00050E00E944ABACA01B9012AE030E040E018
:1073E00050E00E944ABA605D01C060E260939F0471
:1073F00028EE421623E052066104710494F0C301A2
:10740000B20128EE33E040E050E00E944ABACA01DF
:10741000B9012AE030E040E050E00E944ABA605DE5
:1074200001C060E26093A004C301B20124E630E031
:1074300040E050E00E944ABA9AE0C92ED12CE12CDB
:10744000F12CCA01B901A70196010E944ABA605DF8
:107450006093A104C301B201A70196010E944ABA38
:107460006D83662389F08EE28093A204CA01B9017C
:10747000A70196010E944ABA605D6093A3043D8112
:10748000305D3093A40417C0CA01B901A701960169
:107490000E944ABA662339F08EE28093A204605DAE
:1074A0006093A30405C080E28093A3048093A204A8
:1074B00080E28093A4046EE974E084E794E00E9483
:1074C000E3BD20E030E0A901C501B4010E9484B30E
:1074D00087FD05C020E030E040E05FE304C020E02D
:1074E00030E040E05FEBC501B4010E947ABA0E942F
:1074F000E6BBCB010E949B37BC018FE694E00E9463
:10750000E3BD20E030E0A90169817A818B819C8113
:107510000E9484B387FD05C020E030E040E05FE3D7
:1075200004C020E030E040E05FEB69817A818B812C
:107530009C810E947ABA0E94E6BBCB010E949B37D5
:10754000BC018AE694E00E94E3BD0E94482888239B
:1075500021F180912B0F90912C0FA0912D0FB091C4
:107560002E0F0097A105B105C1F0BC01CD016D59E9
:107570007F4F8F4F9F4F24E630E040E050E00E9465
:10758000DAB960912F0F7091300F8091310F909187
:10759000320F0E94DAB9F22E01C0F12C0E949B66D4
:1075A0004B015C01698380910B028F15A1F0F09271
:1075B0000B0248E4F49EB001112480E090E00E94A8
:1075C00089B32AE037ED43E25CE30E94EAB30E940C
:1075D000EDBB6093690480910A025981581709F440
:1075E0008CC080920A02C501B40120E13EE040E077
:1075F00050E00E94DAB929833D8379018CE3482E5B
:10760000512C612C712CC501B401A30192010E947F
:10761000DAB9CA01B901A30192010E94DAB9D62EE2
:10762000C72E60E8861661E5960661E0A606B104FD
:1076300050F1C501B40120E831E541E050E00E947D
:10764000DAB93A832983CF92DF92C70168E170E00B
:107650000E9422BA9F938F933F932F938BE990E1DF
:107660009F938F9389E594E09F938F930E941CB31F
:107670000FB6F894DEBF0FBECDBFE981FA813A970D
:10768000A0F588E033C0F4E6EF16F104B8F47F9378
:10769000DF922D812F9339813F9380EA90E19F9370
:1076A0008F9389E594E09F938F930E941CB30FB64C
:1076B000F894DEBF0FBECDBF85E018C07F93DF9288
:1076C0005D815F9369816F9381E990E19F938F93CF
:1076D00089E594E09F938F930E941CB30FB6F894B2
:1076E000DEBF0FBECDBF86E001C089E0982F990FA5
:1076F000890F8195855A809358040E94C0A5C09037
:107700005404D0905504E0905604F09057049B0127
:10771000AC012C193D094E095F0957FD13C020919A
:107720005304209520935304DC01CB018A549C4FD1
:10773000AF4FBF4F8093540490935504A0935604C9
:10774000B0935704D090530481E00E94903280910E
:10775000100E8431E8F48091120E823008F0B2C02D
:1077600017C086EC90E19A83898302E128E142E028
:1077700068E68CED9DE00E946169882349F0E9800C
:10778000FA8023E042E068E68CED9DE00E94CC5256
:107790008091100E8C3118F58091120E8431F8F022
:1077A0008091F0048823D9F0E4E68E9FC001112473
:1077B00081589F4F6FEF70E00E9436BACB010E9454
:1077C000B43827E62093130E2CE12093140E0E9468
:1077D000FD3365E270E080E090E00E94A3320E94F9
:1077E0004828882349F08091100E843328F4809132
:1077F000120E8A3208F075C08091100E853328F47D
:107800008091120E813308F094C08091100E843361
:1078100028F48091120E823308F092C08091100EED
:10782000803328F48091120E883208F093C0809142
:10783000100E883298F48091120E8D3178F02BE082
:1078400040E86DE180E00E9434408091100E873264
:1078500028F48091120E8F3108F088C08091100EAC
:10786000833328F48091120E8B3208F044C180914A
:10787000100E813408F066C18091120E863308F430
:1078800061C11092130E8EE38093140E80E492E196
:107890000E94D484898360E870E080E492E10E94D1
:1078A000A533F981F53108F04DC160E270E080E068
:1078B00090E00E94A33229812F5F2983F2CF84E6D2
:1078C00090E0E2CCDD2041F08091F004882309F4BF
:1078D00048CF4CEF50E102C046EC50E15A83498357
:1078E00044CF07E028E04AE26AE28CED9DE00E9486
:1078F0006E4005E022E04CE262E38CED9DE00E94E8
:107900006E4024E04AE061E38AE20E9434406091E4
:10791000DE0D7091DF0D82E38093F80D8BE2809392
:10792000F90D28EF3DE042E38CED9DE00E942F68C9
:1079300063CF24E04AE461E386E30E94344065CFEC
:1079400002E02091690442E367E38CED9DE00E9430
:107950006E4064CF809158048093130E80E380932F
:10796000140E89E594E00E94FD3361CF83E080939B
:10797000130E56E25093140E68E570E080E090E03C
:107980000E94A3328BE08093130E66E26093140E84
:10799000DD2029F08FE694E00E94FD3326C080911F
:1079A000EA0C80FD1AC02FE634E03A832983E9818E
:1079B000FA816191FA83E9836623B9F06F3234F476
:1079C000062E000C770B880B990B04C06FE370E058
:1079D00080E090E00E94A332EACF8091950A80FD7A
:1079E000D9CF8FEA90E10E94A13388E28093130EF1
:1079F000F6E2F093140E69E570E080E090E00E94FA
:107A0000A33280E38093130E26E22093140EDD2030
:107A100029F08AE694E00E94FD3328C08091EA0CA8
:107A2000869580FD1AC04AE654E05A834983E9816D
:107A3000FA816191FA83E9836623C1F06F3234F4ED
:107A4000062E000C770B880B990B04C06FE370E0D7
:107A500080E090E00E94A332EACF8091950A86955B
:107A600080FDD7CF8FEA90E10E94A1338DE480930F
:107A7000130EF6E2F093140E6AE570E080E090E0F9
:107A80000E94A33285E58093130E26E22093140E04
:107A9000DD2029F084E794E00E94FD33DFCE809161
:107AA000EA0C8695869580FD1BC044E754E05A8316
:107AB0004983E981FA816191FA83E983662309F4B4
:107AC000CDCE6F3234F4062E000C770B880B990B59
:107AD00004C06FE370E080E090E00E94A332E9CF41
:107AE0008091950A8695869580FDD4CF8CEA90E1A9
:107AF0000E94A133B3CE83E00E94903283E0809352
:107B0000130E83E38093140E66E070E080E090E053
:107B10000E94A33281E00E94903280910C029091E9
:107B20000D020E94B4382CE02093130EE3E3E0939F
:107B3000140E0E94FD3365E270E080E090E00E9448
:107B4000A33295CE0F900F900F900F900F90DF9172
:107B5000CF910F91FF90EF90DF90CF90BF90AF90BB
:107B60009F908F907F906F905F904F90089524E644
:107B7000829FC001112481589F4F6FEF70E00E94D7
:107B800036BA262F643611F080E201C081E380937B
:107B9000A1042A3048F03AE0822F632F0E9416BADF
:107BA0000E9416BA905D01C090E29093A204822FC9
:107BB0006AE00E9416BA905D9093A30485E28093D8
:107BC000A40481EA94E008950F931F930E94C0A536
:107BD0000091BE0D1091BF0D2091C00D3091C10DCF
:107BE0000115110521053105E1F52091C40D222370
:107BF00009F448C0E091C20D21502093C40D21E04A
:107C00002E0F2093C20D3091C50D231302C0109288
:107C1000C20D24E0E29FF0011124EA53F24F0081EB
:107C20001181228133810093BA0D1093BB0D2093F3
:107C3000BC0D3093BD0DDC01CB01800F911FA11D48
:107C4000B11D8093BE0D9093BF0DA093C00DB09356
:107C5000C10D8091BC0D9091BD0D892B99F0409A7A
:107C600011C0DC01CB01801B910BA20BB30BB7FD44
:107C700009C040981092BE0D1092BF0D1092C00D19
:107C80001092C10D1F910F9108950F931F93CF93E1
:107C9000DF938C01EB019091C40D2091C50D9213DF
:107CA00005C00E94E43D0E947455F5CF8091C30D3C
:107CB00034E0839FF0011124EA53F24F11830083D3
:107CC000D383C2839F5F9093C40D8F5F281719F0F1
:107CD0008093C30D02C01092C30DDF91CF911F910D
:107CE0000F9108950F931F93CF93DF938C0167FF3C
:107CF00003C010924F0460E080914F0490E0262F63
:107D0000062E000C330B28173907F4F060934F044C
:107D1000C8010E94D2B2800F911FEC01C01BD10B91
:107D2000CB32D1053CF00197FC012491207C203816
:107D3000D1F3F3CFDD27AE01B80180E492E10E94D8
:107D4000F3B2C05CDD4E1882DF91CF911F910F918D
:107D5000089585E890E190935204809351040E9425
:107D6000037E60E083EB92E10E94723E82EC90E140
:107D70009093A50A8093A40A0895109250048091CC
:107D8000330F80648093330F0E940E6760E084EBB2
:107D900090E10E94723E0C94F180CF93DF93CDB7B7
:107DA000DEB78E8190914F04891768F080934F045D
:107DB0009E01275F3F4F4F8158856AE270E080E463
:107DC00092E10E944BB3DF91CF910895CF93DF935F
:107DD00020914F0421111AC0FC0101900020E9F705
:107DE0003197EF01C81BD90BCB32D1052CF0229172
:107DF000207C2038E1F3F5CFBC01DD27AE0180E423
:107E000092E10E94F8BDC05CDD4E1882DF91CF91F7
:107E100008950F931F930E94C0A500914B041091E9
:107E20004C0420914D0430914E04DC01CB01801BA9
:107E3000910BA20BB30BB7FD0CC086B186FB992743
:107E400090F981E08927349B8260329B8460809323
:107E50004A0480914A04817090914A0491FD8260A5
:107E600090917C04891731F18130A9F028F082309B
:107E700041F0833059F01CC0913089F0923099F074
:107E800017C0992361F0933071F012C0913059F00E
:107E9000923071F404C0992331F0933049F49091F9
:107EA00049049F5F03C09091490491509093490405
:107EB00080937C041F910F91089590E0FC0131970D
:107EC000E231F10508F04EC08827EE58FF4F8F4F82
:107ED0000C9469BA809180008F7703C080918000F4
:107EE0008F7D80938000089580918000877FF9CFF7
:107EF00084B58F7702C084B58F7D84BD089580914D
:107F0000B0008F7703C08091B0008F7D8093B00068
:107F10000895809190008F7707C0809190008F7DA9
:107F200003C080919000877F809390000895809196
:107F3000A0008F7707C08091A0008F7D03C0809143
:107F4000A000877F8093A0000895809120018F7703
:107F500007C0809120018F7D03C080912001877F21
:107F6000809320010895DF92EF92FF920F931F9369
:107F7000CF93DF93082FD62FC42F142FF62EF40E95
:107F8000EE24E394DD24DA948F2D811B1830A8F0C1
:107F90006091DE0D7091DF0D0093F80D8093F90D67
:107FA000E092FB0DD092FA0D28EF3DE04BE38CED13
:107FB0009DE00E942F681850E7CF8C2F86958695FC
:107FC000869598E0899FD00D11244C2F98EF899FBA
:107FD000400D1124442329F187E048276091DE0DEC
:107FE0007091DF0D0093F80DD093F90D81E080932F
:107FF000FB0D4F5F47708FEF90E001C0880F4A95EF
:10800000EAF78093FA0D28EF3DE04BE38CED9DE01D
:10801000DF91CF911F910F91FF90EF90DF900C9423
:108020002F68DF91CF911F910F91FF90EF90DF901C
:108030000895EF92FF920F931F93CF93DF937C01EC
:10804000D62F122FC42F040F212F4C2F6D2FC701B5
:108050000E945F53CF5FC013F7CFDF91CF911F9185
:108060000F91FF90EF900895FF920F931F93CF937E
:10807000DF93182FC62FF42ED22F022F242F462F36
:10808000682F8CED9DE00E946169882309F12F2DF6
:108090004C2F612F8CED9DE00E945F534D2F6C2F74
:1080A000812F0E94B33F8FEF8F0D4D2F6C2F810FCB
:1080B0000E94B33F4FEF4D0F4C0F2F2D612F8CEDD2
:1080C0009DE0DF91CF911F910F91FF900C945F5332
:1080D000DF91CF911F910F91FF900895DF92EF9262
:1080E000FF920F931F93CF93DF93EC01162FF42E83
:1080F000E22E0E946169882331F02E2D4F2D612FD1
:10810000CE010E941940DF91CF911F910F91FF90F6
:10811000EF90DF900895EF92FF920F93CF93DF934C
:10812000C82F7B01D42FCB010E94B2849C2F990FC2
:10813000C90FCC0FDD2391F091E09093FC0D282F17
:10814000220F280F220F2E5F0BE043E36FEF6C0F1F
:108150008CED9DE00E946E401092FC0DC093130EBA
:108160008CE38093140EC7010E94A133DD2319F024
:1081700081E08093FC0DDF91CF910F91FF90EF9004
:1081800008950F93CF93C82F01E020E8482F60E0B7
:108190008CED9DE00E946169882349F020E84C2F16
:1081A00060E08CED9DE0CF910F910C945F53CF91E7
:1081B0000F9108950F931F93CF938B01C42F41FB11
:1081C000662760F90E945532882379F1C0FF18C0F4
:1081D000C8010E94B28425E130E0A901481B510981
:1081E000CA0157FD019695958795C82FC150C7FDC7
:1081F00007C060E270E080E090E00E94A332F6CF1A
:1082000045E16091A704C8010E944C84C82FCC0F9F
:108210008C0FC82FCC0FC73040F060E270E080E0D8
:1082200090E00E94A332C81BF6CFCF911F910F910F
:108230000895CF93982F862FC42F692F0E9455320F
:10824000882311F1CC2331F062E070E080E090E00F
:108250000E94A3328091B804811111C08BEA94E08E
:1082600068E770E00E94A533C8E7C81BC73060F01C
:1082700060E270E080E090E00E94A332F6CF1092BE
:10828000CC0488EB94E0ECCFCF9108958F929F922D
:10829000AF92BF92CF92DF92EF92FF92CF93FC0109
:1082A000C080D180E280F38020E030E44CE156E4ED
:1082B000C701B6010E94EAB34B015C0120E030E047
:1082C000A901C701B6010E9484B387FD05C020E063
:1082D00030E040EA50E404C020E030E040EA50ECF6
:1082E000C501B4010E947ABA20E030E040E251E4D6
:1082F0000E9474BB0E94E6BB6B017C016115710595
:108300008105910561F097FF0AC0F094E094D09444
:10831000C094C11CD11CE11CF11C8DE201C080E2A3
:1083200080939F04C701B60128EE33E040E050E09F
:108330000E944ABA8AE0882E912CA12CB12CCA0145
:10834000B901A50194010E944ABA605D6093A0043E
:108350008EE28093A104C701B60124E630E040E03C
:1083600050E00E944ABACA01B901A50194010E94D5
:108370004ABA605D6093A204C701B601A5019401E9
:108380000E944ABAC62FCA01B901A50194010E94F0
:108390004ABA605D6093A304C05DC093A4048FE9F2
:1083A00094E0CF91FF90EF90DF90CF90BF90AF908F
:1083B0009F908F9008951092890480918D049091E0
:1083C0008E04A0918F04B0919004B7FF08C0109262
:1083D0008D0410928E0410928F041092900480915C
:1083E0008804882331F080918D0480938704109253
:1083F0009D04809186041816D4F4082E000C990B65
:10840000019720918704022E000C330B281739079F
:1084100074F080938704092E000CAA0BBB0B809389
:108420008D0490938E04A0938F04B0939004809158
:10843000870490918504891714F480938504209112
:108440008504022E000C330B2C5F3F4F482F082E63
:10845000000C550B241735071CF4845080938504B9
:1084600008953F924F925F926F927F928F929F9268
:10847000AF92BF92CF92DF92EF92FF920F931F9332
:10848000CF93DF931F921F92CDB7DEB75C016801D7
:1084900040908D0450908E0460908F0470909004F2
:1084A000411451046104710479F091E0141415042D
:1084B0000CF090E09093840410928D0410928E043E
:1084C00010928F04109290041091840430908304D1
:1084D00010928304311005C080910E02882309F4A4
:1084E00073C049012A013B01C9010E94B284082FCF
:1084F000E114F10409F466C0C7010E94B2841A8233
:108500001982C114D104B1F4402F50E0282F30E07B
:10851000CA01820F931F46976CF485E190E0841B9B
:10852000950B821B930B97FD0196959587958A83F2
:1085300081E0898301E027E43EE7A401BE016F5F8B
:108540007F4FCE0102960E949191C114D10491F007
:108550008A81882321F01A8289818F5F898300E0D4
:108560002AE43EE7A601BE016F5F7F4FCE0102966F
:108570000E949191E114F10459F000E027E43EE7F4
:10858000A701BE016F5F7F4FCE0102960E949191BD
:1085900041E04127B30181E00E948B40C5010E9468
:1085A000B284412FB50194E1981B892F0E948B4022
:1085B000332051F0112319F0F201199505C00E94E2
:1085C000F98002C080E09BCF0F900F90DF91CF9198
:1085D0001F910F91FF90EF90DF90CF90BF90AF90E1
:1085E0009F908F907F906F905F904F903F900895F5
:1085F000CF93DF93282F30E0F901E359FD4E8491AA
:10860000F901E95DFD4ED491F901EF51FE4EC4919F
:10861000CC2391F081110E945D3FEC2FF0E0EE0F32
:10862000FF1FE953FE4EA591B491EC91ED2381E03B
:1086300090E021F480E002C080E090E0DF91CF91F3
:1086400008951F93CF93DF93282F30E0F901E3596A
:10865000FD4E8491F901E95DFD4ED491F901EF5190
:10866000FE4EC491CC23C1F0162F81110E945D3FB4
:10867000EC2FF0E0EE0FFF1FE355FE4EA591B491F5
:108680009FB7F894111104C08C91D095D82302C0E3
:10869000EC91DE2BDC939FBFDF91CF911F9108956A
:1086A000CF93DF9390E0FC01E95DFD4E2491FC0146
:1086B000EF51FE4E8491882361F190E0880F991F5D
:1086C000FC01ED56FE4EC591D491FC01E355FE4EE2
:1086D000A591B491611109C09FB7F8948881209544
:1086E00082238883EC912E230BC0623061F49FB704
:1086F000F8948881322F309583238883EC912E2B38
:108700002C939FBF06C08FB7F894E8812E2B288347
:108710008FBFDF91CF9108958F929F92AF92BF92BA
:10872000CF92DF92EF92FF920F931F93CF93DF933D
:10873000CDB7DEB76E970FB6F894DEBF0FBECDBFD4
:10874000D82E70937E0460937D040E94DB41E090FC
:1087500085048CE0C82E91E0F12C23E4A22E21E1C7
:10876000B22E9E012F5F3F4F490131E0D31679F1C0
:10877000D31628F082E0D81609F454C07EC0E11068
:10878000A7C09923D9F0809187041816BCF04091B6
:108790008D0450918E0460918F04709190044F5F0E
:1087A0005F4F6F4F7F4F40938D0450938E046093C3
:1087B0008F04709390048F5F8093870480910E02E2
:1087C000882309F40EC143E06CE871E17DC0E1103B
:1087D0007FC09923D9F0809187041816BCF040918E
:1087E0008D0450918E0460918F04709190044F5FBE
:1087F0005F4F6F4F7F4F40938D0450938E04609373
:108800008F04709390048F5F8093870480910E0291
:10881000882309F4F7C043E065E871E18F2D0E94D9
:10882000DA40F0C0E11054C09923D9F08091870458
:108830001816BCF040918D0450918E0460918F0405
:10884000709190044F5F5F4F6F4F7F4F40938D0447
:1088500050938E0460938F04709390048F5F809385
:10886000870480910E02882309F471C043E06EE70B
:1088700071E18F2D0E94DA406AC0E11029C099236E
:10888000D9F0809187041816BCF040918D04509166
:108890008E0460918F04709190044F5F5F4F6F4F13
:1088A0007F4F40938D0450938E0460938F04709398
:1088B00090048F5F8093870480910E02882309F4CF
:1088C00090C043E065E771E18F2D0E94DA4089C0D6
:1088D00091E0E9120CC010918704113009F051C0E9
:1088E0008091830410928304811145C04AC022E024
:1088F000E2120CC080918704823009F057C0809149
:10890000830410928304811149C050C023E0E21611
:1089100009F45EC084E0E81264C08091870484306A
:1089200009F4B5C080910E02882309F45AC081E091
:1089300090918704943009F080E003E02EE34DE449
:1089400051E16F2D0E940E3332E0D3125BC0809153
:108950000E02882321F095E0E91609F470C086E044
:10896000F394E3942CE0C20E90E035E0F312FDCED8
:1089700080938604B1C00E94F98080919D0481118A
:10898000ABC080910E02882361F181E0113009F0C3
:1089900080E004E024E04BE651E116C089E491E96F
:1089A0000E94F2AD80919D04811196C080910E02CB
:1089B0008823B9F081E090918704923009F080E03B
:1089C00003E02EE341E651E16F2D0E940E3309C012
:1089D00080918704833009F453C080910E02811185
:1089E00067C092E0D9120EC085E0E812B0CF809146
:1089F0008704853089F48091830410928304811167
:108A000003C00AC085E0ACCF87E391E90E94F2ADD4
:108A100080919D04811160C080910E02882309F429
:108A20009ECF81E090918704953009F080E003E0CB
:108A30002EE349E95BE16F2D0E940E3388CF10923F
:108A4000130EC092140E8E010B5E1F4F23E041E007
:108A50006DEC7CEC8CEC9CE30E94FEAE9F938F93BC
:108A6000BF92AF929F928F920E941CB3C4010E944A
:108A7000FD330F900F900F900F900F900F906FCFCE
:108A80008091830410928304811108C0A6CF809145
:108A9000830410928304811116C044CF83E491E9CA
:108AA0000E94F2AD80919D04882309F496CF14C0F2
:108AB00081E090918704933009F080E003E02EE399
:108AC00048E551E181CF8DE391E90E94F2AD8091BB
:108AD0009D04882309F426CF6E960FB6F894DEBF66
:108AE0000FBECDBFDF91CF911F910F91FF90EF90FF
:108AF000DF90CF90BF90AF909F908F9008952F926E
:108B00003F924F925F926F927F928F929F92AF921D
:108B1000BF92CF92DF92EF92FF920F931F93CF936A
:108B2000DF93CDB7DEB7CB56D1090FB6F894DEBFD1
:108B30000FBECDBF3B014A0159016801FEAAEDAA53
:108B40002091C8093091C9094091CA095091CB09B7
:108B5000DC016D917D918D919C910E94EAB30E9400
:108B6000E7BC6F966CAF7DAF8EAF9FAF6F972091D4
:108B7000CC093091CD094091CE095091CF09F30134
:108B800060817181828193810E94EAB30E94E7BC77
:108B9000A3966CAF7DAF8EAF9FAFA3972091D00906
:108BA0003091D1094091D2095091D309D4016D91EE
:108BB0007D918D919C910E94EAB30E94E7BCA7969B
:108BC0006CAF7DAF8EAF9FAFA7972091D409309146
:108BD000D5094091D6095091D709F501608171817D
:108BE000828193810E94EAB30E94E7BCAB966CAF8E
:108BF0007DAF8EAF9FAFAB978091B30983FF0EC05F
:108C0000AB962CAD3DAD4EAD5FADAB972093B60DA1
:108C10003093B70D4093B80D5093B90D8091B109C1
:108C20009091B209892B11F00C942251D6011C911C
:108C300011963C90119712962C90129713960C91C6
:108C40008091940D9091950D891B8F708F3019F440
:108C50000E94D92AF5CFB091940DAC96BFAFAC97D6
:108C60008091940DE82FF0E0FCA3EBA3FBE48F9F31
:108C7000C00111249C012F5F3A4F3AAF29AF809178
:108C8000AA0D9091AB0DA091AC0DB091AD0D6F966A
:108C90002CAD3DAD4EAD5FAD6F97281B390B4A0B28
:108CA0005B0BCA01B901C090AE0DD090AF0DE09042
:108CB000B00DF090B10DA3968CAC9DACAEACBFAC3A
:108CC000A3978C189D08AE08BF08C090B20DD09035
:108CD000B30DE090B40DF090B50DA7962CAD3DAD61
:108CE0004EAD5FADA7972C193D094E095F0969018B
:108CF0007A012B013C01442477FC439455246624DB
:108D00007724242DB7FC2260F7FC24603BE44BA1C0
:108D10005CA1349FF001359FF00D1124EF5FFA4FF5
:108D2000108225ABCDA2DEA2EFA2F8A6F7FE0BC003
:108D300022273327A9012C193D094E095F092DA3CC
:108D40003EA34FA358A72DA13EA14FA158A529A7E7
:108D50003AA74BA75CA78DA69EA6AFA6B8AAB7FE5A
:108D60000BC022273327A901281939094A095B09B1
:108D70002DA73EA74FA758AB2B013C0197FF07C07B
:108D8000442455243201461A570A680A790AA9ADC3
:108D9000BAAD55964D925D926D927C9258972DA5E5
:108DA0003EA54FA558A959962D933D934D935C939D
:108DB0005C972DA13EA14FA158A55D962D933D93A3
:108DC0004D935C9390970E948BB32091F104309166
:108DD000F2044091F3045091F4040E94EAB369ABA9
:108DE0007AAB8BAB9CAB698B7A8B8B8B9C8BC501E5
:108DF000B4010E948BB32091F5043091F6044091A8
:108E0000F7045091F8040E94EAB34B015C016D8BAA
:108E10007E8B8F8B988FC701B6010E948BB32091F8
:108E2000F9043091FA044091FB045091FC040E9433
:108E3000EAB36B017C01698F7A8F8B8F9C8F1D8EBB
:108E40001E8E1F8E18A2B6E04B16510461047104E9
:108E500004F52DA53EA54FA558A92630310541059D
:108E60005105BCF48DA19EA1AFA1B8A50697A1059F
:108E7000B1057CF48BE4ABA1BCA18A9FF0018B9F70
:108E8000F00D1124EF5FFA4F158616861786108AAB
:108E900060C0ADA9BEA92D913D914D915C912DABC6
:108EA0003EAB4FAB58AF20E030E0A9016DA97EA9E1
:108EB0008FA998AD0E9484B3882399F08BE42BA1ED
:108EC0003CA1829FF001839FF00D1124EF5FFA4FC8
:108ED0008DA99EA9AFA9B8AD85879687A787B08BC6
:108EE00038C029A93AA94BA95CA9CA01B9010E94B5
:108EF000EAB369AB7AAB8BAB9CABA5019401C5011E
:108F0000B4010E94EAB39B01AC0169A97AA98BA9BB
:108F10009CA90E947ABA4B015C01A7019601C70186
:108F2000B6010E94EAB39B01AC01C501B4010E94E5
:108F30007ABA0E9428BD2BE4ABA1BCA12A9FF00104
:108F40002B9FF00D1124EF5FFA4F65877687878797
:108F5000908B2DA13EA14FA158A5232B242B252B6F
:108F600021F419A61AA61BA61CA68DA59EA5AFA521
:108F7000B8A984159505A605B70510F4D301C2015B
:108F800029A53AA54BA55CA582179307A407B507A9
:108F900010F4DA01C9012BE44BA15CA1249FF0017C
:108FA000259FF00D1124EF5FFA4F85A396A3A7A389
:108FB000B0A70697A105B10510F40C94C251EA5B65
:108FC000FF4F8091F004808345284628472811F000
:108FD0005F9812988BE4ABA1BCA18A9FF0018B9F94
:108FE000F00D1124EF5FFA4F818D928DA38DB48D1A
:108FF000892B8A2B8B2B11F08A9847988BE42BA115
:109000003CA1829FF001839FF00D1124EF5FFA4F86
:10901000858D968DA78DB0A1892B8A2B8B2B29F05E
:1090200080910801817080930601C090F809D0906A
:10903000F909E090FA09F090FB099601A701612F68
:10904000732D822D902F0E9484B387FD04C0C12E02
:10905000D32CE22CF02E8BE44BA15CA1849FF00179
:10906000859FF00D1124EF5FFA4F258536854785E2
:10907000508960E070E080E89FE30E9474BB6DA3BC
:109080007EA38FA398A79601A7010E94EAB36B0164
:109090007C018091940D9091920D891B8F708FAF00
:1090A000A701960160E074E284E799E40E9474BB32
:1090B0000E94E7BC4B015C018FAD82508630C0F549
:1090C0008091C4099091C509A091C609B091C709C2
:1090D00088169906AA06BB0658F588199909AA099F
:1090E000BB09BC01CD01660F771F881F991F5FADBB
:1090F000052F10E020E030E0A90198010E94DAB9C4
:10910000CA01B9010E9489B30E94E7BC860E971E6E
:10911000A81EB91EC501B4010E9489B39B01AC0110
:1091200060E074E284E799E40E9474BB6B017C0107
:109130000E9482964091EC045091ED046091EE04FF
:109140007091EF04480D591D6A1D7B1D4093EC047E
:109150005093ED046093EE047093EF049BE4ABA195
:10916000BCA19A9FF0019B9FF00D1124E85BFA4F80
:1091700080829182A282B38281110E948F968BE4B9
:10918000EBA1FCA18E9F80018F9F100D11240F5F1A
:109190001A4FD8011D962D913D914D915C9150979C
:1091A00063962CAF3DAF4EAF5FAF6397A7019601BB
:1091B00063966CAD7DAD8EAD9FAD63970E94EAB3B3
:1091C0009B01AC010E94EAB36BAF7CAF8DAF9EAF49
:1091D000F801618372838383948345A056A067A0BE
:1091E00070A4C301B2010E9489B36DA77EA78FA7A7
:1091F00098AB9B01AC01C701B6010E94EAB30E9483
:1092000058BB0E94EDBB27966CAF7DAF8EAF9FAF72
:109210002797D801D6966D937D938D939C93D9977C
:10922000FE017196FEABEDAB28ED39E02D963FAF18
:109230002EAF2D97AE01435E5F4F5AA349A3212C59
:10924000312C50E859A78FE389ABADA9BEA92D9168
:109250003D914D915D91BEABADABC701B6010E9492
:10926000EAB34B015C0120E030E0A9010E94DABCC6
:1092700087FF04C0B7FAB094B7F8B0942D96AEAD9E
:10928000BFAD2D972D913D914D915D912D96BFAF25
:10929000AEAF2D972B962CAF3DAF4EAF5FAF2B9758
:1092A000A50194012B966CAD7DAD8EAD9FAD2B9736
:1092B0000E9484B387FF16C0A50194012B966CAD64
:1092C0007DAD8EAD9FAD2B970E9474BB5B018C0171
:1092D000910149A559A90E9484B387FF03C01501D4
:1092E00009A719ABEDA9FEA929A13AA1E217F30735
:1092F00009F0ABCF20E030E040E85FE3B10189A5A1
:1093000099A90E9484B387FF33C08BE44BA15CA171
:10931000849F8001859F100D11240F5F1A4F27969F
:109320006CAD7DAD8EAD9FAD27970E9489B3910145
:1093300049A559A90E94EAB30E94EDBBD801D6966F
:109340006D937D938D939C93D997910149A559A9CC
:10935000B10189A599A90E94EAB32BAD3CAD4DADF1
:109360005EAD0E94EAB3F8016183728383839483C4
:109370002DA53EA54FA558A96DA17EA18FA198A5A9
:109380000E94EAB36BAF7CAF8DAF9EAF8BE42BA195
:109390003CA1829FF001839FF00D1124EF5FFA4FF3
:1093A00085889688A788B08C81149104A104B104A3
:1093B00009F5818D928DA38DB48D892B8A2B8B2BF2
:1093C000C9F4858D968DA78DB0A1892B8A2B8B2B07
:1093D00089F42091EC093091ED094091EE0950910A
:1093E000EF096BAD7CAD8DAD9EAD0E94EAB30E94DE
:1093F00058BBE6C12091F0093091F1094091F20982
:109400005091F3096BAD7CAD8DAD9EAD0E94EAB37A
:109410000E9458BB0E94EDBB6B017C018091E80467
:109420009091E904A091EA04B091EB04E9ADFAADA2
:10943000218D328D438D548D29A73AA74BA75CA768
:10944000258D368D478D50A129AB3AAB4BAB5CAB2C
:1094500021A132A143A154A12DAB3EAB4FAB58AFDC
:1094600084159505A605B70508F4AFC081149104CD
:10947000A104B10471F16091D8047091D904809174
:10948000DA049091DB046C157D058E059F0508F5C7
:10949000A30192010E94CAB96DA77EA78FA798ABBE
:1094A000A5019401C701B6010E94CAB92DA53EA528
:1094B0004FA558A9261737074807590750F46DA537
:1094C0007EA58FA598A9A50194010E94DAB969012A
:1094D0007A0129A53AA54BA55CA5232B242B252B86
:1094E00051F16091DC047091DD048091DE04909173
:1094F000DF046C157D058E059F05E8F4A30192013C
:109500000E94CAB94B015C0129A53AA54BA55CA5EF
:10951000C701B6010E94CAB986169706A806B90601
:1095200050F4C501B40129A53AA54BA55CA50E943C
:10953000DAB969017A0189A99AA9ABA9BCA9892BD1
:109540008A2B8B2B51F16091E0047091E1048091A2
:10955000E2049091E3046C157D058E059F05E8F407
:10956000A30192010E94CAB94B015C0129A93AA941
:109570004BA95CA9C701B6010E94CAB98616970615
:10958000A806B90650F4C501B40129A93AA94BA906
:109590005CA90E94DAB969017A012DA93EA94FA9F7
:1095A00058AD232B242B252B09F40EC16091E40424
:1095B0007091E5048091E6049091E7046C157D05B7
:1095C0008E059F0508F440C6FFC081149104A104D4
:1095D000B104B9F16091D8047091D9048091DA0492
:1095E0009091DB046C157D058E059F0550F50E945A
:1095F00089B32DA53EA54FA558A90E94EAB32B011A
:109600003C01C501B4010E9489B34B015C01C70153
:10961000B6010E9489B3A50194010E94EAB39B019F
:10962000AC01C301B2010E9484B387FF0AC0A50147
:109630009401C301B2010E9474BB0E94EDBB6B0197
:109640007C0189A59AA5ABA5BCA5892B8A2B8B2B60
:10965000C9F16091DC047091DD048091DE04909189
:10966000DF046C157D058E059F0560F50E9489B3AA
:109670002DA53EA54FA558A90E94EAB34B015C0158
:1096800069A57AA58BA59CA50E9489B32B013C01F5
:10969000C701B6010E9489B3A30192010E94EAB3F7
:1096A0009B01AC01C501B4010E9484B387FF0AC0CD
:1096B000A3019201C501B4010E9474BB0E94EDBBDD
:1096C0006B017C0129A93AA94BA95CA9232B242B66
:1096D000252BC9F16091E0047091E1048091E204CE
:1096E0009091E3046C157D058E059F0560F50E9441
:1096F00089B32DA53EA54FA558A90E94EAB34B01F9
:109700005C0169A97AA98BA99CA90E9489B32B0144
:109710003C01C701B6010E9489B3A30192010E94D6
:10972000EAB39B01AC01C501B4010E9484B387FF79
:109730000AC0A3019201C501B4010E9474BB0E943A
:10974000EDBB6B017C018DA99EA9AFA9B8AD892B9A
:109750008A2B8B2BC9F16091E4047091E504809110
:10976000E6049091E7046C157D058E059F0560F574
:109770000E9489B32DA53EA54FA558A90E94EAB322
:109780004B015C016DA97EA98FA998AD0E9489B398
:109790002B013C01C701B6010E9489B3A3019201CC
:1097A0000E94EAB39B01AC01C501B4010E9484B3DD
:1097B00087FF0AC0A3019201C501B4010E9474BBD6
:1097C0000E94EDBB6B017C018BE4ABA1BCA18A9F25
:1097D00080018B9F100D11240F5F1A4FF801EE5B73
:1097E000FF4FC082D182E282F382C701B6010E949C
:1097F00089B36B017C012BAD3CAD4DAD5EAD0E94DC
:1098000074BB69AB7AAB8BAB9CABF801618B728B91
:10981000838B948B2DEB37E346E051E4C701B6010F
:109820000E94EAB30E94EDBBD801D1966D937D935F
:109830008D939C93D49729893A894B895C896DA132
:109840007EA18FA198A50E94EAB36BAF7CAF8DAFCC
:109850009EAF2D893E894F89588D6DA17EA18FA124
:1098600098A50E94EAB327966CAF7DAF8EAF9FAFED
:109870002797298D3A8D4B8D5C8D6DA17EA18FA18F
:1098800098A50E94EAB32B966CAF7DAF8EAF9FAFC9
:109890002B972D8D3E8D4F8D58A16DA17EA18FA14F
:1098A00098A50E94EAB32F966CAF7DAF8EAF9FAFA5
:1098B0002F97BFADBB2309F47CC2E091960DEDA3B9
:1098C000F091970DFDA73090980D2090990D2DEBFC
:1098D00037E346E855E3BF01832D922D0E9484B300
:1098E00087FD67C28090FC099090FD09A090FE0959
:1098F000B090FF09C090000AD090010AE090020ADF
:10990000F090030A2091040A3091050A4091060A5A
:109910005091070A2DAB3EAB4FAB58AF8091080A70
:109920009091090AA0910A0AB0910B0A23968CAF74
:109930009DAFAEAFBFAF2397C501B40190582BAD1B
:109940003CAD4DAD5EAD0E94EAB32B013C01C701B9
:10995000B601905827962CAD3DAD4EAD5FAD279723
:109960000E94EAB39B01AC01C301B2010E947ABA22
:109970002B013C016DA97EA98FA998AD90582B961B
:109980002CAD3DAD4EAD5FAD2B970E94EAB39B0170
:10999000AC01C301B2010E947ABA2B013C012396AB
:1099A0006CAD7DAD8EAD9FAD239790582F962CADAD
:1099B0003DAD4EAD5FAD2F970E94EAB39B01AC0168
:1099C000C301B2010E947ABA69A77AA78BA79CA7A4
:1099D0002FEE3FEF4FE75FE30E94DABC18160CF45E
:1099E000B7C12FEE3FEF4FE75FEB69A57AA58BA5D7
:1099F0009CA50E9484B387FF08C02FEE3FEF4FE77E
:109A00005FEB29A73AA74BA75CA7A50194016BAD13
:109A10007CAD8DAD9EAD0E9479BA2B013C0169836E
:109A20007A838B839C83A701960127966CAD7DADCD
:109A30008EAD9FAD27970E9479BA67966CAF7DAFC8
:109A40008EAF9FAF67976D837E838F8398872DA995
:109A50003EA94FA958AD2B966CAD7DAD8EAD9FAD97
:109A60002B970E9479BA6B966CAF7DAF8EAF9FAF8C
:109A70006B9769877A878B879C8723962CAD3DAD42
:109A80004EAD5FAD23972F966CAD7DAD8EAD9FAD86
:109A90002F970E9479BA23966CAF7DAF8EAF9FAFA0
:109AA00023976D877E878F87988BAE014F5F5F4FBF
:109AB0005EAB4DABCE0141969AA389A38A01C12C1E
:109AC000D12C7601D8018D909D90AD90BD908D01E7
:109AD00020E030E0A901C501B4010E9484B38823CD
:109AE00071F0A5019401C501B4010E94EAB39B0184
:109AF000AC01C701B6010E947ABA6B017C01E9A1F1
:109B0000FAA1E017F107F1F6C701B6010E9428BDDE
:109B10009B01AC0160E070E080E89FE30E9474BBB1
:109B20006B017C019B01AC01C301B2010E94EAB34D
:109B300069837A838B839C83A701960167966CADBA
:109B40007DAD8EAD9FAD67970E94EAB36D837E8336
:109B50008F839887A70196016B966CAD7DAD8EAD16
:109B60009FAD6B970E94EAB369877A878B879C8742
:109B7000A701960123966CAD7DAD8EAD9FAD239769
:109B80000E94EAB36D877E878F87988B04EB19E07C
:109B900049A86AA85BA87CA8ADA9BEA9CD90DD9014
:109BA000ED90FD90BEABADAB20E030E0A901C70168
:109BB000B6010E9484B3882331F1F801608171817C
:109BC000828193810E9489B3A70196010E9474BB90
:109BD0006B017C0120E030E0A9010E94DABC87FF24
:109BE00004C0F7FAF094F7F8F094242D362D452DA3
:109BF000572DC701B6010E9484B387FF04C04C2CC7
:109C00006D2C5E2C7F2C0C5F1F4F29A13AA14DA912
:109C10005EA92417350709F0BFCF29A53AA54BA5A2
:109C20005CA560E070E080E89FE30E9479BA20E0E4
:109C300030E040E05FE30E94EAB30E9428BD6B0180
:109C40007C012091D4043091D5044091D6045091E8
:109C5000D704642D762D852D972D0E94EAB3A70198
:109C600096010E94EAB34B015C01A701960160E0F6
:109C700070E080E89FE30E9479BA9B01AC01C501C6
:109C8000B4010E9474BB7B018C0120E030E040E80D
:109C90005FE363966CAD7DAD8EAD9FAD63970E9423
:109CA00084B387FF5BC029A53AA54BA55CA5CA0173
:109CB000B9010E94EAB323EC38EB42E35FEB0E9468
:109CC000EAB323EF36E64FE55FE30E9479BA29A5B0
:109CD0003AA54BA55CA50E94EAB32BED3FE049EC09
:109CE0005FE30E947ABA2CEE31E548E35EE30E941E
:109CF00079BA4B015C0124EE3BEC46E150E40E9452
:109D0000DABC18165CF5A50194016BED7FE089E4DF
:109D100090E40E9479BA9B01AC0163966CAD7DAD75
:109D20008EAD9FAD63970E9474BB242D362D452DBB
:109D3000572D0E94EAB35B016C019B01AC01B70196
:109D4000C8010E94DABC18164CF47501860106C0E1
:109D50003BE0E32E47EDF42E03E21BE38BE4ABA1E3
:109D6000BCA18A9FF0018B9FF00D1124EF5FFA4F89
:109D7000A180B280C380D4809501A6016DA17DA58C
:109D8000832D922D0E94DABC181624F4ADA2BDA634
:109D90003C2C2D2C9701A8016DA17DA5832D922D22
:109DA0000E94DABC18164CF4EDA2FDA6302E212E2E
:109DB00004C01DA21DA6312C212C2BAD3CAD4DADF8
:109DC0005EAD2093FC093093FD094093FE0950934A
:109DD000FF0927968CAD9DADAEADBFAD27978093A3
:109DE000000A9093010AA093020AB093030A2B96EB
:109DF0002CAD3DAD4EAD5FAD2B972093040A309353
:109E0000050A4093060A5093070A2F968CAD9DAD24
:109E1000AEADBFAD2F978093080A9093090AA09327
:109E20000A0AB0930B0A8BE4ABA1BCA18A9F800104
:109E30008B9F100D11240F5F1A4F8DA19DA5A32D8F
:109E4000B22DF80181879287A387B48769A97AA97F
:109E50008BA99CA990589B01AC010E947ABAA9AD2C
:109E6000BAAD1D962D913D914D915C9150970E94F8
:109E7000EAB39B01AC016BE077ED83E29BE30E94C8
:109E800079BA2BE0C22E27EDD22E23E2E22E2BE36D
:109E9000F22EF801C582D682E782F086B080C180BA
:109EA000D280E380F480A70196010E94DABC87FD8E
:109EB00002C083E001C081E0B82A8BE42BA13CA161
:109EC000829FF001839FF00D1124EF5FFA4FB08263
:109ED000C092960DD092970DE092980DF092990D48
:109EE0006F968CAD9DADAEADBFAD6F978093AA0D53
:109EF0009093AB0DA093AC0DB093AD0DA3962CAD8C
:109F00003DAD4EAD5FADA3972093AE0D3093AF0D39
:109F10004093B00D5093B10DA7968CAD9DADAEADF5
:109F2000BFADA7978093B20D9093B30DA093B40DDE
:109F3000B093B50DAB962CAD3DAD4EAD5FADAB97CF
:109F40002093B60D3093B70D4093B80D5093B90DD3
:109F50009091940D8091950D981303C084E68093A1
:109F6000910DAC968FADAC978F5F8F708093940DF1
:109F70008091940D9091930D81508F70891709F401
:109F800087C0F090940D8FEF8F0D8F708BA3B090E2
:109F9000930D8091940DB81609F451C0C12CD12CA9
:109FA0003BA13B1509F44BC0632E712C4BE4469D3D
:109FB0008001479D100D11240F5F1A4FD8018C911D
:109FC00083FD28C009AB1DAB1996BC91BDA3F80158
:109FD000F285FDA7D8011B96BC91B9AFF801F485B5
:109FE000F9A7D80115962D903D904D905C9018974B
:109FF000A20191016DA17DA589AD9F2F0E9484B31F
:10A00000811141C1C114D10439F0F601808180FD74
:10A010003AC102C0C9AADDAA8BA181508F708BA35F
:10A020008091930D8B1103C0C9A8DDA8B9CFFBA106
:10A03000FB1529F081E08B0D8F70B82EF1CF2091A8
:10A04000930D2BA3C12CD12C8091940D3BA1831790
:10A05000F9F0832E912C4BE4489D8001499D100D11
:10A0600011240F5F1A4FD8018C9183FD0AC058014B
:10A07000C114D10439F0C6010E94D255811102C029
:10A0800085C156018BA18F5F8F708BA36501DCCFDB
:10A09000D090950D8090940D2BE4D81469F08FEF3B
:10A0A000880D8F70289FF0011124EF5FFA4F908187
:10A0B00093FF02C0882EF1CF212C312C412C512C42
:10A0C0001BA21DA2712C612C00E010E0E12CF12CF0
:10A0D0008D1409F475C04BE44D9D800111240F5F70
:10A0E0001A4FD8018C9183FD19C015966D917D9101
:10A0F0008D919C9118970E9428BDC62EB72EA82E30
:10A10000992EE114F10409F44DC0F701808180FD1E
:10A110000AC0D8018C9180FD06C044C0CBA0BDA070
:10A12000A72C962C44C0F701808181608083C701F1
:10A130000E94D255811132C0F70161817281838101
:10A1400094810E9428BD9B01AC0160E070E080E832
:10A150009FE30E9474BB1B012C019B01AC016C2D81
:10A160007B2D8A2D992D0E94EAB369837A838B8394
:10A170009C832BA13DA1472D562DC201B1010E9408
:10A18000EAB3698B7A8B8B8B9C8BAE014F5F5F4FF1
:10A19000BE016F5E7F4FC7010E94AD94D7018C91C5
:10A1A0008E7F8C932C2C3B2C4A2C592C780181E0EF
:10A1B0008D0D8F70D82ECBA2BDA27A2C692C88CFA2
:10A1C0000115110509F4DEC0F801808181608083EA
:10A1D000C7010E94D255811130C0D80111966D91EE
:10A1E0007D918D919C9114970E9428BD9B01AC019B
:10A1F00060E070E080E89FE30E9474BB6B017C012B
:10A200002DEC3CEC4CE45DE30E94EAB369837A8375
:10A210008B839C839101A201C701B6010E94EAB31E
:10A22000698B7A8B8B8B9C8BAE014F5F5F4FBE012E
:10A230006F5E7F4FC8010E94AD94F80180818E7FD0
:10A240008083A0C080E01AC1A30192010E94CAB914
:10A250004B015C012DA93EA94FA958ADC701B6011C
:10A260000E94CAB986169706A806B90608F0ACCAB5
:10A27000C501B4012DA93EA94FA958AD0E94DAB974
:10A2800069017A01A1CA3BE4369DF001379DF00DCA
:10A290001124EF5FFA4F808181FD43C0C114D104C6
:10A2A00041F0D6011596CD90DD90ED90FC90189779
:10A2B00008C08BE0C82E87EDD82E83E2E82E8BE312
:10A2C000F82EBBE4B69DF001B79DF00D1124EF5FB1
:10A2D000FA4F81899289A389B489BC01CD01905834
:10A2E0009B01AC010E947ABAF80125853685478525
:10A2F00050890E94EAB39B01AC01C701B6010E94DC
:10A3000079BAE62E872E982EA92E262F372F482F82
:10A31000592F6DA17DA589AD99A50E9484B387FFB2
:10A3200004C0EDA08DA499ACA9A42E2D382D492DE3
:10A330005A2DC201B1010E9484B3882309F46CCE66
:10A34000FBE4F69DC001F79D900D11249C012F5F49
:10A350003A4F6901D9018C9181608C93C8010E94A8
:10A36000D255882329F0F60180818E7F808354CED8
:10A370008E2D982DA92DBA2DF60185839683A7835E
:10A38000B0874ACE0E948F9681E078C0D6018C912A
:10A3900081FD52C0D60115962D913D914D915C9154
:10A3A00018972DA33EA34FA358A71501B5E02B0E78
:10A3B000311CF8014580568067807084A3019201AA
:10A3C0006DA17EA18FA198A50E9484B387FF34C0A0
:10A3D000F60181899289A389B489BC01CD01905885
:10A3E0009B01AC010E947ABAD6011D962D913D9138
:10A3F0004D915C9150970E94EAB39B01AC016DA115
:10A400007EA18FA198A50E9479BA6B017C019B0166
:10A41000AC01C301B2010E94DABC18166CF4D80179
:10A420008C9181608C93C5010E94D2558823E1F004
:10A43000F80180818E7F80832BE4289DF001299D87
:10A44000F00D1124EF5FFA4F218532854385548545
:10A4500065817681878190850E9484B3811112CEB7
:10A460003BA13093930D0ECED101CD92DD92ED92B2
:10A47000FC921397BBA1B093930DDECFC559DF4F6C
:10A480000FB6F894DEBF0FBECDBFDF91CF911F9105
:10A490000F91FF90EF90DF90CF90BF90AF909F9083
:10A4A0008F907F906F905F904F903F902F90089586
:10A4B000CF92DF92EF92FF920F931F93CF93DF9390
:10A4C000CDB7DEB764970FB6F894DEBF0FBECDBF31
:10A4D000C98ADA8AEB8AFC8AFC0180819181A28197
:10A4E000B38189839A83AB83BC83FB018081918193
:10A4F000A281B3818D839E83AF83B887FA01808167
:10A500009181A281B38189879A87AB87BC87F90142
:10A5100080819181A281B3818D879E87AF87B88B1F
:10A520008091B1099091B209892B81F4CE014196B5
:10A530007C019E01235F3F4FAE01475F5F4FBE012D
:10A540006B5F7F4F40970E947F4501C080E064961B
:10A550000FB6F894DEBF0FBECDBFDF91CF911F9134
:10A560000F91FF90EF90DF90CF900895CF93DF93FE
:10A5700081110FC0EB010E94D2288DEE92E10E9462
:10A58000AC28CE010E94AC288AE0DF91CF910C94D8
:10A59000A528DF91CF9108954F925F926F927F929D
:10A5A0008F929F92AF92BF92CF92DF92EF92FF92E3
:10A5B0000F931F93CF93DF93EC01562E142F622E2F
:10A5C000442E400E5C018CE1A80EB11C822E912C11
:10A5D0001415E1F06701762C052D772099F0F6012E
:10A5E00084916A817B810C8F1D8F1F8E8E8F9501C8
:10A5F0004BE3CE010E942F68FFEFCF1ADF0A7A9457
:10A60000085FEBCFE80CF91C1F5FE2CFDF91CF9121
:10A610001F910F91FF90EF90DF90CF90BF90AF9080
:10A620009F908F907F906F905F904F9008950E94C1
:10A630005628811117C08091330F82FF0CC0809182
:10A64000B804811103C08BEA94E002C088EB94E067
:10A6500061E00C94E63E8091D304813031F086EDC8
:10A6600092E105C083EB92E102C081EE92E16FEFCF
:10A670000C94723E8DE19DE00E944A738DE19DE055
:10A680000E947D738091330F8D7F8E7F8093330F77
:10A6900010922F0F1092300F1092310F1092320F34
:10A6A00008950E94D2286091A9047091AA0483ECB5
:10A6B00092E10E94BB2880EC92E10C94AC28AF920E
:10A6C000BF92CF92DF92EF92FF920F931F93CF939F
:10A6D000DF93EC01062FE42E122FF22ED62ED20E8F
:10A6E000CC24CA945C018CE1A80EB11C8D2D8F196D
:10A6F00097E09F1570F46A817B818C8FED8E1F8EA1
:10A70000CE8E95014BE3CE010E942F6898EFF90E93
:10A71000EDCF812F86958695869598E0899F000DCF
:10A720001124212F98EF899F200D1124222309F154
:10A7300087E028276A817B810C8FED8E1F8E2F5F2B
:10A7400027708FEF90E001C0880F2A95EAF78E8F6F
:10A750009E01245E3F4F4BE3CE01DF91CF911F91CD
:10A760000F91FF90EF90DF90CF90BF90AF900C943F
:10A770002F68DF91CF911F910F91FF90EF90DF90A5
:10A78000CF90BF90AF90089561E0FC0180810E945E
:10A7900021438FEF0C941931EF92FF921F93CF93C7
:10A7A000DF9300D01F92CDB7DEB77C01162F29832F
:10A7B0003A834B835C83FC0182810E94253160E0F7
:10A7C000F70180810E9421430E9478A1812F80643B
:10A7D0000E9419318C810E9419318B810E9419319C
:10A7E0008A810E94193189810E941931112311F047
:10A7F00087E801C085E90E9419311C3011F40E94DC
:10A800001E3110E00E941E31F701838387FF04C0D0
:10A810001F3F11F01F5FF6CF0F900F900F900F901A
:10A82000DF91CF911F91FF90EF9008950F931F93A9
:10A83000CF93DF93EC0189018C81833039F089E07B
:10A84000440F551F661F771F8A95D1F79A01AB01F8
:10A8500068E1CE010E94CC53811128C08EEF8EBDDD
:10A86000F801C8019E5F0DB407FEFDCF20812EBD0B
:10A870000DB407FEFDCF21812EBD32968E179F07A6
:10A8800091F70DB407FEFDCF8FEF0E9419318FEFC6
:10A890000E9419310E941E318B838F71853041F0E7
:10A8A00083E18983CE010E94C45319C086E016C09B
:10A8B0000E9478A1882379F020E030E0A9016DE0C2
:10A8C000CE010E94CC53811108C00E941E3181111B
:10A8D00004C011E005C087E101C086E1898310E072
:10A8E000CE010E94C453812FDF91CF911F910F9110
:10A8F0000895CF92DF92EF92FF920F931F93CF9321
:10A90000DF93EC0189018C81833039F089E0440FB9
:10A91000551F661F771F8A95D1F79A01AB0161E138
:10A92000CE010E94CC53882339F084E08983CE0184
:10A930000E94C45380E03EC00E94C0A56B017C0110
:10A940002CE2C20E21E0D21EE11CF11C0E941E313D
:10A950008B838F3F61F40E94C0A5DC01CB018C1971
:10A960009D09AE09BF09B7FDF1CF81E11DC08E3F42
:10A97000D1F48FEF8EBDF801D801A150BE4F0DB4B8
:10A9800007FEFDCF9EB591938EBDEA17FB07B9F781
:10A990000DB407FEFDCF8EB58C930E941E310E9430
:10A9A0001E3111E003C08FE0898310E0CE010E94C8
:10A9B000C453812FDF91CF911F910F91FF90EF90A2
:10A9C000DF90CF900895809115028F3708F08F5750
:10A9D0008F5F809315029091770A81E08927809399
:10A9E000770A81110E94093F8091140218161CF009
:10A9F00091E0980F01C090E0882391F0813009F533
:10AA00008091760A811103C089E08093760A809153
:10AA1000760A81508093760A882399F091E011C0DC
:10AA2000809113028F5F80311CF48093130209C060
:10AA3000109213028091750A811103C081E0809306
:10AA4000750A909314028091930A81110E94EE9BE3
:10AA50008091B1099091B209009769F001979093A4
:10AA6000B2098093B109892B31F48AE19BE190937B
:10AA7000A50A8093A40A08950F930FB70F9300912E
:10AA80006E000B7F00936E0078940F930BB70F93BB
:10AA90000CB70F921F922F933F934F935F936F9337
:10AAA0007F938F939F93AF93BF93EF93FF93112463
:10AAB0000E94E354FF91EF91BF91AF919F918F91CD
:10AAC0007F916F915F914F913F912F911F900F90C8
:10AAD0000CBF0F910BBF0F910460F89400936E00B0
:10AAE0000F910FBF0F9118958091750A811101C0C8
:10AAF0000895A8951092750A0C94C0A5CF92DF9284
:10AB0000EF92FF92CF93DF93EC01C880D980EA8067
:10AB1000FB8080E19BE10E94AC28C701B6010E9446
:10AB2000B529CC80DD80EE80FF808CE295E20E942A
:10AB3000AC28C701B6010E94B529C884D984EA842B
:10AB4000FB8488E295E20E94AC28C701B6010E940E
:10AB5000B5298AE0DF91CF91FF90EF90DF90CF9001
:10AB60000C94A528CF93C82F0E94829694E0C99F89
:10AB700090011124F901EE5EF54FD901A25EB54FA7
:10AB80004D915D916D917C9140835183628373837C
:10AB900091E09093110A882319F0CF910C948F962D
:10ABA000CF910895BC012091730A3091740A4091AD
:10ABB000730A5091740A2417350711F09A01F7CFE0
:10ABC00081E02617370709F080E008952F923F9221
:10ABD0004F925F926F927F928F929F92AF92BF92AD
:10ABE000CF92DF92EF92FF920F931F93CF93DF9359
:10ABF00000D01F92CDB7DEB78FEF9FEF9093890003
:10AC0000809388000AE00983212C312C789480916C
:10AC10006F0A9091700AA091710AB091720A892B03
:10AC20008A2B8B2B71F080916F0A9091700AA09102
:10AC3000710AB091720A892B8A2B8B2B09F004C5FB
:10AC4000DCC18091110A8823D1F01092110A809101
:10AC5000730A9091740A892B91F01092100A109245
:10AC6000740A1092730A9091940D8091950D981723
:10AC700031F08091950D8F5F8F708093950D80914D
:10AC8000730A9091740A892B71F2C0906B0AD0906C
:10AC90006C0AE0906D0AF0906E0A4091670A50913C
:10ACA000680A6091690A70916A0A00915A0A10E074
:10ACB00020E030E0DB01CA018C199D09AE09BF0913
:10ACC000081719072A073B0710F4D901C801E82F14
:10ACD0008C0D9D1DAE1DBF1D80936B0A90936C0A59
:10ACE000A0936D0AB0936E0A1B821A82F1E0009164
:10ACF000320A1091330A2091340A3091350A80913A
:10AD0000420A9091430AA091440AB091450A080F63
:10AD1000191F2A1F3B1F0093420A1093430A2093D6
:10AD2000440A3093450A37FD31C080910C0A082E41
:10AD3000000C990BAA0BBB0B40911E0A50911F0AE5
:10AD40006091200A7091210A840F951FA61FB71FDA
:10AD500080931E0A90931F0AA093200AB093210AA1
:10AD600080912E0A90912F0AA091300AB091310A59
:10AD7000B901A801481B590B6A0B7B0B4093420A8F
:10AD80005093430A6093440A7093450A4091360AEF
:10AD90005091370A6091380A7091390A8091460AB9
:10ADA0009091470AA091480AB091490A480F591F4B
:10ADB0006A1F7B1F4093460A5093470A6093480AD4
:10ADC0007093490A77FD31C080910D0A082E000C5E
:10ADD000990BAA0BBB0BC090220AD090230AE090DB
:10ADE000240AF090250A8C0D9D1DAE1DBF1D809379
:10ADF000220A9093230AA093240AB093250A8091F3
:10AE00002E0A90912F0AA091300AB091310A4A017E
:10AE10005B01881A990AAA0ABB0A8092460A909294
:10AE2000470AA092480AB092490AC0903A0AD090C4
:10AE30003B0AE0903C0AF0903D0A80914A0A9091CA
:10AE40004B0AA0914C0AB0914D0A8C0D9D1DAE1D70
:10AE5000BF1D80934A0A90934B0AA0934C0AB0936B
:10AE60004D0AB7FD31C0C0900E0A0C2C000CDD0855
:10AE7000EE08FF088090260A9090270AA090280AE2
:10AE8000B090290AC80CD91CEA1CFB1CC092260AE7
:10AE9000D092270AE092280AF092290AC0902E0A3E
:10AEA000D0902F0AE090300AF090310A4C015D01F9
:10AEB0008C189D08AE08BF0880924A0A90924B0AEF
:10AEC000A0924C0AB0924D0A80903E0A90903F0AA0
:10AED000A090400AB090410AC0904E0AD0904F0A0C
:10AEE000E090500AF090510AC80CD91CEA1CFB1CD7
:10AEF000C0924E0AD0924F0AE092500AF092510A44
:10AF0000F7FC2FC080900F0A082C000C9908AA08A3
:10AF1000BB0840902A0A50902B0A60902C0A70902F
:10AF20002D0A840C951CA61CB71C80922A0A9092AC
:10AF30002B0AA0922C0AB0922D0A80902E0A909093
:10AF40002F0AA090300AB090310AC818D908EA0830
:10AF5000FB08C0924E0AD0924F0AE092500AF0923B
:10AF6000510AF1110CC0E0908400F0908500AA8095
:10AF7000BB80EA18FB08F2E0EF16F104A0F337FDFE
:10AF800002C0889A149A77FD02C08E9A419AB7FD42
:10AF900006C0F0910B01F095F870F09309018090D4
:10AFA0008400909085009B828A82E0908400F090DB
:10AFB0008500AA80BB80EA18FB08F2E0EF16F104D6
:10AFC000A0F337FD02C08898149877FD02C08E98D0
:10AFD0004198B7FD05C080910B01887080930901ED
:10AFE000EE2331F080908400909085009B828A82CD
:10AFF000E150F0E009F07BCE16CEE091730AF091BB
:10B00000740A309709F4A6C480916B0A90916C0A77
:10B01000A0916D0AB0916E0A4091670A5091680A3A
:10B020006091690A70916A0A84179507A607B707A5
:10B03000D0F01092100A1092740A1092730A909134
:10B04000940D8091950D981709F484C48091950D05
:10B050008F5F8F708093950D40EDC42E47E0D42E06
:10B06000E12CF12C4EC14091630A5091640A609129
:10B07000650A7091660A481759076A077B0708F442
:10B0800067C040915F0A5091600A6091610A7091B7
:10B09000620A81A992A9A3A9B4A99924499FA12CC4
:10B0A0005A9F90016A9F300D699F200D311D4A9F64
:10B0B000A00C211D391D599FA00C211D391D689F11
:10B0C000A00C211D391D589FA10C291D391DA694C6
:10B0D000291D391DB49F200D311DB59F300D112440
:10B0E00082AD93ADA4ADB5AD820F931FA11DB11D6F
:10B0F00080935B0A90935C0AA0935D0AB0935E0A0A
:10B1000006A917A920AD31AD081719072A073B0773
:10B1100040F400935B0A10935C0A20935D0A30931D
:10B120005E0A80905B0A90905C0AA0905D0AB090E5
:10B130005E0A80EF9AE121E0FC01C590D590E59090
:10B14000F490C814D904EA04FB0408F4CDC2D7C2B1
:10B150004091560A5091570A6091580A7091590AC5
:10B16000481759076A077B0708F063C04091520AE5
:10B170005091530A6091540A7091550A81A992A97D
:10B18000A3A9B4A98824499F912C5A9F90016A9F32
:10B19000300D699F200D311D4A9F900C211D381DD7
:10B1A000599F900C211D381D689F900C211D381D42
:10B1B000589F910C281D381D9694281D381DB49F4A
:10B1C000200D311DB59F300D1124C901A0E0B0E064
:10B1D00080905B0A90905C0AA0905D0AB0905E0A35
:10B1E000FE9688159905AA05BB0580F4008111819A
:10B1F00022813381881A990AAA0ABB0A801691060D
:10B20000A206B30638F44801590104C08080918039
:10B21000A280B38080EF9AE121E0FC01C590D59037
:10B22000E590F490C814D904EA04FB0408F4CFC2F2
:10B23000D9C280910F0290911002A0911102B09199
:10B240001202B7FF56C086A997A9A0ADB1AD20EFF5
:10B250003AE141E0F901C590D590E590F490C81627
:10B26000D906EA06FB0658F4B695A79597958795F3
:10B27000440F2C5F3F4FEBE12C303E0759F74093D2
:10B280005A0A80329105A105B10508F436C38097AA
:10B29000A109B109811508E09007A105B10508F4DD
:10B2A00009C314E0919F900111242051394EF901F6
:10B2B000329645915491EE27859FB001849F610D90
:10B2C0007E1F06946E1F7E1F1124CB01A0E0B0E00C
:10B2D000F9014591549160E070E0481B590B6A0BED
:10B2E0007B0B40930F0250931002609311027093F6
:10B2F0001202C0900F02D0901002E0901102F09064
:10B3000012028091730A9091740A892B09F094C1FA
:10B310000E94A3969093740A8093730A892B09F470
:10B320008BC18090730A9090740A9B828A82D401A8
:10B330008C9183FF3FC0F401858D968DA78DB0A1C0
:10B34000418D528D638D748D058916892789308DC5
:10B3500000931E0A10931F0A2093200A3093210A9B
:10B360004093220A5093230A6093240A7093250A7B
:10B370008093260A9093270AA093280AB093290A5B
:10B3800081A192A1A3A1B4A180932A0A90932B0A30
:10B39000A0932C0AB0932D0A9091940D8091950D55
:10B3A000981709F4B5CF8091950D8F5F8F708093BA
:10B3B000950DAECFAA81BB815596CD90DD90ED90D5
:10B3C000FC90589781E0C114D104E104F10409F420
:10B3D00080E0EA81FB81018D128D238D348D011572
:10B3E00011052105310509F08260AA81BB815D96B6
:10B3F0004D915D916D917C9190974115510561053D
:10B40000710509F084608093100A1092520A10921C
:10B41000530A1092540A1092550A10925F0A109221
:10B42000600A1092610A1092620AEA81FB8185A18A
:10B4300096A1A7A1B0A58093670A9093680AA093EC
:10B44000690AB0936A0A882499245401881A990ACF
:10B45000AA0ABB0A8092420A9092430AA092440A26
:10B46000B092450A8092460A9092470AA092480AF2
:10B47000B092490A80924A0A90924B0AA0924C0AD2
:10B48000B0924D0A80924E0A90924F0AA092500AB2
:10B49000B092510A81A092A0A3A0B4A0880C991CDC
:10B4A000AA1CBB1CCC0CDD1CEE1CFF1CC092320A7B
:10B4B000D092330AE092340AF092350A000F111F3D
:10B4C000221F331F0093360A1093370A2093380A3D
:10B4D0003093390A440F551F661F771F40933A0A6D
:10B4E00050933B0A60933C0A70933D0A80923E0A57
:10B4F00090923F0AA092400AB092410A880F991F89
:10B50000AA1FBB1F80932E0A90932F0AA093300A84
:10B51000B093310A10926B0A10926C0A10926D0A65
:10B5200010926E0A81A592A5A3A5B4A58093630A83
:10B530009093640AA093650AB093660A85A596A5C0
:10B54000A7A5B0A98093560A9093570AA093580ACA
:10B55000B093590A85A99091940A891721F0809394
:10B56000940A0E9407948091930A81110E94EE9B95
:10B5700088248A94982C540180920F029092100291
:10B58000A0921102B0921202EA81FB8182AD93ADCA
:10B59000A4ADB5AD80935B0A90935C0AA0935D0A5D
:10B5A000B0935E0A20EF3AE141E0F901C590D590F1
:10B5B000E590F490C816D906EA06FB0670F4B69535
:10B5C000A79597958795440F2C5F3F4F6CE0862E8B
:10B5D0006BE1962E8216930641F740935A0A803209
:10B5E0009105A105B10508F4B0C18097A109B10981
:10B5F0008115F8E09F07A105B10508F483C104E0B7
:10B60000909F900111242051394EF90132964591B5
:10B610005491EE27859FB001849F610D7E1F069493
:10B620006E1F7E1F1124F901C590D490E12CF12CDE
:10B63000C61AD70AE108F108C0926F0AD092700AC0
:10B64000E092710AF092720A80916F0A9091700AEA
:10B65000A091710AB091720A8F3F1FEF9107A10567
:10B66000B10528F04FEF5FEF60E070E002C0AC0181
:10B67000BD01841B950BA60BB70B80936F0A9093AB
:10B68000700AA093710AB093720AF89480918400B2
:10B69000909185004096098101500983002339F07B
:10B6A000240E351E2816390608F4B0CA01C01C0144
:10B6B000309289002092880078940F900F900F901C
:10B6C0000F90DF91CF911F910F91FF90EF90DF903E
:10B6D000CF90BF90AF909F908F907F906F905F9032
:10B6E0004F903F902F900895B694A7949794879485
:10B6F000220F04961BE18C30910709F01DCD209399
:10B700005A0A20E282169104A104B10408F459C037
:10B7100000E2801A9108A108B108811418E091068E
:10B72000A104B104F8F024E0929EC00111248051DC
:10B73000994EFC01329625913491F82DEE27F39F16
:10B74000D001F29FA10DBE1F0694AE1FBE1F112493
:10B75000FC01C590D490E12CF12CCA1ADB0AE10857
:10B76000F10822C0D501C401B695A7959795879594
:10B77000FC01EC7FCF0180519D4EFC01C590D4901F
:10B78000FC01329625913491E82DE770E29FC001CB
:10B79000E39F900D112433E0969587953A95E1F754
:10B7A000C81AD90AE12CF12C4C0D5D1D6E1D7F1DB0
:10B7B00040935F0A5093600A6093610A7093620A33
:10B7C000A0CDA0E28A2E912CA12CB12CA1CFB694B1
:10B7D000A79497948794220F04963BE18C309307AB
:10B7E00009F01BCD20935A0A80E288169104A10427
:10B7F000B10408F459C000E2801A9108A108B10808
:10B80000811418E09106A104B104F8F024E0929E9E
:10B81000C00111248051994EFC013296259134913A
:10B82000F82DEE27F39FD001F29FA10DBE1F0694C5
:10B83000AE1FBE1F1124FC01C590D490E12CF12C49
:10B84000CA1ADB0AE108F10822C0D501C401B69585
:10B85000A79597958795FC01EC7FCF0180519D4E70
:10B86000FC01C590D490FC01329625913491E82DCD
:10B87000E770E29FC001E39F900D112403E09695CD
:10B8800087950A95E1F7C81AD90AE12CF12C4C0DDD
:10B890005D1D6E1D7F1D4093520A5093530A6093A5
:10B8A000540A7093550A2DCDE0E28E2E912CA12CD6
:10B8B000B12CA1CFAC01BD01769567955795479501
:10B8C000FA01EC7F9F0120513D4EF90145915491C1
:10B8D000F9013296659174918770869F9001879FD8
:10B8E000300D1124C901F3E096958795FA95E1F79B
:10B8F000481B590B60E070E0F4CC80E290E0A0E0DF
:10B90000B0E0C5CCAC01BD017695679557954795DC
:10B91000FA01EC7F9F0120513D4EF901C590D49072
:10B92000F9013296459154918770849F9001859FCB
:10B93000300D1124C90103E0969587950A95E1F72A
:10B94000C81AD90AE12CF12C77CE80E290E0A0E071
:10B95000B0E04BCE80EDC82E87E0D82EE12CF12C44
:10B96000D7CC8F929F92AF92BF92CF92DF92EF92FD
:10B97000FF920F931F93CF93DF93CDB7DEB7CA58D3
:10B98000D1090FB6F894DEBF0FBECDBFC358DF4F4D
:10B99000188219821A821B82CD57D0408091F402FE
:10B9A0009091F502A091F602B091F702CF57DF4FC8
:10B9B00088839983AA83BB83C158D040CB57DF4F7C
:10B9C00019821882C558D04084E690E0C957DF4FED
:10B9D00099838883C758D0401092900A9E012B57B4
:10B9E0003F4F44E050E0BE016F577F4FCE01895773
:10B9F0009F4F0E94D628C957DF4F88819981C75829
:10BA0000D0400296C957DF4F99838883C758D040EA
:10BA1000CB57DF4F19821882C558D040DD24D3940C
:10BA2000C657DF4FD882CA58D0409E012B573F4F90
:10BA300041E050E0BE0166577F4FCE0189579F4FCE
:10BA40000E94D6289E012B573F4F48E450E064EBFC
:10BA500079E0CE0189579F4F0E94D62880E1E2E528
:10BA6000F2E08E010F5F1F4FD80101900D928A9571
:10BA7000E1F79E012B573F4F40E150E0B801CE0166
:10BA800089579F4F0E94D6289E012B573F4F44E075
:10BA900050E064ED74E0CE0189579F4F0E94D62894
:10BAA0009E012B573F4F4CE050E066E97AE0CE0113
:10BAB00089579F4F0E94D6287E018DE6E80EF11C23
:10BAC000F701D08219821A821B821C829E012B5799
:10BAD0003F4F41E050E0B701CE0189579F4F0E9490
:10BAE000D6289E012B573F4F44E050E0B801CE01CD
:10BAF00089579F4F0E94D62880E090E0A0E2B1E4F1
:10BB000089839A83AB83BC839E012B573F4F44E0CC
:10BB100050E0B801CE0189579F4F0E94D628C358E4
:10BB2000DF4F188219821A821B82CD57D04083E0E2
:10BB3000F701808389839E012B573F4F44E050E0FB
:10BB4000BE0163587F4FCE0189579F4F0E94D62870
:10BB50009E012B573F4F41E050E0B701CE0189577E
:10BB60009F4F0E94D6289E012B573F4F41E050E047
:10BB7000B801CE0189579F4F0E94D6283AE0D32EB4
:10BB8000DA94DD2071F09E012B573F4F44E050E0E6
:10BB9000BE0163587F4FCE0189579F4F0E94D62820
:10BBA000EFCF8CE0F80111928A95E9F79E012B57AF
:10BBB0003F4F4CE050E0B801CE0189579F4F0E94A3
:10BBC000D628C358DF4F188219821A821B82CD579C
:10BBD000D0402AE0D22EDA94DD2071F09E012B575E
:10BBE0003F4F44E050E0BE0163587F4FCE0189577C
:10BBF0009F4F0E94D628EFCF88E0F701982F11922F
:10BC00009A95E9F7F80111928A95E9F783E0C75709
:10BC1000DF4F8883C958D040EA968FAFEA979E01DC
:10BC20002B573F4F41E050E0BE0167577F4FCE0199
:10BC300089579F4F0E94D6289E012B573F4F41E0C6
:10BC400050E0BE0167587F4FCE0189579F4F0E9439
:10BC5000D6289E012B573F4F48E050E0B801CE0157
:10BC600089579F4F0E94D6289E012B573F4F48E08F
:10BC700050E0B701CE0189579F4F0E94D628C35884
:10BC8000DF4F188219821A821B82CD57D0400AE0FA
:10BC900010E00150110971F09E012B573F4F44E015
:10BCA00050E0BE0163587F4FCE0189579F4F0E94DD
:10BCB000D628EFCFF70110828FEF89839E012B5793
:10BCC0003F4F41E050E0B701CE0189579F4F0E949E
:10BCD000D6289E012B573F4F41E050E08E010F5F69
:10BCE0001F4FB801CE0189579F4F0E94D62880E18F
:10BCF000F80111928A95E9F79E012B573F4F40E1D9
:10BD000050E0B801CE0189579F4F0E94D628198272
:10BD10009E012B573F4F41E050E0B801CE018957BB
:10BD20009F4F0E94D6288091620290916302A09159
:10BD30006402B0916502F70180839183A283B3838B
:10BD40008091660290916702A0916802B0916902A9
:10BD500089839A83AB83BC83EA961FAEEA97EB96FE
:10BD60001FAEEB979E012B573F4F44E050E0B701C9
:10BD7000CE0189579F4F0E94D6289E012B573F4FD7
:10BD800044E050E0B801CE0189579F4F0E94D62869
:10BD90009E012B573F4F42E050E0BE0167587F4F56
:10BDA000CE0189579F4F0E94D62884E190E09A8364
:10BDB00089839E012B573F4F42E050E0B801CE01EE
:10BDC00089579F4F0E94D6288CE0EAE6F2E0D8011E
:10BDD00001900D928A95E1F79E012B573F4F4CE061
:10BDE00050E0B801CE0189579F4F0E94D6288FE7B7
:10BDF00090E09A8389839E012B573F4F42E050E0A9
:10BE0000B801CE0189579F4F0E94D62885E0EEECFD
:10BE1000F2E0D80101900D928A95E1F79E012B572F
:10BE20003F4F45E050E0B801CE0189579F4F0E9437
:10BE3000D62819829E012B573F4F41E050E0B801B0
:10BE4000CE0189579F4F0E94D62880E2E6E7F2E0B4
:10BE5000D80101900D928A95E1F79E012B573F4F33
:10BE600040E250E0B801CE0189579F4F0E94D6288A
:10BE7000F70110829E012B573F4F41E050E0B70180
:10BE8000CE0189579F4F0E94D6281982812C912C70
:10BE900080E4A82EBA2CC358DF4F88829982AA82E8
:10BEA000BB82CD57D0409E012B573F4F41E050E021
:10BEB000B801CE0189579F4F0E94D6288CE1F80126
:10BEC00011928A95E9F79E012B573F4F4CE150E0C4
:10BED000B801CE0189579F4F0E94D62888E3E6E932
:10BEE000F2E0D80101900D928A95E1F79E012B575F
:10BEF0003F4F48E350E0B801CE0189579F4F0E9461
:10BF0000D62888E0F80111928A95E9F79E012B570F
:10BF10003F4F48E050E0B801CE0189579F4F0E9443
:10BF2000D6288EE0F80111928A95E9F79E012B57E9
:10BF30003F4F4EE050E0B801CE0189579F4F0E941D
:10BF4000D628C358DF4F188219821A821B82CD5718
:10BF5000D0409E012B573F4F44E050E0BE01635854
:10BF60007F4FCE0189579F4F0E94D6289CE0D92E43
:10BF7000F8018D2D11928A95E9F79E012B573F4FBD
:10BF80004CE050E0B801CE0189579F4F0E94D6285F
:10BF90008CE6F80111928A95E9F79E012B573F4FE5
:10BFA0004CE650E0B801CE0189579F4F0E94D62839
:10BFB0009E012B573F4F4CE050E064E87AE0CE0101
:10BFC00089579F4F0E94D628F7011192DA94E9F71A
:10BFD000C757DF4F1882C958D040ED968CAE9DAE42
:10BFE000AEAEBFAEED979E012B573F4F4CE050E0F9
:10BFF000B701CE0189579F4F0E94D6289E012B572B
:10C000003F4F41E050E0BE0167577F4FCE01895757
:10C010009F4F0E94D6289E012B573F4F44E050E08F
:10C02000BE0167587F4FCE0189579F4F0E94D62887
:10C030001091900A111156C0C957DF4FC880D9809E
:10C04000C758D040F4E6CF1AD108CB57DF4F8881CC
:10C050009981C558D040F7019183808384E690E0B0
:10C06000C957DF4F99838883C758D0409E012B570B
:10C070003F4F44E050E068EF72E0CE0189579F4F98
:10C080000E94D6289E012B573F4F42E050E0B70157
:10C09000CE0189579F4F0E94D6280E94D228B60110
:10C0A00083E39BE10E94A829F7014081518160E070
:10C0B00070E086E29BE10E94972980E498E00E946C
:10C0C000AC28F0E6CF16F2E0DF0639F00E94CE2869
:10C0D00085E49BE10E94AC2811E08091900A182B26
:10C0E0001093900A9091900A81E08927C657DF4FFC
:10C0F0000FB6F894DEBF0FBECDBFDF91CF911F9179
:10C100000F91FF90EF90DF90CF90BF90AF909F90F6
:10C110008F9008952F923F924F925F926F927F92ED
:10C120008F929F92AF92BF92CF92DF92EF92FF9247
:10C130000F931F93CF93DF9300D0CDB7DEB740901E
:10C14000010D5090020D6090030D7090040D8090D1
:10C15000050D9090060DA090070DB090080DC090B1
:10C16000090DD0900A0DE0900B0DF0900C0D0E947F
:10C17000459408EC12E287E192E09B838A8384ED88
:10C18000282E82E2382E198289810E94FA98F801BD
:10C1900085919591A591B491EA81FB8181939193C9
:10C1A000A193B193FB83EA83F10185919591A591C8
:10C1B000B491EA81FB8180879187A287B387F98157
:10C1C000FF5FF9830C5F1F4F84E0280E311CF330B2
:10C1D000D9F60E9430982091010D3091020D4091C6
:10C1E000030D5091040DC301B2010E9484B381116B
:10C1F0001CC0A50194016091050D7091060D809100
:10C20000070D9091080D0E9484B381110EC02091FA
:10C21000090D30910A0D40910B0D50910C0DC70185
:10C22000B6010E9484B38823B9F00F900F900F904D
:10C23000DF91CF911F910F91FF90EF90DF90CF9002
:10C24000BF90AF909F908F907F906F905F904F9036
:10C250003F902F900C94C79B0F900F900F90DF9101
:10C26000CF911F910F91FF90EF90DF90CF90BF90F3
:10C27000AF909F908F907F906F905F904F903F9086
:10C280002F9008953F924F925F926F927F928F927C
:10C290009F92AF92BF92CF92DF92EF92FF920F9355
:10C2A0001F93CF93DF93CDB7DEB7C658D1090FB632
:10C2B000F894DEBF0FBECDBF4DB65EB6C158DF4F9E
:10C2C00019821882CF57D04084E690E0CF57DF4FD5
:10C2D00099838883C158D04001E09E0121583F4F87
:10C2E00044E050E0BE0167587F4FCE018F579F4F0B
:10C2F0000E9468289E0121583F4F42E050E0BE0155
:10C300006D577F4FCE018F579F4F0E94682843E0A3
:10C3100050E0BE0167587F4F88EF92E00E94EABD6F
:10C32000892B11F1ED968FADED97882339F08FE3CE
:10C33000EA968FAFEA97EB961FAEEB970E94D22852
:10C34000BE0167587F4F8BEF9BE10E94BB288DEEAB
:10C350009BE10E94AC2860E089ED9BE10E94723E67
:10C3600081E08093900ABAC4E9961CAE1DAE1EAE61
:10C370001FAEE997C158DF4F19821882CF57D040BE
:10C3800001E09E0121583F4F41E050E0BE016A5755
:10C390007F4FCE018F579F4F0E9468286DB67EB6A3
:10C3A000CA57DF4FE880C658D040F12C23E0E20E98
:10C3B000F11CEE0CFF1CEE0CFF1C8DB79EB78E1906
:10C3C0009F090FB6F8949EBF0FBE8DBFEDB7FEB7A5
:10C3D00031964F018E199F090FB6F8949EBF0FBE7C
:10C3E0008DBFEDB7FEB731966F018E199F090FB65D
:10C3F000F8949EBF0FBE8DBFEDB7FEB731965F01BB
:10C400000091FB0C11E001279E0121583F4FA7012D
:10C41000B401CE018F579F4F0E9468280091FB0CFA
:10C4200001279E0121583F4F44E050E064EC79E041
:10C43000CE018F579F4F0E9468280091FB0C012767
:10C440009E0121583F4FA701B601CE018F579F4F44
:10C450000E9468280091FB0C01279E0121583F4F44
:10C46000A701B501CE018F579F4F0E946828009108
:10C47000FB0C002309F44EC011E001279E01215856
:10C480003F4F44E050E068EE79E0CE018F579F4F78
:10C490000E9468280091FB0C01279E0121583F4F04
:10C4A00044E050E06CEE79E0CE018F579F4F0E9440
:10C4B00068280091FB0C01279E0121583F4F44E062
:10C4C00050E060EF79E0CE018F579F4F0E946828BF
:10C4D0000091FB0C01279E0121583F4F44E050E0A2
:10C4E00064EF79E0CE018F579F4F0E94682800913A
:10C4F000FB0C01279E0121583F4F44E050E068EFBC
:10C5000079E0CE018F579F4F0E94682815E0FF24E5
:10C51000F3948AC0CA57DF4F2881C658D04030E014
:10C520002E5F3F4FD60144EB59E080E090E02817A2
:10C53000390734F0F401C080D180E280F38010C06C
:10C54000FC018430910510F0E3E0F0E0EE0FFF1FF6
:10C55000EE0FFF1FEC5EFA4DC590D590E590F4907C
:10C56000FA01C192D192E192F192AF0128173907F5
:10C570005CF0EC9111967C91119712966C91129748
:10C580001396FC91139714C0FC018430910510F0B0
:10C59000E3E0F0E0EE0FFF1FEE0FFF1FEC5FFA4D40
:10C5A000C590D590E590F490EC2D7D2D6E2DFF2D4E
:10C5B000CE2ED72EE62EFF2EFA01C08AD18AE28A2D
:10C5C000F38A2817390734F0F501108171816281EF
:10C5D000338014C0FC018430910510F0E3E0F0E0FA
:10C5E000EE0FFF1FEE0FFF1FEC50FB4DC590D590D7
:10C5F000E590F4901C2D7D2D6E2D3F2CC12ED72E55
:10C60000E62EF32CFA01C0A2D1A2E2A2F3A2019677
:10C61000F4E0AF0EB11C149664E0860E911C8430D9
:10C62000910509F084CF28CF11500091FB0C112304
:10C6300079F00F259E0121583F4F44E050E0BE01A4
:10C640006B587F4FCE018F579F4F0E946828ECCFC9
:10C6500011E001279E0121583F4F44E050E064ED76
:10C6600074E0CE018F579F4F0E9468280FB6F89450
:10C670007EBE0FBE6DBE0091FB0C01279E012158AE
:10C680003F4F4CE050E066E97AE0CE018F579F4F74
:10C690000E9468280091FB0C01279E0121583F4F02
:10C6A00041E050E0BE0163597F4FCE018F579F4F4D
:10C6B0000E9468280091FB0C01279E0121583F4FE2
:10C6C00044E050E0BE016F5F7F4FCE018F579F4F18
:10C6D0000E9468280091FB0C01279E0121583F4FC2
:10C6E00044E050E0BE016B587F4FCE018F579F4F03
:10C6F0000E9468280091FB0C01279E0121583F4FA2
:10C7000044E050E0BE016B587F4FCE018F579F4FE2
:10C710000E94682801E09E0121583F4F41E050E00F
:10C72000BE0163597F4FCE018F579F4F0E946828EB
:10C730009E0121583F4F41E050E0BE016F5F7F4FA7
:10C74000CE018F579F4F0E946828AE968FADAE974F
:10C75000C9808C9D60011124E12CF12C0091FB0C0F
:10C76000EC14FD0491F001279E0121583F4F44E055
:10C7700050E0BE016B587F4FCE018F579F4F0E94F4
:10C7800068288FEFE81AF80AE9CF81E008279E01B0
:10C7900021583F4F4CE050E0BE016F5F7F4FCE010C
:10C7A0008F579F4F0E9468281AE0FF24F39411507E
:10C7B00089F00091FB0C0F259E0121583F4F44E06A
:10C7C00050E0BE016B587F4FCE018F579F4F0E94A4
:10C7D0006828EDCF01E09E0121583F4F41E050E035
:10C7E000BE016B577F4FCE018F579F4F0E94682825
:10C7F0009E0121583F4F41E050E0BE0163587F4FFA
:10C80000CE018F579F4F0E9468280091FB0C11E0CA
:10C8100001279E0121583F4F48E050E0BE01635977
:10C820007F4FCE018F579F4F0E9468280091FB0CCD
:10C8300001279E0121583F4F48E050E0BE016F5F45
:10C840007F4FCE018F579F4F0E946828CB57DF4FF5
:10C850008881C558D040EE96CFACEE978C9D600194
:10C860001124E12CF12C0091FB0CCE14DF0491F08B
:10C8700001279E0121583F4F44E050E0BE016B5814
:10C880007F4FCE018F579F4F0E9468289FEFE91A74
:10C89000F90AE9CF11E001279E0121583F4F41E0FD
:10C8A00050E0BE0163597F4FCE018F579F4F0E94CA
:10C8B00068280091FB0C01279E0121583F4F41E061
:10C8C00050E0FE0131967F01BF01CE018F579F4F8F
:10C8D0000E9468280091FB0C01279E0121583F4FC0
:10C8E00040E150E0B701CE018F579F4F0E9468286A
:10C8F0000091FB0C01279E0121583F4F41E050E081
:10C90000B701CE018F579F4F0E9468280091FB0C02
:10C9100001279E0121583F4F44E050E0BE0163597A
:10C920007F4FCE018F579F4F0E9468280091FB0CCC
:10C9300001279E0121583F4F44E050E0B701CE014E
:10C940008F579F4F0E9468280091FB0C01279E0182
:10C9500021583F4F42E050E0BE0163587F4FCE0167
:10C960008F579F4F0E9468280091FB0C01279E0162
:10C9700021583F4F42E050E0B701CE018F579F4F03
:10C980000E9468280091FB0C01279E0121583F4F0F
:10C990004CE050E0B701CE018F579F4F0E946828AE
:10C9A0000091FB0C01279E0121583F4F42E050E0CF
:10C9B000B701CE018F579F4F0E94682885E0F7018D
:10C9C00011928A95E9F70091FB0C01279E012158ED
:10C9D0003F4F45E050E0B701CE018F579F4F0E9477
:10C9E00068280091FB0C01279E0121583F4F41E030
:10C9F00050E0B701CE018F579F4F0E9468280091E9
:10CA0000FB0C01279E0121583F4F40E250E0B70147
:10CA1000CE018F579F4F0E9468280091FB0C012781
:10CA20009E0121583F4F41E050E0BE0163597F4FC6
:10CA3000CE018F579F4F0E9468280091FB0C012761
:10CA40009E0121583F4F41E050E0B701CE018F5782
:10CA50009F4F0E9468280091FB0C01279E012158DE
:10CA60003F4F4CE150E0B701CE018F579F4F0E94DE
:10CA700068280091FB0C01279E0121583F4F48E395
:10CA800050E0B701CE018F579F4F0E946828009158
:10CA9000FB0C01279E0121583F4F48E050E0B701B1
:10CAA000CE018F579F4F0E9468280091FB0C0127F1
:10CAB0009E0121583F4F4EE050E0B701CE018F5705
:10CAC0009F4F0E9468280091FB0C01279E0121586E
:10CAD0003F4F44E050E0B701CE018F579F4F0E9477
:10CAE00068280091FB0C01279E0121583F4F4CE024
:10CAF00050E0B701CE018F579F4F0E9468280091E8
:10CB0000FB0C01279E0121583F4F4CE650E0B70136
:10CB1000CE018F579F4F0E94682819821A821B826C
:10CB20001C821D821E821F82188619861A861B8609
:10CB30001C860091FB0C01279E0121583F4F4CE0C1
:10CB400050E0B701CE018F579F4F0E946828009197
:10CB5000FB0C01279E0121583F4F4CE050E0B701EC
:10CB6000CE018F579F4F0E9468280091FB0C012730
:10CB70009E0121583F4F41E050E0BE0163587F4F76
:10CB8000CE018F579F4F0E9468280091FB0C012710
:10CB90009E0121583F4F44E050E0BE0163597F4F52
:10CBA000CE018F579F4F0E946828CF57DF4F888153
:10CBB0009981C158D040843C924041F00E94CE28D7
:10CBC00085E49BE10E94AC2881E001C080E0809375
:10CBD000900A8823D9F00E94D228CF57DF4F68816E
:10CBE0007981C158D0406456710981ED9BE10E9462
:10CBF000D12960E672E084E99FE10E94A8298AE0D9
:10CC00000E94A52860E08FEB9BE12FC0C158DF4F49
:10CC100028813981CF57D040CD57DF4F8881998106
:10CC2000C358D0402817390719F181E08093900A42
:10CC30000E94CE28CD57DF4F68817981C358D040FC
:10CC40008FE99BE10E94A829C158DF4F6881798153
:10CC5000CF57D0408AE99BE10E94A8298AE89BE14E
:10CC60000E94AC2860E08AE79BE10E94723E2CC0E3
:10CC70008091FB0C811128C00E94D22808EF12E09D
:10CC8000F80181918F01882319F00E94A528F8CF1F
:10CC9000CF57DF4F68817981C158D0406456710900
:10CCA0008DE59BE10E94D129C158DF4F4881598110
:10CCB000CF57D04060E070E086E29BE10E94972968
:10CCC00080E498E00E94AC288091FB0C811106C0A2
:10CCD0008091900A811102C00E948A608091FB0CB1
:10CCE000811107C08091290C813019F480E00E94E5
:10CCF000759C9091900A81E089270FB6F8945EBEEA
:10CD00000FBE4DBECA57DF4F0FB6F894DEBF0FBE41
:10CD1000CDBFDF91CF911F910F91FF90EF90DF90EA
:10CD2000CF90BF90AF909F908F907F906F905F90CB
:10CD30004F903F9008950F931F938091D3048130BB
:10CD400019F40E94C0A508C06091780A7091790A10
:10CD500080917A0A90917B0A0091800A1091810A51
:10CD60002091820A3091830A601B710B820B930B16
:10CD700028EE33E040E050E00E94DAB980917C0A6E
:10CD800090917D0AA0917E0AB0917F0ABC01CD01ED
:10CD9000620F731F841F951F1F910F9108951092AA
:10CDA000D3041092800A1092810A1092820A109283
:10CDB000830A1092780A1092790A10927A0A1092D5
:10CDC0007B0A10927C0A10927D0A10927E0A1092C1
:10CDD0007F0A08958091D3048130F1F0823059F4B4
:10CDE0000E949B6660937C0A70937D0A80937E0A02
:10CDF00090937F0A02C00E94CF6681E08093D304A3
:10CE00000E94C0A56093800A7093810A8093820A71
:10CE10009093830A81E0089580E008958091D3047F
:10CE20008150823010F080E008951092D3040E9467
:10CE3000C0A56093780A7093790A80937A0A9093D8
:10CE40007B0A81E00895CF92DF92EF92FF920F93D9
:10CE50001F93CF93DF936C017A018B01C0E0D0E088
:10CE6000CE15DF0581F0D8016D918D01D601ED91D0
:10CE7000FC910190F081E02DC6011995892B11F0EC
:10CE80002196EECF7E01C701DF91CF911F910F91C7
:10CE9000FF90EF90DF90CF90089508950E9487BD96
:10CEA000FC0130819281930F92832181921760F46B
:10CEB00094819F5F94838381830F821710F08FEF9B
:10CEC000820F838381E0089580E00895FC0112823F
:10CED00080818150838314820895FB014181DC01AC
:10CEE00012962C911297421768F013962C91139773
:10CEF000241740F0608115962C91621718F4248154
:10CF00000C940268089580E008950B96FC018491CA
:10CF100008950A96FC0184910895FC018491089576
:10CF20000E948D67882321F0823011F083E00895FC
:10CF300086E00895FC01E60FF11D849190E0982FA2
:10CF400088273196E4918E0F911D089568E00C9426
:10CF50009A6766E00C949A6781E008951F93CF93D7
:10CF6000DF93182FEB010E94D22884EB90E20E94FD
:10CF7000AC28113019F088EA90E202C08EEA90E203
:10CF80000E94AC28BE0180EA90E20E94BB288AE0A1
:10CF9000DF91CF911F910C94A528CF93DF93EC01E3
:10CFA000CB01E881F981608171810E94867388815B
:10CFB0009981DC01ED91FC912081AA81BB81222322
:10CFC00069F02C91293650F43196DC01ED93FC93F5
:10CFD000EA81FB8180818F5F8083E9CF8C918936E4
:10CFE00070F48FE28083E881F981808191810196DC
:10CFF00091838083EA81FB8180818F5F8083DF91D1
:10D00000CF910895FC01A681B7818281481B85815B
:10D01000483018F0A80FB11D4770382F3695369557
:10D020003695562F577080E890E002C09595879509
:10D030005A95E2F7439F402D1124669566956695B3
:10D04000E62FF0E0E40FF11DEA0FFB1F30812223F1
:10D0500011F0832B02C08095832380830895DB0128
:10D06000ED91FC911994DC0114968D919C9115978A
:10D070008617970709F44EC015967C936E93149704
:10D080006115710509F440C057968C915797FB01C3
:10D09000811108C03596E4915896EC935897FB019E
:10D0A0003C9611C0813041F43F96E4915896EC9340
:10D0B0005897FB01709607C03D96E4915896EC9303
:10D0C0005897FB013E96649159966C9359975896E0
:10D0D0008C915897082E000C990B59962C915997C2
:10D0E000821B910927FD93955A962C915A972034CB
:10D0F00041F0829FC001112426E0969587952A95DC
:10D10000E1F75B968C935B9783E897E656969C9342
:10D110008E9355970895BF92CF92DF92EF92FF9230
:10D120000F931F93CF93DF938C01E62EDC011496AF
:10D13000CD91DC911597CE010E948D67F82EF801F4
:10D14000848195810E949067C82EF1E0FF1203C090
:10D150002FE0B22E02C0BB24BA94D80114968D9150
:10D160009C9115970E948967F82EF801848195811A
:10D170000E948567D82ED80114968D919C911597A1
:10D180000E94A667B0E6BE1538F4009729F0C80FD4
:10D19000D91F91E6F92E10C0F801848195810E9473
:10D1A000A967F0E4FE1538F4009729F0C80FD91FDD
:10D1B00081E4F82E01C06196DE1490F4D8015096F7
:10D1C0001C92509753961C92539754961C925497C6
:10D1D00051961C92519752961C9280E090E067C045
:10D1E000DF1460F38C2D90E0FE0124912F3F11F4A9
:10D1F000219658C0FE104DC0D80114968D919C9177
:10D2000015970E948D679E012F5F3F4FFE01882377
:10D2100011F08230E1F48491D80153968C935397A6
:10D22000F901249154962C935497FE013396E4917E
:10D230005096EC935097FE013496E4915196EC93FE
:10D240005197FE013596E4915296EC9320C084915B
:10D25000982F9F709250D80152969C935297829526
:10D260008F7051968C935197F9012491822F8F7072
:10D2700054968C93549722952F7053962C935397D2
:10D28000FE013296E491E295EF705096EC93CE0158
:10D290000EC0FE013296E491EB219C012E0F311D50
:10D2A000C20FD31FFD1409F489CFF3949DCFDF91F2
:10D2B000CF911F910F91FF90EF90DF90CF90BF9093
:10D2C00008950F93FC010150040F84A996A99417A7
:10D2D00018F0081728F402C0081750F0041740F49B
:10D2E0002150260F83A995A9961720F4281720F41A
:10D2F00080E007C0281720F481E0261710F0F8CF4F
:10D3000081E00F9108955F926F927F928F929F922A
:10D31000AF92BF92CF92DF92EF92FF920F931F9343
:10D32000CF93DF93EC01C62E142F622F0E948B68DF
:10D330007C01892B09F445C08C819D810E949067F6
:10D34000A82EDB88BC888989C80E8A898B0D181B9A
:10D350000B2D2D2D412F6C2DCE010E94616988234C
:10D3600071F1EA0CF11C87E08D0DD82ED694D6947D
:10D37000D6945B2C510E4E018CE1880E911C6D2CC5
:10D38000712C5116E1F00C2D57018A2D8E198D1537
:10D3900090F4F50184916A817B810C8F1D8F1F8E23
:10D3A0008E8F94014BE3CE010E942F68FFEFAF1ADE
:10D3B000BF0A085FEACFE60CF71C1F5FE2CF88893F
:10D3C00001C080E0DF91CF911F910F91FF90EF900E
:10D3D000DF90CF90BF90AF909F908F907F906F9095
:10D3E0005F9008958BE1E6E7FDE0ABE5BDE00190DD
:10D3F0000D928A95E1F78091330F80628093330F0D
:10D4000008958091330F8F7B8B7F8093330F0E9421
:10D410004828882321F08DE19DE00C947D730895C8
:10D420008091330F83FF03C084608093330F08958E
:10D430005F926F927F928F929F92AF92BF92CF92A4
:10D44000DF92EF92FF920F931F93CF93DF93CDB7AD
:10D45000DEB76DB67EB6DC010D900020E9F79D01C8
:10D46000281B390B2C5F3F4F4DB75EB7421B530B48
:10D470000FB6F8945EBF0FBE4DBF0DB71EB70F5F5E
:10D480001F4F9F938F9383EF9FE19F938F931F93E2
:10D490000F930E941CB3780154E0E50EF11C0F902D
:10D4A0000F900F900F900F900F90F70180818823BD
:10D4B00059F0082E000C990B0E948CBDF701819346
:10D4C0007F01F3CF0E94D92AC8010E9433358823F7
:10D4D000C9F38FEEE82E8FE1F82E00E010E009C0CE
:10D4E0005520B1F1EA0CFB1C0FB6F8949EBE0FBE9E
:10D4F0008DBE8DB69EB6F701E00FF11F5490A801C6
:10D500004F5F5F4F5A01552029F05AE0551611F030
:10D510008501F1CF8DB79EB78A199B090FB6F89494
:10D520009EBF0FBE8DBFEDB7FEB731966F01A8014C
:10D53000B701CF010E94BEB2F601E00FF11F1082C9
:10D54000C6010E9433358111CBCF0E94D92AF8CF72
:10D550000FB6F8947EBE0FBE6DBEDF91CF911F91C6
:10D560000F91FF90EF90DF90CF90BF90AF909F9082
:10D570008F907F906F905F9008958F929F92AF925F
:10D58000BF92CF92DF92EF92FF92CF938091330FB1
:10D59000877F8093330F8091790D882321F086E770
:10D5A0009DE00E947D7310925A0D1092570D85E3F5
:10D5B0008093560D0E94C0A56B017C0120EDC20E28
:10D5C00027E0D21EE11CF11CA89561E08091560D68
:10D5D0000E94214361E08091560D0E945043209AA1
:10D5E000289A219A2398229A81E00E94253185E089
:10D5F0008093580D0E942531CAE08FEF0E941931A7
:10D60000C150D9F7A89520E030E0A90160E086E597
:10D610009DE00E94CC538093590D813061F00E94AF
:10D62000C0A5DC01CB018C199D09AE09BF09B7FD6E
:10D63000EACF81E062C0A8952AEA31E040E050E0FC
:10D6400068E086E59DE00E94CC53853011F481E0CE
:10D650000AC0C4E00E941E318093590DC150D1F719
:10D660008A3A61F482E080935A0DA89580915A0D10
:10D67000823081F0812C912C540111C00E94C0A5F0
:10D68000DC01CB018C199D09AE09BF09B7FDD4CFD0
:10D6900082E033C0812C912CA12C80E4B82E20E0B4
:10D6A00030E0A90167E386E59DE00E94CC53A50127
:10D6B000940169E286E59DE00E94CC538093590D68
:10D6C000882361F00E94C0A5DC01CB018C199D0963
:10D6D000AE09BF09B7FDE3CF8AE00FC080915A0DB4
:10D6E000823021F520E030E0A9016AE386E59DE083
:10D6F0000E94CC53882361F088E08093570D86E523
:10D700009DE00E94C4530E94D22881EE9FE139C05F
:10D710000E941E31807C803C19F483E080935A0D76
:10D720000E941E310E941E310E941E3186E59DE03E
:10D730000E94C4531092580D81E00E942CA38111C5
:10D740000AC080E00E942CA3811105C00E94CE284F
:10D750008DEC9FE116C068E37DE086E79DE00E94C6
:10D76000DB72811105C00E94CE288CEB9FE109C0BD
:10D770008091330F88608093330F0E94D22880EB12
:10D780009FE10E94AC280E94F26983E080930E0220
:10D79000CF91FF90EF90DF90CF90BF90AF909F9090
:10D7A0008F900895FC0180818823E1F0853ED1F0BF
:10D7B0008E32C1F08091B8048E32A1F09385892F0A
:10D7C0008A7081F4987121E0903109F020E0809115
:10D7D000330F20FB84F98093330F903141F0808523
:10D7E000873411F080E0089581858E37D9F381E088
:10D7F00008950F931F93CF93DF93CDB7DEB7EB97C9
:10D800000FB6F894DEBF0FBECDBF8C018BE59DE057
:10D810000E94BF748BE1EBE5FDE0DE019196019083
:10D820000D928A95E1F748EB54E0BE016F5F7F4FA0
:10D83000CE0181960E945C721816A4F4CE01019666
:10D840000E94D26B882379F3BE016F5F7F4F8BEA12
:10D8500094E00E94A06E6BEA74E0C8010E94B1BD22
:10D86000892B09F7CE0181960E94B376EB960FB60D
:10D87000F894DEBF0FBECDBFDF91CF911F910F9106
:10D8800008950F931F93CF93DF931F921F92CDB7ED
:10D89000DEB72091330F23FF3BC08C01BC0182E037
:10D8A0000E94AE6710922A0F0E94016AA801BE0171
:10D8B0006F5F7F4F80E00E942EA28C01009741F1A4
:10D8C00069817A8126E5AC018DE19DE00E94B976FF
:10D8D0008823A9F08091330F81608093330FC801B2
:10D8E0000E94F96BB80186E990E20E94BB288AE0A9
:10D8F0000E94A52860E0C8010E94E63E09C0B80168
:10D9000080E395E20E94BB2882E59DE10E94AC285D
:10D910000F900F90DF91CF911F910F910895EF928B
:10D92000FF920F931F93CF93DF93CDB7DEB7279767
:10D930000FB6F894DEBF0FBECDBF2091330F23FF8B
:10D94000FEC0F62E8C0181E0681799F0681750F040
:10D9500082E0681394C00E94D22887E190E20E947E
:10D96000AC288DC0B80182E00E94AE6710922A0FE9
:10D9700086C00E944828811105C0B80181E00E943C
:10D98000AE677DC080912A0F882361F00E94CE2867
:10D9900081E590E20E94AC2860E080E090E00E9487
:10D9A000FAA0CDC081E39CE09E838D838FE28093BB
:10D9B000300CFF82CE0105969A83898302969C8360
:10D9C0008B83F12C8BE1E82E8091290FF81658F407
:10D9D000EF9CB0011124655E714FCE0101960E944B
:10D9E000CD67F394F1CF8F818B3558F46DE17DE0F5
:10D9F000CE0101960E94CD678D819E8101979E8305
:10DA00008D83ED81FE811082E0912A0F84E0E89FF2
:10DA1000F0011124E45DF34F80912F0F9091300FAE
:10DA2000A091310FB091320F80839183A283B38391
:10DA30000E94D228B80188E390E20E94BB2860913E
:10DA40002A0F89E6689FB0011124605D734F8DE253
:10DA500090E20E94BB2840912F0F5091300F6091AF
:10DA6000310F7091320F87E290E20E9497298AE08D
:10DA70000E94A52880912A0F8F5F80932A0F0E9411
:10DA8000016AA801BE016F5F7F4F81E00E942EA254
:10DA90008C01009709F453C069817A8121E0AC01BF
:10DAA0008DE19DE00E94B976882309F43FC0809102
:10DAB0002E0D90912F0DA091300DB091310D8093CE
:10DAC0002B0F90932C0FA0932D0FB0932E0F10922D
:10DAD0002F0F1092300F1092310F1092320FB801A9
:10DAE00089E090E20E94BB2840912B0F50912C0FAF
:10DAF00060912D0F70912E0F84E99FE10E9497296C
:10DB00008AE00E94A5288AEF9FE10E94AC28C80104
:10DB10000E94F96B8091B804811102C0C80102C053
:10DB200088EB94E060E00E94E63E09C0B80180E323
:10DB300095E20E94BB2882E59DE10E94AC282796D1
:10DB40000FB6F894DEBF0FBECDBFDF91CF911F910E
:10DB50000F91FF90EF9008956F927F928F929F9216
:10DB6000AF92BF92CF92DF92EF92FF920F931F93EB
:10DB7000CF93DF93CDB7DEB7C356D1090FB6F89474
:10DB8000DEBF0FBECDBF5C018B016DB67EB67E01E0
:10DB900087E5E80EF11C48EB54E0BE016F5F7F4F54
:10DBA000C5010E945C7218160CF0AFC08C8588719C
:10DBB000803109F06CC08DB69EB6BE016F5F7F4F9D
:10DBC000C7010E94A06E0115110521F0F8018081A6
:10DBD000811191C021E081E090E0F70101900020E7
:10DBE000E9F73197EE19FF09E80FF91F32968DB763
:10DBF0009EB78E1B9F0B0FB6F8949EBF0FBE8DBFB6
:10DC0000EDB7FEB731966F01211102C0B80102C015
:10DC10006CEF72E0C6010E94E3BDB701C6010E942D
:10DC2000C4BD6CEF72E0C6010E94C4BD19A21CA263
:10DC300021E0A701B501CE0181960E94B97681113C
:10DC40000AC00E94D228B7018CE99FE10E94BB283C
:10DC50008AE00E94A5288BE1FE01B196DE01DC96E8
:10DC600001900D928A95E1F7B601CE01CC960E9403
:10DC7000AC6DCE01CC960E94B376CE0181960E9407
:10DC8000B3760FB6F8949EBE0FBE8DBE84CFCE0184
:10DC900001960E94D26B882309F47DCFBE016F5F8D
:10DCA0007F4F8BEA94E00E94A06E0115110529F4C4
:10DCB0008BEAC82E84E0D82E09C06801F601819154
:10DCC0006F018823A9F30E94A528F8CFF60181915E
:10DCD0006F01882319F00E94A528F8CF80E20E94E6
:10DCE000A5286D8D7E8D8F8D98A14AE00E942A29EE
:10DCF0000E94B22A50CFF80101900020E9F7319735
:10DD0000CF01801B910B20E068CF0FB6F8947EBE48
:10DD10000FBE6DBECD59DF4F0FB6F894DEBF0FBEFC
:10DD2000CDBFDF91CF911F910F91FF90EF90DF90CA
:10DD3000CF90BF90AF909F908F907F906F900895FD
:10DD4000FC0120E03EE2DB014C91403241F0283002
:10DD500011F430833196DB014C91408331962F5F73
:10DD60006F5F7F4F2B3079F710820895CF938091AA
:10DD70003D128823B9F140913512509136126091CD
:10DD800037127091381225E330E180913E12909164
:10DD90003F120E941654C82F811102C0C0E023C058
:10DDA0004091391250913A1260913B1270913C129D
:10DDB000411551056105710591F025E330E1809130
:10DDC0003E1290913F120E941654882339F310920C
:10DDD000391210923A1210923B1210923C12109289
:10DDE0003D1201C0C1E08C2FCF910895CF92DF92F8
:10DDF000EF92FF92CF936B017C01C42F809135127B
:10DE000090913612A0913712B09138128C159D0561
:10DE1000AE05BF05D1F00E94B66E811102C080E050
:10DE200018C025E330E1B701A60180913E12909120
:10DE30003F120E947954882391F3C0923512D092F8
:10DE40003612E0923712F092381281E0C1118093BD
:10DE50003D12CF91FF90EF90DF90CF9008954F92B9
:10DE60005F926F927F928F929F92AF92BF92CF926A
:10DE7000DF92EF92FF920F931F93CF93DF93EC010A
:10DE8000423051056105710510F480E069C0898553
:10DE90009A85AB85BC850196A11DB11D8417950798
:10DEA000A607B70790F38F89803149F4852E962E07
:10DEB000A72EBB248B899C89AD89BE890FC0803277
:10DEC00021F78B889C88AD88BE88DB01CA01E7E01A
:10DED000B695A79597958795EA95D1F7880E991EDF
:10DEE000AA1EBB1E280139016A017B0141E0C50160
:10DEF000B4010E94F66E882341F29F89903161F44B
:10DF0000DD24EE24FF249601220F331FF901EB5C80
:10DF1000FF4E5182408211C0E894C7F8DD24EE2400
:10DF2000FF249601220F331F220F331FF901EB5CF0
:10DF3000FF4E40825182628273829A89923080F0D1
:10DF40004D815E816F817885840E951EA61EB71E59
:10DF50008092391290923A12A0923B12B0923C12E7
:10DF6000DF91CF911F910F91FF90EF90DF90CF90B5
:10DF7000BF90AF909F908F907F906F905F904F90E9
:10DF80000895CF92DF92EF92FF920F931F93CF935A
:10DF9000DF93FC0181859285A385B4850196A11D3F
:10DFA000B11D84179507A607B70710F480E061C07C
:10DFB0008789803149F4BB27A72F962F852FC388E7
:10DFC000D488E588F6880FC0803281F783899489E8
:10DFD000A589B6896A017B01C7E0F694E794D794D6
:10DFE000C794CA95D1F78C0D9D1DAE1DBF1DE901CB
:10DFF0006A017B018F014091351250913612609178
:10E0000037127091381284179507A607B70739F0B1
:10E0100040E0BC01CD010E94F66E882339F2F80180
:10E020008789803179F4B701A601552766277727BC
:10E03000440F551FFA01EB5CFF4E80819181A0E0F7
:10E04000B0E012C0B701A6014F77552766277727A2
:10E05000440F551F440F551FFA01EB5CFF4E8081A2
:10E060009181A281B381BF7088839983AA83BB8386
:10E0700081E0DF91CF911F910F91FF90EF90DF90A2
:10E08000CF9008954F925F926F927F92AF92BF921E
:10E09000CF92DF92EF92FF920F931F93CF93DF9374
:10E0A00000D01F92CDB7DEB78C0149835A836B83B2
:10E0B0007C835901C12CD12C7601412C82E0582E51
:10E0C000612C712C49815A816B817C819E012F5F6B
:10E0D0003F4FC8010E94C16F882341F1D301C201A3
:10E0E000F801058404C0880F991FAA1FBB1F0A945A
:10E0F000D2F7C80ED91EEA1EFB1E49815A816B81D8
:10E100007C818789803139F481E0483F5F4F610528
:10E11000710538F4D7CF81E0483F5F4F6F4F7F40A4
:10E1200088F2F501C082D182E282F3820F900F90D3
:10E130000F900F90DF91CF911F910F91FF90EF9073
:10E14000DF90CF90BF90AF907F906F905F904F9097
:10E1500008958F929F92AF92BF92CF92DF92EF92EB
:10E16000FF920F931F93CF93DF93EC018B8181116B
:10E1700002C080E078C009891A892B893C8904177C
:10E18000150726073707A8F36A017B01823029F4B7
:10E19000C886D986EA86FB860DC0C114D104E10485
:10E1A000F10451F4188619861A861B861C821D827A
:10E1B0001E821F8281E057C088849984AA84BB8410
:10E1C000E98DFA8D258530E0275F3F4FB501A40129
:10E1D0004150510961097109022E04C07695679575
:10E1E000579547950A94D2F7D701C6010197A1091F
:10E1F000B10904C0B695A795979587952A95D2F74A
:10E2000084179507A607B70720F089288A288B2846
:10E2100071F44D895E896F89788D4C835D836E833F
:10E220007F834C015D018E010C5F1F4F16C0841B64
:10E23000950BA60BB70BF5CF4C815D816E817F816D
:10E240009801898D9A8D0E94C16F91E0891A910879
:10E25000A108B108882309F48CCF81149104A1048A
:10E26000B10451F795CFDF91CF911F910F91FF909E
:10E27000EF90DF90CF90BF90AF909F908F900895D8
:10E280002F923F924F925F926F927F928F929F92C6
:10E29000AF92BF92CF92DF92EF92FF920F931F93B4
:10E2A000CF93DF9300D01F92CDB7DEB79C838B83D3
:10E2B0004B015A01DC0113968C91811103C08FEF41
:10E2C0009FEFE3C0EB81FC81818180FFF8CFEB8180
:10E2D000FC8181899289A389B489408551856285B1
:10E2E0007385841B950BA60BB70BA50160E070E04E
:10E2F00084179507A607B70708F45C0175018B81A1
:10E300009C8104969A838983612C42E0742EE114E7
:10E31000F10409F48BC0AB81BC8118964D915D91DD
:10E320006D917C911B976A01B1E0DB22EB81FC814E
:10E330002381818D928D1A012B0139E056944794E7
:10E34000379427943A95D1F7223061F4FC01828DFD
:10E35000938DA48DB58DBC01CD01620D731D841DFF
:10E36000951D4AC0DC0114961C9111501221C11454
:10E37000D10401F511111EC0452B462B472B59F432
:10E38000EB81FC8185899689A789B08D84839583EB
:10E39000A683B7830FC0AB81BC8114964D915D916C
:10E3A0006D917C91179729813A810E94C16F8823D2
:10E3B00009F485CFEB81FC81218D328D848195819B
:10E3C000A681B7810297A109B109F901058404C0AA
:10E3D000880F991FAA1FBB1F0A94D2F7468557853D
:10E3E00060897189840F951FA61FB71FBC01CD01DD
:10E3F000610F711D811D911D93012C193D0987012C
:10E400002E153F0508F489010115F2E01F0779F583
:10E4100020913512309136124091371250913812B6
:10E42000621773078407950719F421C0C5012DC031
:10E430009401AB01BC0180913E1290913F120E9469
:10E440007954882309F43BCF800E911EEB81FC8127
:10E4500080859185A285B385800F911FA11DB11D77
:10E4600080879187A287B387E01AF10A50CF40E0F6
:10E470000E94F66E882309F422CFB6016B5C7F4EB2
:10E48000A801C4010E94A1BDDFCF0F900F900F9093
:10E490000F90DF91CF911F910F91FF90EF90DF9040
:10E4A000CF90BF90AF909F908F907F906F905F9034
:10E4B0004F903F902F900895DF92EF92FF920F932D
:10E4C0001F93CF93DF93FC012381223060F00085FE
:10E4D0001185228533850F71112722273327012BC0
:10E4E000022B032B11F08FEF5EC04115510511F087
:10E4F000FA0110827A01EB018C018DE0D82E40E206
:10E5000050E0BE01C8010E9440718032910539F08F
:10E5100021E0892B09F420E0822F819544C02881D5
:10E520002223C9F1253E11F02E3231F4E114F10419
:10E5300031F3F7011082E3CFE114F10441F13B859F
:10E540003F733F3021F54A8D5B8D452B01F52F71CF
:10E550003FEF320F3230D8F430E021503109D29EF3
:10E56000C001D39E900D1124D701A80FB91FFE0141
:10E5700020E0AD01253088F431813D932F5F329644
:10E580002D30C1F7288126FF02C0FA0115862B85A0
:10E5900023FDB5CF08C080E006C02B3010F43481D5
:10E5A000ECCF3681EACFDF91CF911F910F91FF9091
:10E5B000EF90DF9008950F931F93CF93DF93FC01AB
:10E5C0002381222311F080E044C08B01EC01FB0188
:10E5D0008789803139F18032B1F783E08B83F8018C
:10E5E000428D538D648D758D4D8B5E8B6F8B788FC7
:10E5F0009E012F5E3F4FC8010E944270882319F38D
:10E600001A8F098F81E08983188619861A861B86DE
:10E610001C821D821E821F82188A1C861D861E86F1
:10E620001F8617C082E08B831D8A1E8A1F8A188E60
:10E63000FB01808D918DA0E0B0E025E0880F991F4F
:10E64000AA1FBB1F2A95D1F7898B9A8BAB8BBC8BEA
:10E65000D7CFDF91CF911F910F910895CF93DF9383
:10E66000EC0141E0611101C040E06C857D858E8543
:10E670009F850E94F66E882341F0888920E2829F60
:10E68000C00111248B5C9F4E02C080E090E0DF91BE
:10E69000CF910895CF93DF93EC018B81882339F1DB
:10E6A000898187FF20C061E0CE010E942E73FC01AA
:10E6B000892BE9F08081853ED1F08B81823040F456
:10E6C00089899A89AB89BC89848F958FA68FB78FEA
:10E6D0008D899E89AF89B88D938F828FB58BA48BDE
:10E6E00089818F778983DF91CF910C94B66E81E019
:10E6F000888380E0DF91CF910895CF93DF93EC0181
:10E700000E944A731B82DF91CF910895CF93DF93CC
:10E71000EB01FC012381211102C080E028C02250BE
:10E72000223020F48FE28883198220C060E00E94AA
:10E730002E73009791F3FC0190E080E02EE230818F
:10E74000303269F0883029F4DE01A90FB11D2C9315
:10E750009F5FDE01A90FB11D30813C939F5F8F5FEA
:10E7600031968B3061F7C90FD11D188281E0DF919E
:10E77000CF9108953F924F925F926F927F928F92C6
:10E780009F92AF92BF92CF92DF92EF92FF920F9340
:10E790001F93CF93DF93CDB7DEB72C970FB6F894C6
:10E7A000DEBF0FBECDBF5C01DC0159968D909C9001
:10E7B0005A97F40181859285A385B4859C01AD01AA
:10E7C0002F5F3F4F4F4F5F4F29873A874B875C87BB
:10E7D000D5011496CD90DD90ED90FC901797C11463
:10E7E000D104E104F10439F0BFEFCB1ADB0AEB0AE4
:10E7F000FB0A312C07C0F401C080D180E280F38095
:10E8000033243394260137011D821E821F8218860D
:10E81000F40181859285A385B4852D813E814F8148
:10E820005885281739074A075B0708F064C08985AF
:10E830009A85AB85BC858C159D05AE05BF0550F44A
:10E8400082E0C82ED12CE12CF12C92E0492E512CE3
:10E85000612C712C9E012F5F3F4FB701A601C401AF
:10E860000E94C16F882309F446C089819A81AB81D7
:10E87000BC81892B8A2B8B2B41F0260137019FEF1E
:10E88000491A590A690A790A05C0C414D504E6046C
:10E89000F70491F02D813E814F8158852F5F3F4FC6
:10E8A0004F4F5F4F2D833E834F8358873FEFC31AEF
:10E8B000D30AE30AF30AACCF0FEF1FEF2FEF3FE0CD
:10E8C000B301A201C4010E942F6FF82E882399F092
:10E8D000D50114964D915D916D917C9117974115DD
:10E8E00051056105710549F093018201C4010E943F
:10E8F0002F6F811102C0F12C29C0D50114964D92C1
:10E900005D926D927C921797332051F0D301C20132
:10E910000196A11DB11DF40180839183A283B3836D
:10E92000F50185899689A789B08D892B8A2B8B2B38
:10E9300069F4D50155964D925D926D927C925897EF
:10E9400011968C911197806811968C938F2D2C962F
:10E950000FB6F894DEBF0FBECDBFDF91CF911F91F0
:10E960000F91FF90EF90DF90CF90BF90AF909F906E
:10E970008F907F906F905F904F903F90089540E010
:10E9800050E0BA010C94A9704F925F926F927F92FF
:10E990009F92AF92BF92CF92DF92EF92FF920F932E
:10E9A0001F93CF93DF931F92CDB7DEB78C017B010E
:10E9B0005A01C22EDB0159968D919C915A97F8010C
:10E9C000928F818FCB010E94BF74912CF7018085BB
:10E9D0009185A285B3854189528963897489841799
:10E9E0009507A607B70708F060C025E0B695A7957C
:10E9F000979587952A95D1F7F82FFF70DF2ED701CD
:10EA000013968C91823008F460C041E050E0BE0162
:10EA10006F5F7F4FC7010E944071019719F4898190
:10EA200090E002C08FEF9FEF019609F44EC0F7010E
:10EA300080859185A285B3854F96A11DB11D8087E4
:10EA40009187A287B387F0E2DF9EB00111246B5C4F
:10EA50007F4E61157105C9F1DB018C91882319F096
:10EA6000853EC1F46CC191100EC080913512909119
:10EA70003612A0913712B0913812F8018487958729
:10EA8000A687B787D08ADB018C91882361F099240F
:10EA900093949CCF4BE050E0C5010E9494BD892B1C
:10EAA00009F094CF14C0992493948C2D82748234ED
:10EAB00061F4992009F48BC0F801D08861E0C801A5
:10EAC0000E942E73009709F00DC180E03BC1C7FC86
:10EAD000FCCFF0E2DF9EA00111249A012B5C3F4E97
:10EAE000D9011B968C91817121F08C2D827109F0D6
:10EAF0006AC08091351290913612A0913712B09170
:10EB00003812F80184879587A687B787D08ACA010B
:10EB10008B5C9F4E7C01DC0154964D915C91559726
:10EB200060E070E0DA0199278827858B968BA78BA8
:10EB3000B08FF701428D538D60E070E0482B592B68
:10EB40006A2B7B2BD80155964D935D936D937C93E7
:10EB50005897F9018385887161F4F701848D958D4B
:10EB6000A68DB78DF801818B928BA38BB48B81E03E
:10EB700010C0803141F598012F5E3F4FD801599662
:10EB80008D919C915A970E9442708823E1F084E015
:10EB9000F80183838C2D8F70D80111968C93119777
:10EBA000F801148215821682178218961D921D9202
:10EBB0001D921C921B97C4FEB5C0C8010E949CA167
:10EBC0008111B0C082CFD80113961C927ECFD7019D
:10EBD00013968C911397823009F477CF51968D91CB
:10EBE0009D910D90BC91A02D803E9F4FAF41B105EE
:10EBF00008F06BCFC7010E94BA73882309F465CF70
:10EC00000E94B66E882309F460CFD70159962D91E2
:10EC10003C915A9714968D919D910D90BC91A02D89
:10EC20000297A109B109F901058404C0880F991F51
:10EC3000AA1FBB1F0A94D2F7468457846088718844
:10EC4000480E591E6A1E7B1E81E080933D12409241
:10EC5000351250923612609237127092381280E05C
:10EC600092E0E5E3F0E1DF019C011D92215030408C
:10EC7000E1F7DD24D394D7015996ED91FC915A9791
:10EC80008481D81698F425E330E1B301A2014D0D3B
:10EC9000511D611D711D80913E1290913F120E9485
:10ECA0001654882309F411CFD394E5CF80E092E085
:10ECB000A0E0B0E0058404C0880F991FAA1FBB1F05
:10ECC0000A94D2F7F7014189528963897489840FC4
:10ECD000951FA61FB71F818B928BA38BB48B85E3E7
:10ECE00090E1D12C20E2DC011D922A95E9F72BE07E
:10ECF000F501DC0101900D922A95E1F721E238E25D
:10ED0000FC01318B208B40E058E057874687338BDE
:10ED1000228B318F208F578B468B0E94B66E8111CC
:10ED2000D8CED3CEC5FE09C0F80141895289638986
:10ED30007489C8010E94A97005C081E003C09110C8
:10ED4000A6CE93CE0F90DF91CF911F910F91FF90A0
:10ED5000EF90DF90CF90BF90AF909F907F906F909B
:10ED60005F904F900895FC01238121110C947D73D5
:10ED700008952F923F924F925F926F927F928F925F
:10ED80009F92AF92BF92CF92DF92EF92FF920F933A
:10ED90001F93CF93DF93CDB7DEB7C254D1090FB61F
:10EDA000F894DEBF0FBECDBF4C015B016A01322E6D
:10EDB00019821C821C8E1F8E6115710511F410E0E2
:10EDC000A6C0FC0183818111FACFFA0180818F32C4
:10EDD00009F09BC0F50183818250823010F48501D7
:10EDE0000CC0F501618D728DCE014C960E94DB72D4
:10EDF000882329F38E01045E1F4FC6016C01019622
:10EE0000F60120812F32D1F3CE0101967C013C0125
:10EE10002E019CE1490E511C2396EFAE23972F2C17
:10EE20009BE09150E7E3F0E0EC0FFD1FE90FF11DCF
:10EE300080E280839111F5CF960147E0D9018D9151
:10EE4000882369F18F3259F18E3239F44A3009F44E
:10EE5000B6CF98E04AE09D01F1CFE9EBF0E22491D2
:10EE6000222321F031968213FACFA9CF491708F453
:10EE7000A6CF813208F4A3CF8F3709F4A0CF21E0C9
:10EE8000290FE7E3F0E0EC0FFD1FE90FF11D9FE90B
:10EE9000980F9A3108F480528083922FDCCF8FA98B
:10EEA000803209F48CCF6901F90180812F5F3F4FD7
:10EEB0008F32C9F38823F9F021E0AE01495C5F4F3E
:10EEC000B801C7010E94C474882309F478CF0A15D9
:10EED0001B0519F0C8010E947D736E147F0441F078
:10EEE00023969FAD2397822D8701E92EF82E98CF88
:10EEF000942D852DF9CF232DAE01495C5F4FB801CC
:10EF0000C4010E94C474182F02C08B017DCFCE01B2
:10EF10004C960E94B376CE0101960E94B376812F63
:10EF2000CE5BDF4F0FB6F894DEBF0FBECDBFDF91D3
:10EF3000CF911F910F91FF90EF90DF90CF90BF90F6
:10EF4000AF909F908F907F906F905F904F903F9089
:10EF50002F9008950C94F980CF93DF93EC01CB01AF
:10EF6000BA010E948BB32AE037ED43E25DE30E94D1
:10EF700074BB20E030E0A9010E947ABA0E94EDBB88
:10EF8000688379838A839B83DF91CF910895CF93A0
:10EF9000DF93EC01CB01BA010E948BB320E030E09B
:10EFA00040E251E40E9474BB20E030E0A9010E94DD
:10EFB0007ABA688379838A839B83DF91CF9108959E
:10EFC000CF93DF93EC01CB01BA010E948BB32AE00F
:10EFD00037ED43E25DE30E9474BB20E030E0A9011D
:10EFE0000E947ABA688379838A839B83DF91CF9169
:10EFF0000895CF93DF93EC01CB01BA010E948BB34C
:10F0000020E030E0A9010E947ABA688379838A837C
:10F010009B83DF91CF910895CF93DF93EC01CB01D8
:10F02000BA010E948BB320E030E0A9010E947ABAB5
:10F03000688379838A839B83DF91CF910895CF93EF
:10F04000DF93EC01CB01BA010E948BB320E030E0EA
:10F050004AE754E40E9474BB20E030E0A9010E941A
:10F060007ABA688379838A839B83DF91CF910895ED
:10F07000CF93DF93EC01CB01BA010E948BB320E068
:10F0800030E0A9010E947ABA0E94E6BB79836883C6
:10F09000DF91CF910895CF93DF93EC01CB01BA01BB
:10F0A0000E948BB329EC38EC48EC5EE30E9474BB01
:10F0B00020E030E040E05FE30E947ABA0E94EDBBBE
:10F0C0006883DF91CF9108950E948BB32AE037EDDA
:10F0D00043E25DE30E9474BB20E030E0A9010E949E
:10F0E0007ABA0C94B0810E948BB32AE037ED43E2E8
:10F0F0005DE30E9474BB20E030E0A9010E947ABA6F
:10F100000C948E820E948BB320E030E0A9010E9413
:10F110007ABA0C948E820C9445940C9445940C9479
:10F1200045944F925F926F927F928F929F92AF928F
:10F13000BF92CF92DF92EF92FF920F931F93CF93E4
:10F14000DF930E94DB41D0918504C0E0D11121C042
:10F150008091870481110CC08091830410928304F4
:10F16000882331F00E94F98080919D048111F6C2BC
:10F1700080910E02882309F4D9C081E09091870420
:10F18000911180E004E024E046E451E26C2F0E94FB
:10F190000E33C090B809D090B909E090BA09F09048
:10F1A000BB098091BC099091BD09A091BE09B091A5
:10F1B000BF098C159D05AE05BF0510F4D701C6012A
:10F1C000C090B409D090B509E090B609F090B709A5
:10F1D000BC01CD016C157D058E059F0510F4C7019E
:10F1E000B6010E9489B36B017C01D13061F480913A
:10F1F0008704813009F07FC08091830410928304DA
:10F2000081111EC078C0D23061F4809187048230B1
:10F2100009F0FBC0809183041092830481119EC089
:10F22000F4C0D33009F08BC080918704833009F09B
:10F230006FC1809183041092830481110EC168C153
:10F240000E94F7A72AE037ED43E25DE3C701B6016C
:10F250000E94EAB320E030E0A9010E947ABA4B0193
:10F260005C0120E030E040E05FE40E9484B387FD71
:10F2700005C0812C912CA12C3FE4B32E2AE037ED60
:10F2800043E25DE36091E8097091E9098091EA0940
:10F290009091EB090E94EAB320E030E0A9010E94BE
:10F2A0007ABA20E030E040E85FE30E9479BA0E9439
:10F2B000EDBB2B013C01C501B4010E94E6BB7B0103
:10F2C0008C0121E0E21AF10801091109812C912C2D
:10F2D00025ECA22E2BE7B22E620121E030E040E0C7
:10F2E00050E068EE79E085E191E20E9487A6809186
:10F2F0009D04811133C280910E028823B9F011E080
:10F3000080918704813009F010E06091E8097091E4
:10F31000E9098091EA099091EB090E948E829C0193
:10F3200045E151E26C2F812F0E943BA6CF5FDF5F4A
:10F33000C53009F00BCF87E0809386040FC2D4302C
:10F3400009F07CC080918704843009F045C1809128
:10F35000830410928304811103C13EC10E94F7A768
:10F360006091C0097091C1098091C2099091C3094F
:10F370000E9489B320E030E0A9010E947ABA4B01D3
:10F380005C0120E030E040E05FE40E9484B387FD50
:10F3900005C0812C912CA12C9FE4B92E20E030E0F7
:10F3A000A9016091EC097091ED098091EE099091AD
:10F3B000EF090E947ABA20E030E048EC52E40E9463
:10F3C00079BA0E94EDBB2B013C01C501B4010E943A
:10F3D000E6BB7B018C0124E6E21AF1080109110960
:10F3E000812C912C8BECA82E8BE7B82E620124E6A1
:10F3F00030E040E050E06CEE79E08BE091E20E947A
:10F4000087A680919D048111A9C180910E02882355
:10F4100009F48CCF11E080918704823009F010E06C
:10F420006091EC097091ED098091EE099091EF09DE
:10F430000E948E829C014BE051E274CFD53009F0DE
:10F4400080C080918704853009F01DC180918304BC
:10F45000109283048111DBC016C10E94F7A72AE035
:10F4600037ED43E25DE3C701B6010E94EAB320E055
:10F4700030E0A9010E947ABA4B015C0120E030E043
:10F4800040E05FE40E9484B387FD05C0812C912C8D
:10F49000A12C1FE4B12E2AE037ED43E25DE3609139
:10F4A000F0097091F1098091F2099091F3090E949D
:10F4B000EAB320E030E0A9010E947ABA20E030E00F
:10F4C00040E85FE30E9479BA0E94EDBB2B013C014A
:10F4D000C501B4010E94E6BB7B018C0121E0E21A68
:10F4E000F10801091109812C912CB5ECAB2EBBE779
:10F4F000BB2E620121E030E040E050E060EF79E0B7
:10F5000082E091E20E9487A680919D04811126C12C
:10F5100080910E02882309F409CF11E080918704BD
:10F52000833009F010E06091F0097091F109809149
:10F53000F2099091F3090E948E829C0142E051E20F
:10F54000F1CED63009F0F2CE80918704863009F0F2
:10F55000EAC080918304109283048111AFC0E3C09C
:10F560000E94F7A76091B4097091B5098091B6091E
:10F570009091B7090E9489B32AE037ED43E25DE339
:10F580000E94EAB320E030E0A9010E947ABA20E0AC
:10F5900030E040E850E40E9479BA0E94EDBBEBE80D
:10F5A0008E2EE8E79E2EFFEBAF2EFBE7BF2E6B0102
:10F5B00014E7E12E1FE0F12E00E010E024E030E03F
:10F5C00040E050E064EB79E08BEF90E20E9487A688
:10F5D00080919D048111C2C080910E02882309F49C
:10F5E000A5CE11E080918704843009F010E060918D
:10F5F000B4097091B5098091B6099091B7090E943C
:10F6000089B30E94B0819C014BEF50E28BCE0E94E7
:10F61000F7A76091B8097091B9098091BA099091E2
:10F62000BB090E9489B32AE037ED43E25DE30E9403
:10F63000EAB320E030E0A9010E947ABA20E030E08D
:10F6400040E850E40E9479BA0E94EDBB3FE8832E67
:10F6500038E7932E4FEBA42E4BE7B42E6B0114E743
:10F66000E12E1FE0F12E00E010E024E030E040E069
:10F6700050E068EB79E084EF90E20E9487A68091E9
:10F680009D0481116BC080910E02882309F44ECE37
:10F6900011E080918704853009F010E06091B8098D
:10F6A0007091B9098091BA099091BB090E9489B300
:10F6B0000E94B0819C0144EF50E234CE0E94F7A733
:10F6C0006091BC097091BD098091BE099091BF09FC
:10F6D0000E9489B32AE037ED43E25DE30E94EAB37A
:10F6E00020E030E0A9010E947ABA0E94EDBB8DE8CB
:10F6F000882E88E7982E9FEBA92E9BE7B92E6B01E9
:10F7000018E7E12E1FE0F12E00E010E020E030E0ED
:10F71000A9016CEB79E08DEE90E20E9487A68091C2
:10F720009D0481111BC080910E02882309F4FECD37
:10F7300011E080918704863009F010E06091BC09E7
:10F740007091BD098091BE099091BF090E9489B353
:10F750000E94B0819C014DEE50E2E4CDDF91CF914B
:10F760001F910F91FF90EF90DF90CF90BF90AF90DF
:10F770009F908F907F906F905F904F9008956CEA6C
:10F7800077E784E698E70C94108160EE77E783E7EB
:10F7900098E70C9410816CE078E782E898E70C9485
:10F7A000108167EC77E787E49DE70C9410816FE1A7
:10F7B00078E786E59DE70C94108169EF77E78FEE97
:10F7C0009BE70C94108168E378E786E99DE70C9449
:10F7D00010816BE478E782EA9DE70C9410810E9427
:10F7E0008BB320E030E0A9010E947ABA0C94C18268
:10F7F0000F931F93CF93DF930E94DB41D091850439
:10F80000C0E0D1110BC08091870481112AC0809182
:10F8100083041092830481111EC023C0D13061F48F
:10F8200080918704813009F03DC08091830410925B
:10F830008304811127C036C0D23009F057C08091AF
:10F840008704823009F07EC0809183041092830483
:10F85000811168C077C00E94F98080919D04811158
:10F8600011C180910E028823C1F181E0909187043B
:10F87000911180E004E024E046E451E26C2F0E9404
:10F880000E332BC00E94F7A720E030E040E85FE392
:10F8900068ED79E086EE90E20E943CA780919D049D
:10F8A0008111F0C080910E028823B9F011E080919F
:10F8B0008704813009F010E06091D8097091D9096E
:10F8C0008091DA099091DB090E94C1829C0146EE89
:10F8D00050E26C2F812F0E943BA6CF5FDF5FC530C7
:10F8E00009F08FCF86E080938604CCC0D33061F4DA
:10F8F00080918704833009F05CC08091830410926A
:10F900008304811146C055C0D430A1F5809187048D
:10F91000843009F076C080918304109283048111B1
:10F9200061C06FC00E94F7A720E030E040E85FE3CD
:10F930006CED79E08FED90E20E943CA780919D04F0
:10F940008111A0C080910E02882339F211E08091CC
:10F950008704823009F010E06091DC097091DD09C4
:10F960008091DE099091DF090E94C1829C014FEDD8
:10F9700050E2AFCFD53009F0B0CF80918704853009
:10F9800009F067C08091830410928304811152C0F2
:10F9900060C00E94F7A720E030E040E85FE360EE3F
:10F9A00079E088ED90E20E943CA780919D0481114E
:10F9B00069C080910E02882309F48FCF11E08091F5
:10F9C0008704833009F010E06091E0097091E1094B
:10F9D0008091E2099091E3090E94C1829C0148ED67
:10F9E00050E277CF0E94F7A720E030E0A90164EF52
:10F9F00079E083ED90E20E943CA780919D04811103
:10FA000041C080910E02882309F467CF11E08091F4
:10FA10008704843009F010E06091F4097091F509D1
:10FA20008091F6099091F7090E94C1829C0143EDF3
:10FA300050E24FCF0E94F7A720E030E0A90168EF25
:10FA400079E089EC90E20E943CA780919D048111AD
:10FA500019C080910E02882309F43FCF11E08091F4
:10FA60008704853009F010E06091F8097091F90978
:10FA70008091FA099091FB090E94C1829C0149EC96
:10FA800050E227CFDF91CF911F910F9108950E94EF
:10FA90008BB320E030E040E251E40E9474BB20E0F0
:10FAA00030E0A9010E947ABA0C94C981CF92DF920A
:10FAB000EF92FF92CF93DF9300D01F92CDB7DEB7C6
:10FAC0000E948BB320E030E04AE754E40E9474BB0C
:10FAD00020E030E0A9010E947ABA6B017C0120E0AD
:10FAE00030E0A9010E9484B387FD05C027E137EB10
:10FAF00041E558E304C027E137EB41E558EBC70186
:10FB0000B6010E947ABA69837A838B839C83CE0183
:10FB100001960E9446410F900F900F900F90DF9139
:10FB2000CF91FF90EF90DF90CF9008950E948BB31C
:10FB300020E030E0A9010E947ABA0E94E6BBCB0126
:10FB40000C94B4380E948BB329EC38EC48EC5EE39B
:10FB50000E9474BB20E030E040E05FE30E947ABA8C
:10FB60000E94EDBB862F0C94B73D63E972E084E6FA
:10FB700090E00E94453E6AEB72E084E690E00C94CF
:10FB8000453E81110C94B57D68EB71E084E190E015
:10FB90000C94453E0E946B9E0C94C17D0E94B15C0A
:10FBA0000C94C17D0F931F93522F2091D60D30914D
:10FBB000D70D2817390721F19093D70D8093D60DD3
:10FBC0008B0120E030E000938D0410938E0420938D
:10FBD0008F043093900440938504509386048A5E8A
:10FBE000984321F41092D80C1092990C82E08093E3
:10FBF0000E0281E080939D041092CD0C109284043B
:10FC00001F910F910895CF93DF9380910E02882367
:10FC100041F0609151047091520441E081E00E94F2
:10FC2000DA4080919A0C81111CC0C091D60DD09100
:10FC3000D70D20E040E060E070E083E09EE70E94A6
:10FC4000D27D81E080939A0C0E948C9410929A0C41
:10FC500020E040E060E070E0CE01DF91CF910C94B5
:10FC6000D27DDF91CF9108958091940D9091950D63
:10FC7000891B8F7051F48091D304813031F08091D1
:10FC8000330F82FB882780F9089581E00895FC01F5
:10FC900084910895FC0180810895BF92CF92DF92F4
:10FCA000EF92FF920F931F93CF93DF936B01890124
:10FCB0004A3009F49DC0453109F06EC0DB0112964F
:10FCC000ED91FC911397F280C681D781809102015A
:10FCD000809582708093000188E28A950000E9F7A0
:10FCE00020E1B22EBF0C38E2E32E88EF0E94EA3109
:10FCF0008E2D8A950000E9F7BFE1BF1508F45EC0BC
:10FD00008F2D807780680E94EA318F2D8295807FC9
:10FD10000E94EA318E2D8A950000E9F780E80E9462
:10FD2000EA3180E00E94EA318E2D8A950000E9F7E1
:10FD30008AEF0E94EA318E2D8A950000E9F78E0144
:10FD4000005F1F4F8881807F0E94EA3189918295F0
:10FD5000807F0E94EA31C017D107A1F78E2D8A95C6
:10FD60000000E9F7F394BF10C0CF809102018270C8
:10FD700080930001F601C281D381CE010E945067B9
:10FD80008111D3C1DF91CF911F910F91FF90EF901F
:10FD9000DF90CF90BF900895DB011296CD91DC915A
:10FDA0001397842F90E0FC017497E433F105F0F48D
:10FDB0008827EC57FF4F8F4F0C9469BA10EE1F0D38
:10FDC0001068812F807F0E94EA31812F8295807F89
:10FDD0000E94EA318E2D8A950000E9F780E80E94A2
:10FDE000EA3180E89FCF8981F901808381E0CACF21
:10FDF00080910101826080930101809102018270F3
:10FE000080930001809101018160809301018091C4
:10FE10000201817080930001099A119A8091020178
:10FE2000809582708093000188E28A950000E9F74E
:10FE300088E790E02EE93FE0CEE9DFE0F901319775
:10FE4000F1F70197C9F788EF0E94EA3118E2812F94
:10FE50008A950000E9F780E20E94EA3180E00E9482
:10FE6000EA31812F8A950000E9F780E00E94EA31AB
:10FE700080E80E94EA31812F8A950000E9F780E04E
:10FE80000E94EA3180E10E94EA31812F8A950000C8
:10FE9000E9F7CE010197F1F7CE010197F1F7CE0115
:10FEA0000197F1F7CE010197F1F7CE010197F1F734
:10FEB000CE010197F1F7CE010197F1F7CE0101973D
:10FEC000F1F7CE010197F1F7CE010197F1F7CE01DD
:10FED0000197F1F7CE010197F1F7CE010197F1F704
:10FEE000CE010197F1F72197F1F780E20E94EA3104
:10FEF00080E40E94EA31812F8A950000E9F780E2D0
:10FF00000E94EA3180E60E94EA311A950000E9F782
:10FF1000D0E0C8E218E28D2F807780680E94EA3135
:10FF20008D2F8295807F0E94EA318C2F8A95000068
:10FF3000E9F780E80E94EA3180E00E94EA318C2FE4
:10FF40008A950000E9F78AEF0E94EA318C2F8A95A2
:10FF50000000E9F790E2119880910201817080938E
:10FF60000001119A00001198809102018170809324
:10FF70000001119A00001198809102018170809314
:10FF80000001119A00001198809102018170809304
:10FF90000001119A000011988091020181708093F4
:10FFA0000001119A000011988091020181708093E4
:10FFB0000001119A000011988091020181708093D4
:10FFC0000001119A000011988091020181708093C4
:10FFD0000001119A000011988091020181708093B4
:10FFE0000001119A000011988091020181708093A4
:10FFF0000001119A00001198809102018170809394
:020000021000EC
:100000000001119A00001198809102018170809383
:100010000001119A00001198809102018170809373
:100020000001119A00001198809102018170809363
:100030000001119A00001198809102018170809353
:100040000001119A00001198809102018170809343
:100050000001119A00008C2F8A950000E9F7915059
:1000600009F079CF88EF0E94EA31812F8A9500004C
:10007000E9F7DF5FD03209F04ECF80E00E94EA312D
:1000800080EC0E94EA3188E28A950000E9F78091CD
:10009000020182708093000181E074CE4D8150E0B6
:1000A000440F551F60E070E08E819F810E94AABDC1
:1000B000CE010E94666781E065CEF901818193815E
:1000C000913009F46EC0933009F040C048EF480FFA
:1000D00091E02B81241708F490E021E03A81831706
:1000E00008F420E031E0841708F030E0492F432B7A
:1000F000242319F4932309F479CED8011296FC90A5
:10010000EE24EA94D12C44C0B901CE010E946D675F
:1001100081E038CEF90110828A8181838D818150FE
:1001200082838B81838381E02DCE4D8150E0440F0B
:10013000551F60E070E08E819F810E94AABD81E022
:1001400021CE8D81D9018C9381E01CCE2B81281783
:1001500008F44CCE2A81821708F448CEF280913000
:10016000C9F1D8F19230B9F4E12CDD24DA9410C051
:10017000B801CE010E946D67F8018181D8019C9180
:100180009D0D9C938E0D11968C93FF0C09F42ECE31
:10019000F7FEF4CFEDCF933009F4B2CFE12CD12CA0
:1001A000F7CF48E0480F91E02B81281708F490E042
:1001B00021E03A81431708F420E031E0481708F0C5
:1001C00030E0492F432B242319F4932309F40ECE56
:1001D000F801F280EE24E39495CFE12CDD24D39452
:1001E000D7CF20E040E060E070E08AEE98E30C9426
:1001F000D27DE091990CEE2389F0E150E093990CC7
:1002000088E0E89FF0011124E556F34F6281738185
:1002100027814681808191810C94D27D0C94F1805C
:100220000F931F93CF93DF93FC01EB0180918D041B
:1002300090918E04A0918F04B0919004B7FF08C0F4
:1002400010928D0410928E0410928F0410929004DC
:100250008091910490919204A0919304B0919404A0
:1002600040918D0450918E0460918F0470919004A0
:1002700084179507A607B70744F480938D049093DD
:100280008E04A0938F04B093900480910E02882373
:1002900001F140918D0450918E0460918F04709112
:1002A00090048091950490919604A0919704B09148
:1002B00098048A019B01080F191F2A1F3B1FC901BF
:1002C000B8011995BC0180919B0490919C040E94F7
:1002D000013480918304811108C080918A048823AD
:1002E000D1F180910E028823B1F18091990490910F
:1002F0009A040097B1F000918D0410918E04209122
:100300008F0430919004409195045091960460912F
:10031000970470919804400F511F621F731FFE01D4
:100320001995E0918B04F0918C04309741F0809105
:100330008A04811103C080918304811119958091F1
:10034000830410928304882331F0DF91CF911F91B1
:100350000F910C94F980DF91CF911F910F91089527
:10036000CF93DF9300D01F92CDB7DEB70E94EDBBD5
:100370000E9489B369837A838B839C83CE01019623
:100380000E942E380F900F900F900F90DF91CF9119
:1003900008958F929F92AF92BF92CF92DF92EF9289
:1003A000FF92CF936B017C0120E030E0A9010E9415
:1003B00084B387FD05C067E177EB81E598E304C06E
:1003C00067E177EB81E598EBA70196010E947ABA85
:1003D0006B017C0120E030E0A9010E9484B387FF1B
:1003E00008C0C701B601905820E030E048EC52E464
:1003F00006C020E030E048EC52E4C701B6010E949C
:10040000EAB320E030E040EA50E40E947ABA20E00B
:1004100030E040E251E40E9474BB0E94E6BB6B01F5
:100420007C0180E280939E0480E1C81687E2D806B2
:10043000E104F10494F0C701B60120E137E240E0A5
:1004400050E00E944ABACA01B9012AE030E040E017
:1004500050E00E944ABA605D01C060E260939F0470
:1004600088EEC81683E0D806E104F10494F0C701D1
:10047000B60128EE33E040E050E00E944ABACA01DB
:10048000B9012AE030E040E050E00E944ABA605DE5
:1004900001C060E26093A00484E6C816D104E104C0
:1004A000F10494F0C701B60124E630E040E050E0EA
:1004B0000E944ABACA01B9012AE030E040E050E0A7
:1004C0000E944ABA605D01C060E26093A1048AE0C4
:1004D000882E912CA12CB12CC701B601A501940145
:1004E0000E944ABAC62FCA01B901A50194010E940F
:1004F0004ABA605D6093A2048EE28093A304C05D5B
:10050000C093A4048EE994E0CF91FF90EF90DF9028
:10051000CF90BF90AF909F908F900895CF92DF9231
:10052000EF92FF92CF93DF9300D01F92CDB7DEB74B
:100530006B017C0120E030E0A9010E9484B387FDBB
:1005400005C067E177EB81E598E304C067E177EBED
:1005500081E598EBA70196010E947ABA69837A83B4
:100560008B839C83CE0101960E942E380F900F90B2
:100570000F900F90DF91CF91FF90EF90DF90CF9091
:100580000895CF92DF92EF92FF926B017C0120E001
:1005900030E0A9010E9484B387FD05C067E177EBD5
:1005A00081E598E304C067E177EB81E598EBA7016B
:1005B00096010E947ABA6B017C0120E030E0A9012B
:1005C0000E9484B387FD05C020E030E040E05FE397
:1005D00004C020E030E040E05FEBC701B6010E94BC
:1005E0007ABA0E94E6BBCB01FF90EF90DF90CF90EC
:1005F0000C94B438AF92BF92CF92DF92EF92FF92F9
:100600000F931F93CF93DF93EC015B018A01FB01F2
:10061000199587FD05C090E0A0E0B0E0219628C1C3
:10062000982F907E903CC9F48F7190E0A0E0B0E0EC
:100630006C017D0126E0CC0CDD1CEE1CFF1C2A9514
:10064000D1F7CE010196F50119958F73A701960197
:10065000282BDA01C90122960BC1982F907F903E7A
:1006600029F58F70C82ED12CE12CF12C86E0CC0C12
:10067000DD1CEE1CFF1C8A95D1F7CE010196F50119
:1006800019958F73C82A96E0CC0CDD1CEE1CFF1C5C
:100690009A95D1F7CE010296F50119958F73A701AE
:1006A0009601282BDA01C9012396E2C0982F987F82
:1006B000903F91F58770C82ED12CE12CF12CF6E0FB
:1006C000CC0CDD1CEE1CFF1CFA95D1F7CE01019677
:1006D000F50119958F73C82AA6E0CC0CDD1CEE1C21
:1006E000FF1CAA95D1F7CE010296F50119958F73DB
:1006F000C82AB6E0CC0CDD1CEE1CFF1CBA95D1F765
:10070000CE010396F50119958F73A7019601282B49
:10071000DA01C9012496ACC0982F9C7F983F09F05C
:100720003FC08370C82ED12CE12CF12C56E0CC0CAC
:10073000DD1CEE1CFF1C5A95D1F7CE010196F50188
:1007400019958F73C82A66E0CC0CDD1CEE1CFF1CCB
:100750006A95D1F7CE010296F50119958F73C82AD3
:1007600076E0CC0CDD1CEE1CFF1C7A95D1F7CE0197
:100770000396F50119958F73C82AE6E0CC0CDD1CB1
:10078000EE1CFF1CEA95D1F7CE010496F5011995F0
:100790008F73A7019601282BDA01C901259668C03D
:1007A000982F9E7F9C3F09F04CC08170C82ED12CA1
:1007B000E12CF12C86E0CC0CDD1CEE1CFF1C8A9594
:1007C000D1F7CE010196F50119958F73C82A96E0ED
:1007D000CC0CDD1CEE1CFF1C9A95D1F7CE010296C5
:1007E000F50119958F73C82A26E0CC0CDD1CEE1C90
:1007F000FF1C2A95D1F7CE010396F50119958F7349
:10080000C82A36E0CC0CDD1CEE1CFF1C3A95D1F753
:10081000CE010496F50119958F73C82A46E0CC0CD9
:10082000DD1CEE1CFF1C4A95D1F7CE010596F501A3
:1008300019958F73A7019601282BDA01C901269615
:1008400017C0982F907C903841F4807C803869F4F0
:100850002196CE01F5011995F8CF8E7F8D3F28F0B6
:100860002196CE01F5011995F8CF80E090E0DC01EA
:100870000115110529F0F80180839183A283B383C8
:10088000CE01DF91CF911F910F91FF90EF90DF90FC
:10089000CF90BF90AF900895EF92FF920F931F9368
:1008A000CF93DF9300D01F92CDB7DEB7062F142F62
:1008B0007C01112309F44AC0AE014F5F5F4F67E42A
:1008C0007EE7C7010E94FA827C0169817A818B816F
:1008D0009C816115710581059105C1F16D3371052B
:1008E00081059105A1F06E3771058105910579F0BB
:1008F00011506A3271058105910519F00E94A332E9
:10090000D8CF65E470E080E090E00E94A332602FD1
:1009100070E089819A81AB81BC81CD97A105B10539
:1009200019F081E390E002C080E390E0680F791F46
:10093000072E000C880B990B0E94A332115031F046
:10094000612F70E0C7010E944933181B812F0F905F
:100950000F900F900F90DF91CF911F910F91FF900B
:10096000EF9008951F93CF93DF9300D01F92CDB7E0
:10097000DEB710E0AE014F5F5F4F67E47EE70E9495
:10098000FA8249815A816B817C81452B462B472B0A
:1009900011F01F5FEFCF812F0F900F900F900F90EE
:1009A000DF91CF911F9108951F93CF93DF9300D0D4
:1009B0001F92CDB7DEB710E0AE014F5F5F4F6AE424
:1009C0007EE70E94FA8249815A816B817C81452BA6
:1009D000462B472B11F01F5FEFCF812F0F900F9009
:1009E0000F900F90DF91CF911F9108950F931F9358
:1009F000CF93DF930E94DB41D0918504C0E0D111F9
:100A00000BC080918704811161C080918304109292
:100A10008304811155C05AC0D13021F580918704DB
:100A2000813071F48091830410928304882341F013
:100A30008CE997E80E94F2AD80919D04811100C17C
:100A400080910E02882309F486C081E0909187048A
:100A5000913009F080E003E02EE346E451E26C2F90
:100A60000E940E330E94347E182FD23061F48091A0
:100A70008704823009F044C080918304109283047B
:100A8000811136C03DC0D33061F48091870483303A
:100A900009F096C08091830410928304811188C06C
:100AA0008FC0D43009F05AC080918704843009F097
:100AB0003CC08091830410928304811130C035C002
:100AC0000E94F98080919D048111BAC080910E022C
:100AD000882309F440C081E090918704911180E05F
:100AE00004E024E040EA52E26C2F0E940E3333C04F
:100AF0008BEB96E80E94F2AD80919D048111A0C01D
:100B000080910E02882319F181E090918704923040
:100B100009F080E003E02EE348EE51E215C00E94A8
:100B2000CE7D80919D0481118BC080910E0288231F
:100B300009F457C081E090918704943009F080E077
:100B400000E22EE348EC51E26C2F0E940E33112399
:100B5000F9F085E01EC00E94347E182F1111F9CFE4
:100B6000D53009F049C0809187048530D1F080915B
:100B70000E02882369F081E090918704953009F096
:100B800080E000E22EE34AEB51E26C2F0E940E332C
:100B900087E0CF5FDF5FC53009F031CF80938604F7
:100BA0004FC0809183041092830481111DC0DFCF58
:100BB0008EEB96E80E94F2AD80919D04811140C0B9
:100BC00080910E02882369F081E090918704933030
:100BD00009F080E003E02EE347ED51E26C2F0E9424
:100BE0000E33112349F0B5CF0E94CA7D80919D0438
:100BF000882309F4BCCF24C0D63051F680918704F5
:100C0000863071F48091830410928304882341F02C
:100C10000E94C49D0E94B57D80919D04811110C0E9
:100C200080910E02882309F4B3CF81E0909187046C
:100C3000963009F080E000E22EE349EA51E2A5CFC8
:100C4000DF91CF911F910F910895EF92FF920F9333
:100C50001F93CF93DF93E82E0E94DB41D091850450
:100C6000C0E08E2D90E09C012553334F7901D111C6
:100C70000BC080918704811151C080918304109230
:100C80008304811145C04AC0D13059F48091870452
:100C9000813001F5809183041092830481110FC08B
:100CA00019C0D23061F580918704823009F04AC0C2
:100CB000809183041092830481113EC043C040E0C0
:100CC00050E0B70186E992E20E94F7A680919D0468
:100CD00081114AC080910E02882389F011E0809131
:100CE0008704813009F010E0F70180810E94B73D50
:100CF0009C0146E952E26C2F812F0E943BA6CF5FF8
:100D0000DF5FC53009F0B3CF83E0809386042CC049
:100D10000E94F98080919D04811126C080910E026D
:100D2000882369F381E090918704911180E004E0C9
:100D300024E049EF51E214C00E94CE7D80919D04D1
:100D4000811112C080910E028823C9F281E0909136
:100D50008704923009F080E000E22EE348EC51E293
:100D60006C2F0E940E33CBCFDF91CF911F910F914B
:100D7000FF90EF90089580E00C94258681E00C941C
:100D800025860F931F93CF93DF930E94DB41D09171
:100D90008504C0E0D1110BC08091870481112AC065
:100DA000809183041092830481111EC023C0D1302E
:100DB00061F480918704813009F03BC08091830405
:100DC00010928304811127C034C0D23009F055C07D
:100DD00080918704823009F06BC080918304109267
:100DE0008304811157C064C00E94F98080919D04E2
:100DF00081119DC080910E028823B1F181E0909114
:100E00008704911180E004E024E046E451E26C2F75
:100E10000E940E3329C00E94F7A747EF58E868ECFC
:100E200079E08CE391E20E94ADA780919D0481114D
:100E30007EC080910E028823B9F011E08091870472
:100E4000813009F010E06091C8097091C909809162
:100E5000CA099091CB090E94C9819C014CE351E2DF
:100E60006C2F812F0E943BA6CF5FDF5FC53009F05A
:100E700091CF84E0809386045AC0D330A9F7809143
:100E800087048330D9F58091830410928304811103
:100E900027C034C00E94F7A74BEF58E86CEC79E00C
:100EA00082E391E20E94ADA780919D0481113FC031
:100EB00080910E028823C1F211E080918704823074
:100EC00009F010E06091CC097091CD098091CE09B4
:100ED0009091CF090E94C9819C0142E351E2C0CFA9
:100EE0000E94F7A749EF58E860ED79E088E291E2C7
:100EF0000E94ADA780919D04811119C080910E02BE
:100F0000882309F4B1CF11E080918704833009F080
:100F100010E06091D0097091D1098091D20990912F
:100F2000D3090E94C9819C0148E251E299CFDF9127
:100F3000CF911F910F910895EF92FF920F931F93FE
:100F4000CF93DF930E94DB41D0918504C0E08DE513
:100F5000E82E81E2F82ED1110BC080918704811117
:100F600029C0809183041092830481111DC022C086
:100F7000D13059F4809187048130A1F580918304A8
:100F800010928304811124C02DC0D23009F081C099
:100F900080918704823009F0A0C080918304109270
:100FA0008304811192C099C00E94F98080919D04B0
:100FB0008111EEC080910E02882329F181E0909189
:100FC0008704911180E004E024E049EF51E218C069
:100FD000F092A50AE092A40A0E94F18080919D04FB
:100FE0008111D6C080910E02882369F081E0909132
:100FF0008704913009F080E000E22EE348E951E2F5
:101000006C2F0E940E330E94347E81110EC0D530A9
:1010100071F480918704853009F0A7C08091830422
:1010200010928304811199C0A0C015E001C016E0A0
:101030001D1326C090918704911314C080918304DE
:1010400010928304882371F020E040E060E070E0BB
:101050008FEC98E8DF91CF911F910F91FF90EF9067
:101060000C94D27D80910E02882351F081E09D1373
:1010700080E003E02EE342E651E26C2F0E940E3343
:10108000CF5FDF5FC53009F066CF1F5F1093860426
:101090007FC0D33059F4809187048330B1F58091BB
:1010A000830410928304811128C02FC0D43009F02A
:1010B000AACF80918704843009F03FC080918304D7
:1010C00010928304811131C038C088EF9BE70E94E1
:1010D000F2AD80919D0481115BC080910E02882346
:1010E00009F491CF81E090918704923009F080E07B
:1010F00003E02EE34FE851E283CF81E998E70E94B5
:10110000F2AD80919D04811143C080910E0288232D
:1011100009F479CF81E090918704933009F080E061
:1011200003E02EE342E851E26BCF8DEF98E80E9496
:10113000F2AD80919D0481112BC080910E02882315
:1011400009F461CF81E090918704943009F080E048
:1011500003E02EE34DE751E253CF81EC96E80E9485
:10116000F2AD80919D04811113C080910E028823FD
:1011700069F081E090918704953009F080E003E008
:101180002EE344E751E26C2F0E940E3316E078CF35
:10119000DF91CF911F910F91FF90EF900895EF9203
:1011A000FF920F931F9387E0E82E82E2F82E00E073
:1011B00010E022E631E248EE58E869E072E288E5A4
:1011C00091E20E9431421F910F91FF90EF9008959C
:1011D000CF930E94C49D0E94B15CC82F882319F050
:1011E00080E00E94759C8C2FCF910C94C17D0C9453
:1011F00030980C9430980C9430986F927F928F9224
:101200009F92AF92BF92CF92DF92EF92FF920F9395
:101210001F93CF93DF9300D01F92CDB7DEB70E940C
:10122000DB4160908504712C862D870D59F48091E7
:10123000870481111BC08091830410928304811163
:101240000FC014C0813011F580918704813009F0FE
:101250005BC0809183041092830481111FC054C02D
:101260000E94F98080919D04811187C080910E02B7
:10127000882361F081E090918704911180E004E07F
:1012800024E046E451E2672D0E940E33739485E01A
:101290007812CACF82E0809386046FC020E030E0ED
:1012A0004AE754E46091D4047091D5048091D60447
:1012B0009091D7040E94EAB320E030E0A9010E9497
:1012C0007ABA20E030E040E85FE30E9479BA0E94F9
:1012D000EDBB812C912C87EDA82E8BE7B82E6B01EE
:1012E00013EFE12EFF24F39400E010E021E030E062
:1012F00040E050E064ED74E08BE191E20E9487A64B
:1013000080919D04811139C080910E02882309F4D7
:10131000BDCF11E080918704813009F010E0C090CA
:10132000D404D090D504E090D604F090D70420E007
:1013300030E0A901C701B6010E9484B387FD05C052
:1013400027E137EB41E558E304C027E137EB41E5FE
:1013500058EBC701B6010E947ABA69837A838B83FE
:101360009C83CE0101960E9446419C014BE151E2D3
:10137000672D812F0E943BA689CF0F900F900F9071
:101380000F90DF91CF911F910F91FF90EF90DF9021
:10139000CF90BF90AF909F908F907F906F90089567
:1013A0008091290F8823C9F081508093290F8823C9
:1013B00059F090E001972BE1289FF001299FF00D53
:1013C0001124E55EF14F02C0E6E7FDE08BE1ABE5FD
:1013D000BDE001900D928A95E1F78091290F81116E
:1013E00009C08091330F80628093330F80E090E0DA
:1013F000DC0104C081E090E0A0E0B0E080938D04C7
:1014000090938E04A0938F04B0939004109285045F
:1014100081E080939D0483E080930E020895EF9213
:10142000FF920F931F9387E0E82E82E2F82E00E0F0
:1014300010E022E532E24DEB5EE360E172E285E12D
:1014400092E20E9431421F910F91FF90EF90089518
:10145000CF92DF92EF92FF920F931F93CF93DF9380
:10146000CDB7DEB7CDB6DEB68091B804811103C02A
:101470006BEA74E002C068EB74E0FB0101900020AD
:10148000E9F7CF01861B970B01962DB73EB7281BB6
:10149000390B0FB6F8943EBF0FBE2DBF0DB71EB768
:1014A0000F5F1F4F80E2EDB7FEB78183C801019641
:1014B0000E94E3BD87E0E82E82E2F82E29E632E2C0
:1014C00046E75AE869E072E28EE392E20E94314216
:1014D0000FB6F894DEBE0FBECDBEDF91CF911F9147
:1014E0000F91FF90EF90DF90CF9008958BEA94E0FA
:1014F0000E94186A0E94F1800C941753AF92BF9219
:10150000CF92DF92EF92FF920F931F93CF93DF93CF
:10151000CDB7DEB7EB970FB6F894DEBF0FBECDBFE9
:1015200080918804882349F18BE59DE00E94BF7477
:101530008BE1EBE5FDE0DE01919601900D928A953D
:10154000E1F700E010E048EB54E0BE016F5F7F4F31
:10155000CE0181960E945C7218163CF4CE01019671
:101560000E94D26B080F111DEECFCE0181960E9412
:10157000B3761093D30C0093D20C0E94DB41A09061
:101580008504B12CA11020C08091870481110CC06A
:101590008091830410928304882331F00E94F980A3
:1015A00080919D04811129C180910E02882361F0F0
:1015B00081E090918704911180E004E024E040EA0A
:1015C00052E26B2D0E940E338091330F85FD10C0C7
:1015D00083FF0EC081E0A81225C08091870481306E
:1015E00079F48091830410928304811103C008C0B0
:1015F00011E019C00E94D08980919D048111FDC025
:1016000080910E02882309F47EC081E090918704C6
:10161000913009F080E000E22EE34BE852E26B2DBE
:101620000E940E3312E080910E02882309F46CC0F0
:1016300001E0010FC12CD12C1FEF100F8091D20CB3
:101640009091D30CC816D90608F05EC0A11256C0FE
:1016500001977C01EC18FD088BE59DE00E94BF74AA
:101660008BE1EBE5FDE0DE01919601900D928A950C
:10167000E1F7F12C48EB54E0BE016F5F7F4FCE01E4
:1016800081960E945C72181694F4CE0101960E9415
:10169000D26B882379F3EF1008C0BE016F5F7F4FD4
:1016A0008BEA94E00E94A06E02C0F394E3CFCE01D7
:1016B00081960E94B3768091330F9091870484FFC6
:1016C00009C0911310C0809183041092830481118A
:1016D00023C009C0911385C08091830410928304B4
:1016E000811177C07EC080910E02882339F081E09D
:1016F000911380E041E06B2D0E9419418FEFC81AD1
:10170000D80A0F5F99CF12E0B394A39485E0B81282
:1017100039CF1093860471C019821C8280915E0DAE
:10172000811103C066E77DE002C06BE57DE021E04A
:101730004BEA54E0CE0101960E94B976882319F154
:101740008BE1FE013196ABE5BDE001900D928A95EB
:10175000E1F78091330F8F7D8093330FA091290F94
:10176000AA30E0F481E08A0F8093290F8BE18A9FF1
:10177000D0011124A55EB14FEBE5FDE001900D9283
:101780008A95E1F70BC00E94D2286BEA74E085E7E6
:1017900092E20E94BB288AE00E94A528CE01019611
:1017A0000E94B3761092850482E090E0A0E0B0E061
:1017B00080938D0490938E04A0938F04B093900433
:1017C00081E080939D041092CD0C83E080930E0203
:1017D00014C088E29AE80E94F2AD80919D048111C4
:1017E0000CC080910E02882309F488CF81E090918B
:1017F0008704911380E040E07ECFEB960FB6F8941B
:10180000DEBF0FBECDBFDF91CF911F910F91FF9033
:10181000EF90DF90CF90BF90AF900895CF92DF927E
:10182000EF92FF920F931F93CF93DF930E94DB41C0
:10183000C091850410E08AE1E82E82E2F82EC11101
:1018400020C08091870481110CC080918304109284
:101850008304882331F00E94F98080919D048111D6
:10186000B3C180910E02882361F081E090918704DA
:10187000911180E004E024E04DE552E2612F0E94E6
:101880000E339091D3048091330F913021F082FB7D
:10189000DD27D0F901C0D1E083FBCC24C0F883FF61
:1018A00004C00E944828D82E01C0D12CDD2359F154
:1018B000C13061F480918704813009F025C18091A5
:1018C000830410928304811119C11EC1C23061F4D6
:1018D00080918704823009F08DC08091830410923A
:1018E000830481117FC086C0C33009F047C0809156
:1018F0008704833009F023C180918304109283040C
:10190000811115C11CC10E945628882371F0C13075
:1019100071F480918704813009F027C1809183049C
:101920001092830481111BC120C1D1E001C0D2E01B
:10193000DC1322C0809187048D130EC08091830434
:1019400010928304882341F08FE692E90E94F2AD61
:1019500080919D04811138C180910E02882361F02D
:1019600081E0909187049C1380E003E02EE34FE830
:1019700052E2612F0E940E33DF5F01C0D4E0DC131E
:1019800022C0809187048D130EC080918304109231
:101990008304882341F083ED9FE80E94F2AD80919B
:1019A0009D04811111C180910E02882361F081E0B4
:1019B000909187049C1380E003E02EE34BE252E217
:1019C000612F0E940E3381E08D0F8C1326C0809111
:1019D00087048C13E5C080918304109283048111E5
:1019E000D7C0DEC08FE09AE80E94F2AD80919D04DE
:1019F0008111EAC080910E02882309F4E3C081E0DE
:101A000090918704923009F080E003E02EE342E5F4
:101A100052E2612F0E940E33D4E082E08D0FCC2081
:101A200009F44CC0D11062C08C1320C0909187047F
:101A30009C130EC08091830410928304882341F08C
:101A4000F092A50AE092A40A80919D048111BCC085
:101A500080910E02882351F081E09C1380E000E227
:101A60002EE34EE152E2612F0E940E3383E08D0F90
:101A70008C1322C0809187048C130EC08091830444
:101A800010928304882341F08EE79AE80E94F2AD19
:101A900080919D04811198C080910E02882361F08D
:101AA00081E0909187049C1380E003E02EE342E301
:101AB00051E1612F0E940E3384E017C08C1314C0D3
:101AC000909187049C1302C01092830480910E02AF
:101AD000882351F081E09C1380E000E22EE344E48F
:101AE00052E2612F0E940E3383E08D0F1F5FCF5FA4
:101AF000153009F0A4CE8093860466C00E94A93EEA
:101B000080919D04811160C080910E02882309F4A8
:101B100059C081E090918704913009F080E000E2A3
:101B20002EE345E850E1612F0E940E334BC087E45D
:101B300090E90E94F2AD80919D04811145C0809191
:101B40000E02882309F43EC081E09091870493300F
:101B500009F080E003E02EE34DE452E25ACF0E9408
:101B60001C3880919D0481112FC080910E02882322
:101B700069F081E090918704913009F080E000E203
:101B80002EE347E352E2612F0E940E33D2E0F4CEFF
:101B900086EF94E80E94F2AD80919D04811114C0FB
:101BA00080910E02882309F438CF81E09091870458
:101BB0009C1380E003E02EE349EF51E2612F0E9485
:101BC0000E332BCFD4E0FFCEDF91CF911F910F9139
:101BD000FF90EF90DF90CF9008953F924F925F92E9
:101BE0006F927F928F929F92AF92BF92CF92DF922D
:101BF000EF92FF920F931F93CF93DF93CDB7DEB792
:101C00002A970FB6F894DEBF0FBECDBF9A8789879B
